:1000000000800020BD010000F5700200C1700200F8
:10001000C1700200C1700200C1700200C170020014
:10002000C1700200C1700200C1700200F5700200D0
:10003000F5700200C17002000592020009920200F0
:10004000F5700200F5700200F5700200F570020014
:10005000F5700200F5700200F5700200F570020004
:10006000F5700200F5700200F5700200F5700200F4
:10007000F5700200F5700200F5700200F5700200E4
:10008000F5700200F5700200F5700200F5700200D4
:10009000F5700200F5700200F5700200F5700200C4
:1000A000612C02006D2C0200F5700200F570020058
:1000B000F5700200F5700200F5700200F5700200A4
:1000C000F5700200F5700200F5700200F570020094
:1000D000F5700200F5700200F5700200F570020084
:1000E000F5700200F5700200F5700200F570020074
:1000F000F5700200F5700200F5700200E17F020069
:10010000F5700200F5700200F5700200F570020053
:10011000F5700200F5700200F5700200F570020043
:10012000F5700200F5700200F5700200F570020033
:10013000F5700200F5700200F5700200F570020023
:10014000F5700200F5700200F5700200F570020013
:10015000ED9302000194020015940200299402001C
:10016000F570020091820200F5700200F570020045
:10017000F5700200F5700200F5700200F5700200E3
:10018000F5700200F5700200F5700200F5700200D3
:10019000F5700200F5700200F5700200F5700200C3
:1001A000F5700200F5700200F5700200F5700200B3
:1001B000F5700200F5700200F5700200564B4CF22B
:1001C000205210B51A804DF628121A8000BF00BFC9
:1001D00026F094FF514B4FF010621A60504A9A601B
:1001E000504ADA60504A136813F4807301BF4F49D4
:1001F0000B604FF4A85313604D4B4E491A7810070B
:1002000042BF1A7842F008021A704B4B2A221A7029
:100210004A4A4B4B8B4204D252F8040F43F8040B6A
:10022000F8E7484B484A0021934202D243F8041BA6
:10023000FAE7464A4648002350F8231042F82310B4
:1002400001336F2BF8D1434B434A802103F8011B44
:100250009342FBD1414B3D4A1A60414B8A221A70AE
:10026000A3F5805324225A70A0221A709A7991071C
:10027000FCD59A79D206FCD43A4A937903F00C0360
:10028000082B384BF9D103221A7140225A719A79FE
:100290009406FCD533498A79324B5006FBD5324A55
:1002A000324911600221516020221A709A7902F0BD
:1002B0000C020C2AFAD12E4B2E4A1A602E4B2F4AD2
:1002C0001A6000225A60072243F8042C2C4AC3F813
:1002D0000C2D62B627F04CFB144B1B68DA0705D5D2
:1002E000284827F005F9284B284A1A60284B1B7824
:1002F0005B0609D5244C254B22689A4204D121483B
:1003000027F0F6F8002323602DF01AFB26F0FCFE00
:1003100029F0FDFBFEE700BF0E20054030800440C1
:10032000823F04000100002B10D0034014D0034092
:1003300002D00740188DFF1F00E00740048D030026
:100340001C87FF1F188DFF1F08DAFF1F0082FF1F89
:100350000000000000E400E05FE400E008ED00E0E1
:100360000050064000400640448004400000030165
:1003700004800440C010050014E000E0FF76010096
:10038000000020201A44BC621CE00340A5C3945A1C
:1003900000F00740FFFFFFFFFFFFFFFFFFFFFFFF32
:1003A000FFFFFFFFFFFFFFFFFFFFFFFFFFFFFFFF5D
:1003B000FFFFFFFFFFFFFFFFFFFFFFFFFFFFFFFF4D
:1003C000FFFFFFFFFFFFFFFFFFFFFFFFFFFFFFFF3D
:1003D000FFFFFFFFFFFFFFFFFFFFFFFFFFFFFFFF2D
:1003E000FFFFFFFFFFFFFFFFFFFFFFFFFFFFFFFF1D
:1003F000FFFFFFFFFFFFFFFFFFFFFFFFFFFFFFFF0D
:10040000FFFFFFFFFFFFFFFFFFFFFFFFDEF9FFFF23
:1004100010B5054C237833B9044B13B10448AFF33E
:1004200000800123237010BD188DFF1F0000000005
:10043000008D0300084B10B51BB108490848AFF305
:1004400000800848036803B910BD074B002BFBD0A0
:10045000BDE81040184700BF000000001C8DFF1FC2
:10046000008D0300188DFF1F0000000070B50568A7
:10047000044628460E4626F08BFD864203D03146C0
:10048000284626F099FD204670BD2DE9F0418046B2
:100490000E4614461AB3012A02D100230B701EE047
:1004A00026F076FD01250746307097B1AC420ADD93
:1004B00008EB050026F06CFD0746192027F042FAEC
:1004C00077550135F1E7002D03DD3544002305F8AC
:1004D000013C192027F036FA0120BDE8F0812046C2
:1004E000BDE8F0812DE9F04112491C4600AF90466D
:1004F000054629F03CF9E31D23F00703ADEB030D9E
:10050000224640466946FFF7C0FF661EE8466C4635
:10051000C8EB04039E4208DD14F8011B284629F0AD
:1005200019FA192027F00EFAF2E72846BD46BDE871
:10053000F08100BFAB150300F0B585B0002401AE1B
:100540001046234609220F463146019402948DF845
:100550000C4029F079FA30462DF0AFFB0130C5B2DE
:10056000E3B29D420AD93B19315D00936846FFF71B
:100570007DFF192027F0E6F90134F1E7284605B0A0
:10058000F0BD26F0C1BC70B5044608460D462DF0FE
:1005900094FB23680246294620465B68BDE870400C
:1005A000184738B50546FFF7EEFF0446284628F001
:1005B00079FF204438BD38B50A220023054628F0CB
:1005C00095FF0446284628F06DFF204438BD26F0EC
:1005D0009BBC002070477047024A136801331360C8
:1005E000704700BF14B9FF1F024A536801335360BC
:1005F000704700BF14B9FF1F2C4B2D4A1B7810B554
:100600002C4C3BB12388C3F309035BB113889BB225
:1006100043B10AE02388C3F30903BBB113889BB23B
:10062000A3B129E02449002312E02188128889B26D
:1006300092B29202642392FBF3F391FBF3F203FB79
:10064000121383B91C4B1A786AB911E01A490123B5
:100650000B7013889BB223B1184B0978187826F0D9
:10066000CDFF00232380238801339BB2238010BD5C
:1006700001221A70197813E02388128899B292B275
:100680009202642392FBF3F391FBF3F203FB121348
:10069000002BE8D1084A11780029E4D013701178B2
:1006A000064B187826F0AAFFDDE700BF28C4FF1F1D
:1006B000C6C5FF1F1CB9FF1FDF8EFF1F0EB9FF1F2E
:1006C00010B5044628F070FE204610BD10B5034B4F
:1006D0000360044621F0F0FB204610BD28270300EC
:1006E00010B50446FFF7F2FF2046142129F01BFA4B
:1006F000204610BD10B5034B0360044621F0DCFB1F
:10070000204610BD7033030010B50446FFF7F2FF1A
:100710002046142129F007FA204610BD10B5034BDE
:100720000360044621F0C8FB204610BD4831030099
:1007300010B50446FFF7F2FF2046142129F0F3F923
:10074000204610BD10B5034B0360044621F0B4FBF6
:10075000204610BD142F030010B50446FFF7F2FF2A
:100760002046142129F0DFF9204610BD26F024BCD4
:1007700038B50C46054626F00BFC844205D02146D0
:100780002846BDE8384026F017BC38BD38B50C46C1
:10079000C1F307210546FFF7EBFF0A2027F0D2F847
:1007A000681CE1B2FFF7E4FF0A20BDE8384027F0FB
:1007B000C9B810B5029C521AE41AA242A0EB01007B
:1007C000C6BF04FB00000132604390FBF2F0184406
:1007D00010BD10B5029C521AE41AA242A0EB01000F
:1007E000C6BF04FB00000132604390FBF2F01844E6
:1007F00010BD10B50C4604220146204626F0FEFB33
:10080000204610BD10B5C0F3072104464FF4D17047
:10081000FFF7ACFF0A2027F095F8E1B240F2A310F1
:10082000FFF7A4FF0A20BDE8104027F08BB8F8B509
:100830000C460E1D0D46471A781926F0A9FB05F83F
:10084000010BB542F8D12046F8BD26F0A1BBFFFF51
:1008500010B50B4C2378042B0DD94FF4CC70FFF757
:10086000F4FF0322212888BFFF20064926F026FF37
:10087000054828F099FD23780133237010BD00BF8F
:10088000A0C5FF1F256F0100388EFF1F08B540F27D
:100890009710FFF7DAFF012126F0DEFE40F29710F5
:1008A000FFF7D3FF002126F0A9FEFA2027F04AF82F
:1008B00040F29710FFF7C9FF002126F0CDFE00207F
:1008C00008BD38B50546FFF7C0FF0446681CFFF7B2
:1008D000BCFF0146204628F007FF00B238BD29F0D2
:1008E00027B829F029B808B5FFF74DFE08BD002349
:1008F0000A2228F0FBBD28F034BE00230A2228F08B
:10090000F5BD9DF80010009128F036BE38B50546BB
:1009100028F027FE0446284628F0C4FD204438BDB0
:1009200038B50546FFF7E9FF0446284628F0BAFD2A
:10093000204438BD002A10B40BDB074B541E9C42E8
:1009400007D830235A43013A232A02D910BC28F091
:10095000E3BC002010BC7047575555051FB5002457
:10096000B0F90C30B0F90A20B0F908100294032451
:100970000194B0F90E400094406824F0E3FC04B008
:1009800010BD0B8883834B88C3838B880384704797
:1009900030B502F11704013900F117030444A342F2
:1009A00004D011F8015F03F8015FF8E780F8242014
:1009B00030BD0022FF238281438200F114025030B7
:1009C00022F8023F8242FBD17047FFFF10B5044678
:1009D00021F09EFA014B2360204610BD142F030026
:1009E00010B5044621F094FA014B2360204610BD57
:1009F0007033030010B5044621F08AFA014B2360DE
:100A0000204610BD4831030010B5044621F080FA9D
:100A1000014B2360204610BD2827030070B586B027
:100A20008DE80F00194B9DF828601A78052A1D469D
:100A300007D06946164821F08DFC011C18BF012122
:100A400000E000212B78032B1ED1EEB11148FFF7F7
:100A500052FF009A10490F4828F03BFD0DF10704A2
:100A60000DF10F0514F8012F0C490A4828F031FD4B
:100A7000AC42F7D10A4B9DF805201B680593059BF6
:100A80000849044828F025FD06B070BD04B9FF1FD1
:100A90003CC5FF1F848AFF1FDC140300E21403001F
:100AA0004CD8FF1FE81403002DE9F74F40F219104E
:100AB000FFF7CBFE092811D1C14BC24D01221A719B
:100AC00008225A71C04A1A600022AC5CBC499818CE
:100AD0000132082A0472F8D10023D1E00A2859D142
:100AE000BA4CBB4E082363714FF4DE632360337846
:100AF0001B0103F0100323723378DB0003F01003B3
:100B0000A37233789B0003F01003237333785B00E8
:100B10000025012703F0100325716572E5726573E6
:100B2000E573A373009794E80F00FFF777FFA94AD6
:100B3000657240F2F16323601378E5729B0003F065
:100B40003C032372137865731B099B00A372257302
:100B5000E573A573009794E80F00FFF75FFF40F27D
:100B6000F26323603378657203F0100323723378E5
:100B7000E572FB4003F01003A372337865739B08A2
:100B800003F0100323733378E573DB091B01A373B0
:100B900000974DE00B284ED18F4F8C4C8F4D97F81E
:100BA00000800023A8262371082306FB08586371E0
:100BB0004FF4C263D8E90E0123602CF063F9C0F34F
:100BC00007202072D8E90E012CF05CF997F801801B
:100BD000607206FB0858D8E90E012CF053F9C0F3F7
:100BE0000720A072D8E90E012CF04CF997F802808A
:100BF000E07206FB0858D8E90E012CF043F9C0F367
:100C000007202073D8E90E012CF03CF9FB786073C3
:100C100006FB0355D5E90E012CF034F9C0F307208B
:100C2000A073D5E90E012CF02DF90123E073009398
:100C300094E80F00EFE20C2825D1644964480023B2
:100C40000B7108234B714FF4E0630B60A5230B720B
:100C500003780478027812F0010F027802F00102A2
:100C600003F0040342F0040204F0020442EA8302A7
:100C70000CBF0225002542EA84032B434B7201235B
:100C800000930FC9C7E2082840F0FB804F4C524F39
:100C9000524E6071002323713B78A82202FB03634C
:100CA00093F89030FBB1DFF83881D8F804504FF456
:100CB0008E70FFF7CAFDADB202234246D9B2884218
:100CC0000AD958F82310A94288BF52F8235003F1DB
:100CD000010388BFADB2F1E741F288335D43AB1247
:100CE000AD14257263727B78A82202FB036393F82C
:100CF0009030FBB1DFF8E880D8F898514FF48E704F
:100D0000FFF7A3FDADB202234146DAB290420AD901
:100D100003F16502013358F822E0AE4584BF51F873
:100D20002250ADB2F1E741F288335D43AB12AD140E
:100D3000A572E372BB78A82202FB036393F890309C
:100D4000FBB1DFF89C80D8F82C534FF48E70FFF77E
:100D50007CFDADB202234146DAB290420AD903F1DA
:100D6000CA02013358F822E0AE4584BF51F8225040
:100D7000ADB2F1E741F288335D43AB12AD14257398
:100D80006373FB78A82202FB036696F8903083B366
:100D9000134ED6F8C0544FF48E70FFF756FDADB227
:100DA00002233146DAB290421CD903F22F120133EA
:100DB00056F82270AF4284BF51F82250ADB2F1E72D
:100DC00074C5FF1F8FC5FF1F01C0CC1CB4C5FF1F1A
:100DD00001B9FF1FDD8EFF1F06B9FF1F008FFF1F28
:100DE0000CCAFF1F41F288335D43AB12AD14A573EB
:100DF000E3734FF4C863236001230093A84D94E884
:100E00000F00FFF70BFE05F108062B46002203F842
:100E1000012F9E42FBD1A34FA3483A7890F800E0FF
:100E200040F2416302F00F02236041F28831531C0B
:100E300091FBF3F20EF00F0313FB02F39BB263720C
:100E40001B1223723B7802781B09013391FBF3F1EB
:100E5000130913FB01F39BB2E3721B12A37201236C
:100E6000009394E80F00FFF7D9FD002305F8013F38
:100E7000B542FBD140F2426323608C4B1B78237355
:100E80009DE0012840F0A980894C8A49002308226E
:100E9000237162712372884A6372A372E3722373AF
:100EA00063730B78A82000FB0323894693F89070A6
:100EB0009046EFB1814E75684FF48E70FFF7C5FC18
:100EC000ADB202233246D9B288420AD956F823106D
:100ED000A94288BF52F8235003F1010388BFADB285
:100EE000F1E741F288335D43AB12AD1425726372B2
:100EF00099F80130A82202FB038898F890605EB34D
:100F0000DFF8B881D8F898514FF48E70FFF79DFC48
:100F1000ADB202234146DAB290420AD903F165022A
:100F2000013358F822E0AE4584BF51F82250ADB2EB
:100F3000F1E741F288335D43AB12AD14A572E37261
:100F40005FB95E4ED6F898514FF48E70FFF77DFC76
:100F5000ADB2022331461CE05FB3584F7D684FF4B9
:100F60008E70FFF772FCADB202233A46D9B28842C6
:100F70000AD957F82310A94288BF52F8235003F129
:100F8000010388BFADB2F1E7AD102573002ED8D1B3
:100F90000FE0DAB290420AD903F16502013356F844
:100FA0002270AF4284BF51F82250ADB2F1E7AD10CC
:100FB000657340F2666323603C4B1B78A373404D1E
:100FC0002B78E3730123009394E80F00FFF726FDCD
:100FD0002B780133DBB22B701FE102282ED1314F69
:100FE000314E334B39783578082201F00F015A71B0
:100FF00040F26C7241F288301A604A1C90FBF2F1A8
:1010000005F00F0212FB01F292B25A7212129A729A
:10101000264A1278DA723A7831781209013290FB56
:10102000F2F00A0912FB00F292B200241A731212B3
:101030001C711C725A739C73DC732EE003280ED152
:101040001B4B0821597140F202611960FF2119728E
:101050001649002208781A715A72987217E005280A
:1010600030D1134B0821597140F2F97119600F49C1
:10107000087800F00100187208780978C1F380013F
:101080000022C0F34000997207491A71587209781A
:10109000D9721A735A739A73DA730122B9E000BFD6
:1010A000BBC5FF1FDE8EFF1FDD8EFF1F01B9FF1FB7
:1010B000B4C5FF1F06B9FF1F008FFF1F0CCAFF1F1B
:1010C000DC8EFF1F062840F09A80554C554FDFF804
:1010D0006881DFF868A1082363714FF4C863236057
:1010E000514B1A7802F0010222721A78C2F34002C0
:1010F00062721A78C2F38002A2721A78C2F3C00236
:10110000E2721A78C2F3001222731A78C2F3401204
:1011100062731A781B78DB09E373C2F38012012330
:1011200000262671A273009394E80F00FFF776FC67
:1011300040F24163236025464FF0A8094FF0650B4C
:1011400016F8083009FB037393F89030E3B14FF4BD
:101150008E70FFF77AFB0021002200230BFB06FCB8
:1011600001315FFA81FE704508D90CEB010E5AF887
:101170002EE012EB0E0243F10003F1E7013892FB7F
:10118000F0F21312237262720136042E04F102048B
:10119000D6D10123009395E80F00FFF73FFC40F202
:1011A00042632B60214B002103F1080203F8011F69
:1011B0009342FBD11E4E1F4C3278207802F00F0272
:1011C000531C41F2883191FBF3F200F00F0313FB43
:1011D00002F39BB22B721B126B72337822781B09BD
:1011E000013391FBF3F1130913FB01F39BB2AB72D3
:1011F0001B12EB720123009395E80F000BE0072808
:101200000BD1074B00221A714FF4407101225A7121
:10121000196000920FCBFFF701FC03B0BDE8F08F1F
:10122000B4C5FF1F008FFF1F01B9FF1FBBC5FF1F04
:10123000DE8EFF1FDD8EFF1F06B9FF1F0CCAFF1FCA
:101240002DE9F347C04CC14FC14E3B780821617175
:101250004FF4D0712160BF490878884601284FF0CB
:10126000400161720BBFE921B321A172A1720CBFD1
:101270000321102103F00F030022E1721033FE213D
:10128000E3732271227221736173A27300230093AE
:1012900094E80F00FFF7C2FB4FF420730120236096
:1012A000FFF7D3FAFF28054600F06A813378012B57
:1012B00040F06681A84AA82303FB0025D5E90E016A
:1012C0000022A64B2BF006FB2BF0B4FD00B2C5B2FA
:1012D000C0F307200023FE22012123726272A5724F
:1012E000E07223736273A173E273009394E80F00BA
:1012F000FFF794FB4FF4227323603378012B0ED158
:101300009749984B0022D1E900012BF031F90022D6
:10131000954B2BF009FC2BF0B5FDC0B200E0C720C7
:1013200092490A78894602F0FF031AB90D22227207
:10133000607210E00B78012B01D1702308E00B786C
:10134000022B01D18F2303E00B78032B0CD1E9236F
:10135000237260720023A372E37223734D236373BD
:10136000FF23A373BF23E373002694E80F000096C6
:10137000FFF754FB0122A2727D4AE6724FF0FE0A8B
:101380004FF4287310782360642280233146CDF80F
:1013900000A0637226736673A673E673FFF709FAFB
:1013A000207294E80F000096FFF738FB4FF460734B
:1013B000236058236372FD23E37207232373F02312
:1013C000267284F80AA06373A67384F80FA094E8C9
:1013D0000F000096FFF722FB99F800105A4D634A60
:1013E0004FF49063236001F0FF0351B996222A72F3
:1013F0002C22AB72EB722B736B73AB736A72BA23D2
:1014000028E01378012B0AD1E8232B722C236B726E
:10141000AE72EE722E736E73AE73C4231AE013783D
:10142000022B0AD161232B722C236B72AE72EE72E7
:101430002E736E73AE734D230CE01378032B0AD119
:101440001B232B722C236B72AE72EE722E736E7393
:10145000AE733723EB730023009394E80F00FFF77C
:10146000DDFA4FF4916323603B78424A364D03F036
:101470000F030F2B14BFDBB20E237821D25CE17275
:101480000B322272FE226272A27222731B010022B0
:101490006273A273E373009294E80F00FFF7BEFA41
:1014A0004FF49463236098F80030012B4FF0B2039F
:1014B0002B7205D110226A72AB72EA722B7305E0AF
:1014C00011226A72EA72AB722B7310226A73AB73C9
:1014D000EA73002594E80F000095FFF79FFA4FF498
:1014E000B16323600823237278236572A372E572C7
:1014F00025736573A573E57394E80F000095FFF7F6
:101500008DFA3B780133DBB23B703B7803F0FF028E
:101510000BB9194B1A70194A13780133DBB21370E7
:101520001378032B07D999F800300133DBB289F81F
:1015300000300023137099F80030032B3AD90B4B7D
:1015400000221A7036E000BF74C5FF1F30C5FF1FB0
:1015500002B9FF1FF18EFF1F008FFF1F0000104018
:10156000D891FF1F000048400000E83F348EFF1F65
:10157000C0C4FF1FC6260300E28EFF1F358EFF1F6B
:101580003378022B13D00D49A82303FB0511D1E9B1
:101590000E0100220A4B2BF00FFC18B1FF2D04D0D6
:1015A000002005E06020FF2594E6602092E661209F
:1015B00005468FE602B0BDE8F08700BF008FFF1F31
:1015C00000407F4008B54FF4CC70FFF73EF9002192
:1015D00026F042F84FF4CC70FFF737F9012126F0DE
:1015E0000DF80A20BDE8084026F0ACB90B7903716C
:1015F00030B58B6883600B4600F11A0413F80C2F8A
:10160000027300F10D0213F8015F02F8015B9442CE
:10161000F9D1CB69C36130BD10B5042894BF04462D
:1016200003242146084821F005FC032C074A084BF7
:1016300015BFF0214FF4A0711180118014BF4FF439
:10164000A072F0221A8010BD58C6FF1F0488FF1F29
:101650003C88FF1F2DE9F041044690B003200F465F
:10166000FFF7DAFF012C25D1974B98481B680493AC
:101670000499974E974DFFF740F997499348FFF724
:1016800032F9002332785C1CDBB29A420FD9A822CF
:10169000022102FB0353D3E90E238C480091FFF78C
:1016A00030F98D498948FFF71EF92346EAE78B494F
:1016B0008648B4E0022C40F0B480894B1B78FF2BA5
:1016C00040F0AF80804E874933680293029B0A68DE
:1016D0009A1A854B18784EF6602343439A4202D9F2
:1016E000FF2F00F0A5800024804B04AA03F1080C12
:1016F0001546186859689646AEE8030008336345F6
:101700007246F6D118689988DFF804829B79CEF882
:101710000000AEF804108EF8063098F80030FF2F65
:1017200018BF3B4630338DF81930BCB1704967485B
:10173000FFF7D9F898F800106448FFF7D8F86D491A
:101740006248FFF7D0F829466B481FF073FA08B1DA
:101750006A4900E06A495D48FEF723FF69481FF0C7
:10176000D8F898B9294664481FF058FA132300287E
:101770002A46614908A808BF01241FF00BFA08A9EE
:101780006048FFF733FF08A81FF080F8FCB15E49FE
:101790005C484F4DFFF7A7F800242B78E1B299423F
:1017A00004F101040FD2002208A818F077FD08A95F
:1017B000544827F057FE08A827F099FF464951489A
:1017C000FFF791F8E9E745494E48FEF7EAFE4D4834
:1017D0001FF09FF828B333680893089949483C4E96
:1017E0003C4DFFF78AF83C494648FFF77CF8002358
:1017F00032785C1CDBB29A420FD9A822022102FB8C
:101800000353D3E90E233F480091FFF77AF832499A
:101810003C48FFF768F82346EAE730493948FEF7C5
:10182000C0FE3A4B1878FFF7F7FE10B0BDE8F08124
:1018300033680393364D039B0B602B780133DBB287
:10184000092B00D900232B702978DFF8D8804FF4BA
:10185000D070FEF78DFF2F4821F008FC09224FF6CB
:10186000E0738DE80C0032211F230122294823F068
:1018700011FD0121274821F084FB012400230222CD
:101880003621244888F8004022F054FE00212148E7
:1018900021F07DFB20491F48FFF725F829781D48D6
:1018A000FFF725F81D4A1E49B2F90020B1F90010D2
:1018B0001848002322F03EFE0021164821F067FB65
:1018C000002388F800300FE74CD8FF1F848AFF1FE1
:1018D0002AC4FF1F008FFF1F5C150300AB15030018
:1018E0000B88FF1F34C5FF1F68C5FF1F1E150300AF
:1018F000FB1403000F1503002CD5FF1F161803005F
:10190000F21F0300F8C4FF1F131503002688FF1FF2
:101910003F88FF1F58C6FF1F211903003C88FF1F87
:101920000488FF1FC8C5FF1F2DE9F04F814689B00D
:101930006848694D694F8846002121F028FB012144
:10194000644821F01EFB0320FFF766FE0B2444F2DF
:10195000082301930094BC23012246215D4823F013
:1019600099FC46F22C33019300940F230122372176
:10197000584823F08FFC002302223B21554822F0D7
:10198000D9FD57495348FEF7AEFF2C782CB1FF2CF8
:1019900008BF3C78013CA4B200E0FF24514A039206
:1019A000702606FB0926464446F22C3A337E494807
:1019B000A34214BF53464FF4FC634FF00B0B01934B
:1019C000012233234B21CDF800B023F063FC002328
:1019D00002224D213F4822F0ADFD3B780822E1B2C2
:1019E00004A818F05BFC04A93A4827F03BFD04A8C2
:1019F00027F07DFE327E2B783648CDF800B09A4233
:101A000014BF53464FF4FC63019301223323832117
:101A100023F040FC0023022285212E4822F08AFD7B
:101A20003B782978082204A818F038FC04A9294832
:101A300027F018FD04A827F05AFE2C78FF2C06D0BA
:101A4000264B1B78013B9C4203D0013402E000246A
:101A500000E0FF24039A1F48702303FB0929C844B0
:101A600046F22C3698F818300B25A34214BF3346A3
:101A70004FF4FC630193009533230122BB2123F033
:101A800009FC00230222BD21124822F053FD3B78BD
:101A90000822E1B204A818F001FC04A90D4827F0BF
:101AA000E1FC04A827F023FE8DE860000F2301224B
:101AB000F321084823F0EEFB00230222F72105481A
:101AC00022F038FD08490348FEF70DFF09B0BDE8D4
:101AD000F08F00BF58C6FF1FA0C5FF1F2AC4FF1FFD
:101AE0002D150300B8BCFF1F2F150300013808B5E2
:101AF000052810D8DFE800F0050305090709522181
:101B000004E0062102E0D22100E0C6210648BDE83B
:101B1000084024F07BBED221034824F077FE034B1B
:101B200000221A7008BD00BF18C5FF1FF08EFF1FEE
:101B300010B5074A0023702101FB0324D8B294F8A2
:101B400058401CB10133112BF6D1FF2010BD00BF4E
:101B5000B8BCFF1F38B5074D0024281990F858303D
:101B60001BB1FF2200211EF06FFA7034B4F5EE6F46
:101B7000F3D138BDB8BCFF1F10B58CB01B49684607
:101B800027F0F5FD5323009A194904A81FF002F825
:101B900004A91848FFF72AFD04A81EF077FE0024C8
:101BA0002046FEF752FE013402461349114827F041
:101BB00090FCB4F5BE7FF3D110490E48FEF793FEBA
:101BC0004FF4C8742046FEF740FE013402460A492D
:101BD000084827F07EFCB4F5167FF3D105481EF0C7
:101BE0008CFE684627F083FD0CB010BD3115030054
:101BF0002CD5FF1FF8C4FF1FE21403004215030099
:101C00000D4B03600B7903718B6883600B7B03734F
:101C100003460A4A30B543F80D2B01F1190401F1CE
:101C20000D0252F8045B43F8045BA242F9D112782A
:101C30001A70CB69C36130BD04870300E8770300E5
:101C40001B4B73B501220446014600201A7018F0A0
:101C5000FDFA10B1174B1B78DBB9174B1B782BB370
:101C60002146012018F0F2FA00B32146022018F0B4
:101C7000EDFAD8B90121204618F0D4FA0F4A1378AA
:101C8000013313700E4B1B6801930E4B019A1A60BF
:101C90000CE00D4B14201D6827F041FF0646FEF7AF
:101CA00095FE3146284620F0CFF9D6E702B070BD48
:101CB00003B9FF1F3B88FF1F31C5FF1FAAC7FF1FC6
:101CC0004CD8FF1F1CD5FF1F98D7FF1F2DE9F347E6
:101CD000384EA82202FB00678246D7E90E4500294C
:101CE0003ED097F89130FF2B08D002FB0361D1E979
:101CF0000E01D7E926232BF073F8D0B1D7E9168966
:101D0000204642464B4629462BF06AF830B9D7E9BF
:101D10001223204629462BF059F850B10022002307
:101D2000404649462BF03EF818B95046FFF788FF69
:101D300016E0A82303FB0A6393F8A12082B193F86D
:101D4000A2206AB11C4A1D48126801921C4A0199DE
:101D500012680078891A642210FB02F2914222D89C
:101D6000A82707FB0A67D7E91423204629462BF04A
:101D700041F810B1C7E9144519E0D7E910892046A8
:101D800042464B4629462BF017F830B90022002373
:101D9000404649462BF006F848B1A82303FB0A66E3
:101DA000C6E9104503E0002283F8A220D8E702B07C
:101DB000BDE8F087008FFF1F4CD8FF1F31C5FF1F04
:101DC0001CD5FF1F73B5144603EB430203EB8203DC
:101DD000CA1805B200230C208DE809000E46052321
:101DE00012B229460B4823F055FAFF2C0FD004EB12
:101DF000440204EB82020B214FF6E07332448DE87B
:101E00000A0012B205232946024823F043FA02B021
:101E100070BD00BF58C6FF1F022938B503460846EB
:101E200005D1FF222C21FFF7CDFF002038BD1D4A30
:101E30001D491278A82404FB021494F86840012C70
:101E400014BF0B240D24013C03B918B3A34203DBD8
:101E500001280CD100241EE020B95C1EE4B2042C41
:101E60000AD114E0012804D15C1CE4B202E000288D
:101E7000F3D01C46042C0CD0072C0CD1A82505FB54
:101E80000212516840F6FF72914204D008B9013C39
:101E900000E00134E4B222462C210220FFF792FF39
:101EA000204638BDA0C5FF1F008FFF1F2DE9F0435E
:101EB0000B88FF2B89B005460C4617460CD1488885
:101EC000092809D8874B8A88C0B21870864B1A70C7
:101ED000FFF7A2FB002001E12389844E092B0ED1DC
:101EE000834A142303FB052301221A7440F2AB102A
:101EF000FEF7ABFC7F4B18701B78A38154E00B2BD3
:101F00003CD16389092B04D17B4B7C4A1B78DBB223
:101F100005E00A2B0AD1784B794A1B78DBB212789C
:101F2000934211D00023A381E28113E00B2B05D152
:101F3000714B1B78FF2B65D0002364E00C2B09D17B
:101F40006D4B1B78FE2BF6E70122A2816D4A9BB2F6
:101F50001380E3816C4B93F80080B8F1FF0F0FD032
:101F6000654B1A78642A0BD818782AF03DFC674B29
:101F7000A82202FB0838C8E90E0101E0052B13D1A5
:101F80003A78002A40F09F8070236B43F2544FF060
:101F9000700808FB05684FF0000988F8089038467B
:101FA0002BF08BFE08F80090702303FB0566638915
:101FB000ADF818300125A389ADF81A3006A9E389D8
:101FC00086F858503046ADF81C30FEF7DAFC002099
:101FD000A388628821880290207A0190E08800908E
:101FE00030461EF06DF82389112B0ED10320FEF729
:101FF0002CFC474B1B7883425BD908A92A4601F881
:102000000C0D51E00123A381A4E70B2B2FD1638991
:102010000E2B14D13F4F3B7803F0F002A37B134308
:102020003B70397840F2C510FEF7A2FB3B7803F015
:102030000F033384384B1B7803F00F0315E00F2B8D
:1020400037D1344FE2893B7803F00F0343EA0213A0
:10205000DBB23B70397840F2C510FEF789FB3B7864
:102060001B0933842C4B1B781B0973841FE005AFBD
:102070007BB92A4A106805900E3434F8021FFF29F4
:10208000DAB204D0F9540133042BF6D11A4639469A
:1020900014E0072B0DD12846FEF7D7FBFF2808D008
:1020A0008DF814002A4639463046FEF771FC284662
:1020B00014E008A9238A01F80C3D01223046FEF7FE
:1020C00067FC01200AE038462BF0F7FD024670203D
:1020D000394600FB05602BF00DFE58E709B0BDE85E
:1020E000F08300BF2688FF1F0E88FF1FB8BCFF1FAC
:1020F00020B9FF1FF18EFF1F0FB9FF1F00B9FF1F8F
:10210000EAC9FF1FC6C5FF1F0988FF1F008FFF1FF9
:102110002AC4FF1FDE8EFF1FDD8EFF1F98120300F3
:102120002DE9F04FB14DDFF8CCA2002687B00C4668
:1021300000F1FF3900F1BF083746AB4619F8013FFF
:102140003B2B40F07081092F04D10F2E40F2968076
:102150000F2695E02EB37B1E172B22D8DFE813F055
:10216000180024004F005900630070007A008400BA
:1021700021009F00A900B300BE00C800D200DC000F
:10218000E600F400FE00080113011D012B014C01C3
:102190001022002102A82CF089FCA82303FB045381
:1021A00058600023202235E11022002102A82CF0E3
:1021B0007DFCA823C0B203FB04530228187201D18E
:1021C000012208E003280BD0042801D1022202E0FA
:1021D000072803D10522864B1A70E2E7082802D1AE
:1021E000834B1870DDE7092801D10622F3E70A289E
:1021F00001D10722EFE70B28D3D10922EBE70A220E
:10220000002102A82CF052FCA82303FB04535872AF
:10221000C7E70A22002102A82CF048FCA82303FBF0
:1022200004539872BDE70A22002102A82CF03EFC5C
:10223000A823003003FB045318BF0120D872B0E775
:102240001022002102A82CF031FCA82303FB045328
:102250001873A6E71022002102A82CF027FCA8235F
:1022600003FB045318619CE70A22002102A82CF00A
:102270001DFCA82303FB0453187592E7002E90D091
:10228000A8236343E818324602A9153001932BF0C6
:1022900031FD019B2B441E440023737581E700210F
:1022A00002A82CF069FBA82303FB0453C3E90A012D
:1022B00077E7002102A82CF05FFBA82303FB04535F
:1022C000C3E90C016DE70A22002102A82CF0EEFB05
:1022D000A82303FB045383F8680062E7002102A8E7
:1022E0002CF04AFBA82303FB0453C3E91C0158E765
:1022F000002102A82CF040FBA82303FB0453C3E9F0
:102300001E014EE7002102A82CF036FBA82303FB98
:102310000453C3E9200144E7002102A82CF02CFB60
:10232000A82303FB0453C3E922013AE70A22002150
:1023300002A82CF0BBFBA823003003FB045318BFFA
:10234000012083F890002CE7002102A82CF014FB58
:10235000A82303FB0453C3E9120122E7002102A8CA
:102360002CF00AFBA82303FB0453C3E9160118E76A
:102370000A22002102A82CF099FBA82303FB045396
:1023800083F891000DE7002102A82CF0F5FAA823AC
:1023900003FB0453C3E9260103E70A22002102A834
:1023A0002CF084FBA823003003FB045318BF01204A
:1023B00083F8A000F5E60A22002102A82CF076FBA3
:1023C000A82303FB0453002814BF0122002283F832
:1023D000A1201EBF9AF8003001338AF80030A823EC
:1023E00003FB04B3002283F8A220DAE6008FFF1F6C
:1023F00005B9FF1FBBC7FF1F0A22002102A82CF04E
:1024000055FBA823003003FB045318BF012083F8B9
:10241000A300C6E602A9CA5401330F2BFAD1013733
:10242000FFB200262FE10A2B04D00D2B02D0192F6A
:1024300040F01F81A448A82303FB040240F6FF7567
:102440005168A94241D1537A0BB9A04B15E0012B39
:1024500001D19E4B2EE0022B02D19C4B9C7004E1DB
:10246000032B02D1994BDC70FFE0042B02D1974B78
:102470001C71FAE0052B02D1954B1C70F5E0062B80
:1024800001D1944BF9E7072B01D1934BF5E7082BCA
:1024900001D1924BF1E7092B01D1914BEDE70A2BCA
:1024A00001D1904BE9E70B2B01D18F4BE5E70C2BCA
:1024B00002D18D4B5C70D8E00D2B01D18B4BDCE74A
:1024C0000E2B40F0D2808A4BD7E740F6FE75A9422A
:1024D00040F0B880117A062940F0C780517A41B99E
:1024E0004FF4207353600223537293720026814F7E
:1024F0000AE001290DD14FF4207369A7D7E90067DD
:102500005360052353729172C2E90A6700260027BF
:10251000A9E0022902D14FF4227313E003290DD15F
:102520004FF43073744F536000260123C2E90A67E9
:10253000537293725CA7D7E9006794E004290CD129
:102540004FF460736D4F536000260123C2E90A67A0
:102550005372937200266A4F85E005290FD14FF41C
:10256000727353A7D7E900675360002353720123A6
:10257000C2E90A67937250A7D7E9006773E006299A
:1025800003FB04030DD14FF484625E4F5A600222B4
:1025900000265A720122C3E90A679A7200265A4F2E
:1025A0004DE05A7A072A04D14FF484625A6003221C
:1025B0002BE0082A0DD14FF48462504F5A60042258
:1025C00000265A720122C3E90A679A7200264C4F0C
:1025D00035E0092A0AD14FF490625A6004225A72F7
:1025E00001229A722EA7D7E9006724E00A2A06D1B1
:1025F0004FF4B1625A6004225A72012217E00B2A8A
:102600000DD14FF4B1625A600722404F5A72002632
:102610000122C3E90A679A7200263D4F0FE00C2A97
:1026200023D14FF494625A6006225A72022224A7E0
:10263000D7E900679A72C3E90A6700260027C3E951
:102640000C6712E040F6FD7399420ED14FF4B1636E
:102650002E4F536000260723C2E90A6753722C4F9E
:10266000012393720026C2E90C67A82303FB04042C
:1026700010E0A3F12102592A05D806AA32440136F6
:1026800002F8103CF6B2C1457FF458AD0E4AA823BB
:1026900003FB0424606807B0BDE8F08FAFF300804F
:1026A000000000A09999D93F0000000000F08BC005
:1026B000000000C07268E93F00000040DF6759C0B9
:1026C00000000040E17A843F008FFF1F06B9FF1F22
:1026D0004188FF1F3E88FF1F0388FF1F0788FF1FD9
:1026E0000988FF1F4088FF1F3788FF1F0288FF1FD0
:1026F0000A88FF1F0000D03F00001C400000E83F98
:10270000000048C00000E03F000049C00000F03F6A
:1027100000004EC02DE9F04F0246BDB072B6532303
:1027200004A8A1491EF036FA04A81EF0F2F830B150
:102730009E4FDFF8ACA24FF00008B946CEE062B67B
:102740009B499C48FEF7CFF827E1A826DFF874B232
:1027500099496643BD19002358468BF800302BF089
:10276000A4FA2B7A062B06F1100640F0BF803E44F7
:102770000536EB7A01962A7D0092904922460CA8F4
:102780002BF048FA0CA958462BF068FAA82303FB53
:1027900004948B4994F868200CA82BF03BFA0CA900
:1027A00088482BF05BFAD4E91C012AF08BFB0CABB8
:1027B0000822012124F018FD0CA982482BF04EFAC2
:1027C000814980482BF04AFAD4E91E012AF07AFBAD
:1027D0000CAB0822012124F007FD0CA979482BF04D
:1027E0003DFA794977482BF039FAD4E920012AF0EB
:1027F00069FB0CAB0822012124F0F6FC0CA97148FE
:102800002BF02CFA70496F482BF028FAD4E92201FA
:102810002AF058FB0CAB0822012124F0E5FC0CA99E
:1028200068482BF01BFA684966482BF017FA94F8B1
:10283000902066490CA82BF0EDF90CA961482BF00B
:102840000DFAD4E912012AF03DFB0CAB0222012162
:1028500024F0CAFC0CA95B482BF000FA5A495948ED
:102860002BF0FCF9D4E916012AF02CFB0CAB022268
:10287000012124F0B9FC0CA952482BF0EFF994F88F
:1028800091204F490CA82BF0C5F90CA94D482BF00D
:10289000E5F9D4E926012AF015FB0CAB022201214F
:1028A00024F0A2FC0CA947482BF0D8F994F8A31007
:1028B00094F8A13094F8A02000910CA844492BF082
:1028C000A9F90CA93F482BF0C9F93E4904A8FEF725
:1028D0000AF804A81DF073FF08F101089AF8003007
:1028E0005FFA88F4A3423FF630AF4FE06A68394997
:1028F0000CA82BF08FF90CA958462BF0AFF9297BC7
:102900006B7A2A7A0291E97A0191A97A00910CA84E
:1029100031492BF07FF90CA958462BF09FF92A6911
:102920002C490CA82BF076F90CA958462BF096F9F7
:102930002A7D26490CA82BF06DF90CA958462BF0DE
:102940008DF9BA19053225490CA82BF063F90CA9A9
:1029500058462BF083F9D5E90A012AF0B3FA0CABFB
:102960000822012124F040FC0CA958462BF076F9EE
:10297000154958462BF072F9D5E90C012AF0A2FA54
:102980000CAB0522012124F02FFCFBE604A81DF06E
:1029900016FF04A81DF0B1FF62B604A81DF076FF73
:1029A0003DB0BDE8F08F00BF2CD5FF1F008FFF1F8B
:1029B00044150300848AFF1F5B1503005E150300A6
:1029C0009B150300E7C6FF1F5C1503009C15030061
:1029D000A01503007D150300841503009415030062
:1029E0002AC4FF1FF0B5354B1C7891B007460E4640
:1029F000002C60D008230A2231496846FDF772FD99
:102A00000622694604A827F069F82E4908A826F08E
:102A1000AEFE08A904A827F03EF8054608A826F04F
:102A200066FE04A826F063FE65B906232A466946B9
:102A300008A827F033F808A9684626F00DFF08A873
:102A400026F055FE204904A826F091FE694604A808
:102A5000FDF745FF1D4B1B78012B0CBF1C491D4981
:102A600004A8FDF73EFF049D1B4901232A4608A840
:102A70001EF090F89FB11EB11848FFF74BFE0AE018
:102A800008A81DF027FF30B108A81DF0ACFEC0B2A9
:102A900026F00EFBF4E708A81DF02FFF02E0284601
:102AA000FFF738FE08A81DF0F1FE04A826F01FFE6F
:102AB000684626F01CFE204611B0F0BD27D5FF1F4A
:102AC00038C5FF1FCF1A0300AC150300A4C6FF1FB3
:102AD000B2150300B71503002CD5FF1FBC1503006A
:102AE0002DE9F0438DB00E461746984608AC544D7C
:102AF0000C2800F28280DFE800F0071B232B333B19
:102B0000434B535B636B73004E49204626F02FFE08
:102B100046F22C33029314202823009300FB065026
:102B200001943C234246394616F05CFE204682E082
:102B30000DF110094349484626F019FE424956E076
:102B40000DF110093F49484626F011FE3F494EE07D
:102B50000DF110093B49484626F009FE3C4946E084
:102B60000DF110093749484626F001FE39493EE08B
:102B70000DF110093349484626F0F9FD364936E093
:102B80000DF110092F49484626F0F1FD33492EE09A
:102B90000DF110092B49484626F0E9FD304926E0A1
:102BA0000DF110092749484626F0E1FD2D491EE0A8
:102BB0000DF110092349484626F0D9FD2A4916E0AF
:102BC0000DF110091F49484626F0D1FD27490EE0B6
:102BD0000DF110091B49484626F0C9FD244906E0BD
:102BE0000DF110091749484626F0C1FD214920463C
:102BF00026F0BDFD4FF4FC630BE00DF11009114907
:102C0000484626F0B4FD1C49204626F0B0FD4FF69C
:102C1000E073039314202823009342463C23394653
:102C200000FB06500294CDF8049016F080FE20467A
:102C300026F05DFD484626F05AFD0DB0BDE8F08354
:102C400020B9FF1FCB150300D5150300DB150300CA
:102C5000E3150300EB150300F6150300FA15030056
:102C6000021603000B1603001116030019160300C9
:102C70001F160300271603002F16030038B50D4654
:102C80000B49044626F073FD0DB90A490AE0092DE7
:102C900001D1094906E00A2D01D1084902E0072DBA
:102CA00003D10749204626F0DFFD204638BD00BF8E
:102CB000371603003B1603003F16030043160300BC
:102CC00047160300F7B5002A46F22C360C4618BF0B
:102CD0004FF4FC668A1C0623411C054600930196AE
:102CE000032312B209B2134822F0D4FA6B1D04F187
:102CF00008011BB2621C09B200910196194612B27A
:102D00000C4820F0D1FB27B2AB1D09341BB224B212
:102D10003A4619468DE85000064820F0C5FBEB1DE9
:102D20001BB28DE850003A461946024820F0BCFB21
:102D300003B0F0BD58C6FF1F2DE9F34146F22C3316
:102D40000D4604464FF6E071002A0CBF1A460A46AB
:102D5000671C09236E1C073424B236B24FF00008FA
:102D6000019200932AB201B23FB21048073522F017
:102D700091FA2DB22346324639468DE840010B4880
:102D800020F092FB2346324621468DE82001074879
:102D900020F08AFB8DE820013B463246214603485D
:102DA00020F082FB02B0BDE8F08100BF58C6FF1FD3
:102DB000F0B5032087B0FEF72FFC00214C484D4EA4
:102DC00020F0E5F801214A4820F0DBF8484820F0DF
:102DD0004DF900240C238DE8180022460F232146CC
:102DE000434822F057FA3378032B4BD140F2AD1011
:102DF000FDF72BFD002845D03F4F3D886D083E3D37
:102E0000EDB2E30229199BB20134009300220C2396
:102E1000C9B23748A4B222F041FB202CF1D1398845
:102E200049080C204FF478431E398DE80900002230
:102E30003C2309B22E4822F02DFA3C8864083D3428
:102E4000E4B20025EB02611B9BB2009300220C232D
:102E5000C9B22748013522F021FB202DF2D13C8850
:102E600026496408053C02A826F081FCA4B205238B
:102E70000093234802AB0222214617F075FD02A8F9
:102E800026F035FC1F4C3078FEF7C6FB23780B2B61
:102E90002CD01D4B1A78003218BF012201211420BA
:102EA000FFF74AFF194B01211A782320FFF70AFF89
:102EB0000A2246F22C338DE80C00012211460D2324
:102EC0000B4822F0E7F9002302220521084821F0EF
:102ED00031FB2378092B05D902220023114604482F
:102EE00021F028FB21780248FDF701FD07B0F0BD75
:102EF00058C6FF1F2688FF1F0488FF1F4F160300B8
:102F0000B8BCFF1F0688FF1F31C5FF1F3B88FF1F8E
:102F100007B5002A0CBF4FF478434FF4FC630193CC
:102F2000072300930AB2042301B2034822F0B2F946
:102F300003B05DF804FB00BF58C6FF1F012808B5A9
:102F400003D0022803D1044902E0044900E0044907
:102F50000448FDF7C8FC08BD621603005A160300BA
:102F60006916030058C6FF1F2DE9F84306460F46B1
:102F7000DDE908019046994629F0F8FA002200237D
:102F800004460D4629F00EFFE8B942464B4630464E
:102F9000394629F0EBFADDE90A2306460F46DDE95A
:102FA0000C0129F0E3FA02460B463046394629F077
:102FB00091FC22462B4629F0B7FDDDE90A2329F0D2
:102FC000D7FABDE8F883DDE90A01BDE8F883FFFF21
:102FD0002F4B37B501221A7000242E4B054621468F
:102FE0002D481C7021F02AFBFFF7E2FE012D07D1CE
:102FF0002A4B224623F814200134112CFAD11BE06D
:10300000022D19D1264B2448B3F900304FF6FF7238
:1030100001920C220092214622F03CF923460F2215
:10302000DC211D4821F086FA21461B481FF0AFFF26
:103030001C491948FDF757FC4FF6FF7116481FF061
:10304000A6FF194B1B78042B1FD1134820F00EF854
:10305000032111481FF095FF002314220A210E4876
:1030600021F068FA4FF6FF710B481FF090FF0F49EF
:103070000948FDF738FC0A21074800233C2221F0CB
:1030800059FA0B490448FDF72EFC03B030BD00BFD0
:103090003A88FF1F10B9FF1F58C6FF1F2EC4FF1F1D
:1030A0000488FF1F7116030004B9FF1F7616030082
:1030B0008116030073B504B20DB2002316462146F3
:1030C0002A460E4821F036FA0D4B1B7803F0FF021A
:1030D00093B90A232146019200932A461E230748EA
:1030E00022F0D8F8074B05481A783241D30754BF6D
:1030F00005490649FDF7F7FB02B070BD58C6FF1F32
:10310000C8C5FF1FF0C4FF1F971603009A160300DF
:103110002DE9F34107B20FFA81F80023144639462E
:1031200042461A4821F006FA194B1B785BBB194A34
:10313000194D115D2B5D994204D0631CD25CEB5C90
:103140009A4202D1154B1B78EBB100260A238DE879
:1031500048004246394628230C4822F09BF8295D56
:103160000A483346102226F0C1F901340C490748B9
:10317000FDF7B9FB295D05483346102202B0BDE8D2
:10318000F04126F0B3B902B0BDE8F08158C6FF1F88
:10319000C8C5FF1F408EFF1FF0C4FF1F3A88FF1FE6
:1031A000CF1A03002DE9F04F4E4F4F4D4F4B0026E5
:1031B0008DB080460C463E70F2B2052A18D8DFE882
:1031C00002F0030817170D122978C80710D501213E
:1031D0000DE0297889070BD5022108E02978C80677
:1031E00006D5032103E02978890601D50421397029
:1031F0001978DFF8F8B0002940F074813C4829784C
:1032000090F800E0DFF8E0908EEA0101314111F022
:10321000010F824640F03D8136490978002940F08F
:103220003881013604F10A02072E92B201D0144609
:10323000C2E79BF8003003F0FF06002B40F05281FC
:1032400008F11E073FB215B233462A4639462A48CE
:1032500021F070F999F800301B0607D5254B1B7833
:1032600003F0FF02002B40F01B8116469BF8002064
:1032700002F0FF03002A40F035810FFA88FB1E4858
:103280002A46594621F056F999F8010066B129F00D
:1032900023FF1A4929F074FF194929F067FE29F024
:1032A000C5FA06460F4631E0C0EBC0006523A0F525
:1032B0006070584340F2EB1390FBF3F029F0A4FA4E
:1032C0000022002306460F4629F076FDE0B90022D1
:1032D0000C4B3046394629F08DFDB8B10026094F18
:1032E00014E000BFE0C7FF1FF0C4FF1FC8C5FF1FE9
:1032F000408EFF1F3A88FF1F58C6FF1F96434B3F63
:103300009643CB42000059400026002799F801203F
:103310009AF801309A4240F0D280744B1B78002B0F
:1033200040F0CD8004F11401022289B24046FFF73B
:10333000EFFE04F11E01042289B24046FFF7E8FEC9
:103340006B4D04F1280189B206224046FFF7E0FEEA
:103350002978FF292DD0674B1B788B4229D9664EDF
:103360006248A82707FB016EDEE90E23007807906C
:1033700001200690052005904FF0000C04F13C0060
:10338000CDF824C080B24FF6FF7CCDF820C0049069
:10339000CDF80C800291DEE91801CDE90001574813
:1033A00018F01AFE2B7807FB0363D3E90E01C3E97B
:1033B00018016978FF292ED04E4B1B788B422AD9F1
:1033C0004D4E4A48A82707FB016EDEE90E23007820
:1033D000079001200690052005904FF0000C04F1A5
:1033E0004600CDF824C080B24FF6FF7CCDF820C057
:1033F0000490CDF80C800291DEE91801CDE90001BE
:103400003E4818F0E9FD3A4B5B7807FB0363D3E9CC
:103410000E01C3E918010120FDF717FAFF2861D05A
:10342000344B1B7883425DD92B7883425AD0304B82
:103430005B78834256D0304E2C4FA82505FB0061A7
:103440004FF0000ED1E90E2350343F78CDF824E040
:103450004FF6FF7ECDF820E007974FF0050E0127CD
:10346000A4B2CDF814E006970494CDF80C80029035
:10347000D1E91801CDE90001204818F0ADFD38462A
:10348000FDF7E3F905FB0060D0E90E23C0E918233E
:1034900028E0214640460B93FFF70CFE0B9BC0E64D
:1034A0000A23019600932A4619233946144821F02D
:1034B000F1FE14491248FDF716FA0126D6E64FF040
:1034C00000090A238DE808022A461E2359460C48A3
:1034D00021F0E0FECDF8009032463B460848FDF76B
:1034E00010FA1FE70DB0BDE8F08F00BF3A88FF1F4C
:1034F0002488FF1F2AC4FF1F008FFF1FB8BCFF1FB7
:1035000058C6FF1FF91B03002DE9F04F9E4B9F4C3F
:103510001B7813F0FD0087B001D1207014E09C4AA5
:103520001278C82A15D9DB0713D59A4B187880B9B9
:10353000994B1B78FF2B0CD1984B05221A70984A97
:10354000137843F001031370904B187007B0BDE877
:10355000F08F944B1A78012A1D4629D01B78042B32
:1035600016D1914B914A5B7812789A4210D9904AC1
:10357000A82101FB0323D3E90E678E4B586829F07D
:1035800055F902460B463046394629F029FC78B9F0
:103590002B78042B05D1844B844A1B7812789A42ED
:1035A00008D82A787F4B022A16D01A78042A15D117
:1035B0000020C9E77E4AA82101FB0323D3E90E6757
:1035C0007C4B186829F032F902460B4630463946E2
:1035D00029F006FC0028E4D06420B5E71A78052A13
:1035E00014D01A78062A13D01A78072A12D01A781B
:1035F000082A11D01B78092B40F0C2806E4B6B4912
:103600001A78097891429A4608D8B9E050209BE789
:103610003C2099E7282097E7142095E71B78DFF8EE
:1036200090B1A82101FB03B3D3E90E679AF80030EB
:1036300001FB03B3D3E912459AF8003001FB03B153
:1036400022462B46D1E9160128F090FF00220023E4
:103650008046894629F0A6FB90B922462B46304683
:10366000394628F083FF0022544B29F033F94246B3
:103670004B4629F059FA0022002328F079FF01E097
:103680000020002129F0FEFBC6B2092E75D89AF859
:1036900000109AF80030DFF82881A82707FB01B155
:1036A00007FB03B3D3E91223D1E9160128F05EFF2B
:1036B0000022424B29F038FA9AF8003007FB03B396
:1036C000D3E90E23CDE900239AF8003007FB03BBB2
:1036D000DBE9122304460D463046CDE9022329F0EA
:1036E00093F822462B4629F0F5F8824618F8060092
:1036F0008B4629F079F806F10109064648460F463F
:1037000029F082F822462B4629F0E4F852465B461F
:1037100028F02CFF0022002318F80980CDE90401CD
:1037200029F040FB20BBDDE90223DDE9000128F0A0
:103730001DFF52465B4628F019FF044640460D46E1
:1037400029F052F832463B4628F010FF02460B465D
:103750002046294629F0BEF8DDE9042329F0E4F9E2
:1037600002460B463046394628F002FF06460F4611
:103770003046394629F05EFB03E0114B987AE3E6C8
:103780002078C0B2E0E600BFABC7FF1FC0C4FF1F78
:1037900030C5FF1FE28EFF1F0B88FF1FE0C7FF1F12
:1037A000F0C4FF1FF18EFF1F2488FF1F2AC4FF1FD4
:1037B000008FFF1F98C5FF1F29C4FF1F0000244072
:1037C00084C5FF1F244B33F8102044F208239A428B
:1037D0003AD00FD81F2A2FD001D8B2B339E0B2F5B2
:1037E000FC6F23D040F2FF739A4232D1FF22114680
:1037F00000202CE04FF6C0439A4221D009D8B2F500
:10380000784F16D04FF61F039A4222D1FF22002193
:103810001CE04FF6E0739A4205D04FF6FF739A42D0
:1038200017D1FF2211E00022FF2107E00022FF2133
:103830000CE00022114605E0FF220021084606E0C8
:103840000022A521FF2002E0A5221146104623F008
:1038500000B90020704700BF1088FF1FF8B50E4B5D
:103860001B780546BBB10D4F0024FF2D0ABF07EBA7
:10387000440328465878FFF7A5FFA6B20246314612
:103880000748013423F0B3F8082CEED10448BDE812
:10389000F84022F0DFBFF8BDFC87FF1F2788FF1F1D
:1038A00018C5FF1F0D4B30B51B889B1A994285B078
:1038B00011DA5408031B0A44044412B24FF6E075AF
:1038C00024B202928DE8140003950AB21BB201B231
:1038D000034820F06DFD05B030BD00BF3C88FF1FE0
:1038E00058C6FF1F064B82B01A68009200991A68EA
:1038F0000192019A521A8242F9D902B0704700BF70
:103900004CD8FF1F13B504461CF06DFF8DF8060060
:1039100020461CF068FF8DF80700BDF8060002B0D5
:1039200010BD13B504461CF05EFF8DF80400204660
:103930001CF059FF8DF8050020461CF054FF8DF84F
:10394000060020461CF04FFF8DF80700019802B0DA
:1039500010BDFFFFFFFFFFFFF8B5234CA82303FBBB
:10396000004408460D4628F04FFFD4E9222328F0F2
:10397000B1FF0646C5F57F7003300F4628F044FFBF
:1039800002460B463046394629F0CEF826F02CFA8E
:10399000D4E9202306460F4628F09CFF32463B46DA
:1039A00028F098FFD4E91E2328F0E2FD32463B467A
:1039B00028F090FFD4E91C2328F0DAFD02460B46DC
:1039C00000200A4929F0B0F805A3D3E9002328F024
:1039D000CDFD29F02FFA00B2F8BD00BFAFF3008093
:1039E0000000006066127140008FFF1F0000F03F72
:1039F0002DE9F04F8B4B1B78042B91B082460C467F
:103A000016462BD11323884A884908A81DF0C2F80E
:103A100008A98748FDF7EAFD08A81CF037FF84488D
:103A20001CF077FFB8B152468249814825F051FD1C
:103A3000651EE71D15F8012F7F497D4825F049FDDA
:103A4000AF42F7D17D4B7E491B680793079B7848AF
:103A5000324625F03EFD76481CF04FFF794B1D792C
:103A600019680023DAB2AA4208D2DA0088188A5804
:103A7000924503F10103F5D103792BB9724B5B68D1
:103A80009A4540F05181002303F1010B0DE093F8BA
:103A90000890B9F1060F16D0B9F1070F16D12278A8
:103AA0001B69934214D00BF1010B5FFA8BFB664A42
:103AB000654F0BF1FF35EDB2A82303FB05235A68D0
:103AC0009245E4D030E14FF0010803E0C84601E040
:103AD0004FF00008A82606FB057600230022CDE95A
:103AE0000823B37A012B0AD1F37A13B9737AE25619
:103AF0000EE0737AE25C0023CDE908234FE0B8F1D1
:103B0000010F17D1022B08D1F37A1BB9737AE25E49
:103B1000D317F1E7737AE25AEDE7042B3FD1F37A3A
:103B200013B9737AE258F3E7737AE35808930023E2
:103B3000099334E0B8F1000F18D1022B07D1F37AC2
:103B400013B9737AE25E08E0737AE35A09E0042B52
:103B500025D1F37A1BB9737AE258D2BAD8E7737ACF
:103B6000E3585BBA0893CDF8248018E0B8F1040F4D
:103B700015D1042B13D1737AE118E25C4878CB7825
:103B8000120642EA00421A438B7842EA0322D31714
:103B9000CDE90823089828F049FEC6E90E01A826B9
:103BA00006FB0576327B3369FF2A22D1FF2B2DD10C
:103BB000DDE9080128F060FE80466079894628F03A
:103BC00013FE02460B460020204926F08BF90246E0
:103BD0000B464046494628F0A7FF8046E0888946C4
:103BE00028F012FE02460B464046494628F0BEFC2D
:103BF0003CE05BB1B9F1070F08D0DDE90801002115
:103C0000184028F0A1FC28F037FE27E0B8F1040F97
:103C10004FF0A8061CD106FB0576D6E90A23D6E9A3
:103C20000E011DE004B9FF1FBC1503002CD5FF1FBA
:103C3000F8C4FF1FDD140300E21403004CD8FF1F7B
:103C4000E8140300ECC9FF1F008FFF1F0000244091
:103C5000DDE9080128F010FE06FB0576D6E90A2307
:103C600028F038FED6E90C2328F082FCC6E90E01C4
:103C70004FF0A80808FB057898F86830012B43D16D
:103C8000D8E90E23CDE90223D8E92023D8E91C671F
:103C9000CDE90023D8E92223D8E91E01CDE9042388
:103CA00032463B4628F062FC0022002380468946CB
:103CB00029F078F8F8B932463B46DDE9020128F0F0
:103CC00055FCDDE9002306460F46DDE9040128F036
:103CD0004DFC02460B463046394628F0FBFD424675
:103CE0004B4628F021FF02460B46DDE9000128F093
:103CF0003FFCCDE900010E4AA82303FB0523DDE9C3
:103D00000012C3E90E120AE0022B08D1BDF92010FF
:103D10002846FFF721FE28F077FDC8E90E010121B2
:103D20002846FDF7D3FFBEE611B0BDE8F08F00BF17
:103D3000008FFF1F2DE9F047A54AA82303FB0023AE
:103D40008AB05E7A042E05460F46924600F2E48061
:103D5000A04B985D23F048F816F0FD0F04B23ED159
:103D600040F28E339C423ADC40F27A339C4202DDD0
:103D7000A0F1080432E040F266339C4202DDA0F17B
:103D80000D042BE0B4F5517F02DBA0F1120425E015
:103D9000B4F5397F02DDA0F119041FE040F276236B
:103DA0009C4202DDA0F1240418E040F262239C4210
:103DB00002DDA0F1280411E0B4F5117F02DDA0F1CD
:103DC00022040BE0B4F50C7F02DDA0F11C0405E039
:103DD00040F206239C4202DDA0F1180424B2A8237D
:103DE00003FB05A3D3E90E234FF4CA7373437A4A46
:103DF000D058652101FB06014FF0650E42F82140C5
:103E0000D1580131D150D158B94224BF0121D150EC
:103E10000020002300210EFB06F601335FFA83FE2B
:103E2000774508D906EB030E52F82EE010EB0E0092
:103E300041F10001F1E77A1E4FF0A808D31708FB03
:103E400005A829F0BFFB28F00FFD98F86830022B79
:103E500006460F460ED128F0EDFF01B22846FFF7C7
:103E60007BFD28F0D1FCD8E90A2328F033FDD8E9FE
:103E70000C2332E0012B37D1D8E91C23CDE90423F0
:103E8000D8E92023D8E91E01CDE90223DDE9042386
:103E900028F06CFB00220023CDE9060128F082FF08
:103EA00000BBDDE90223D8E9220128F05FFBDDE950
:103EB0000423804689463046394628F057FB02469F
:103EC0000B464046494628F005FDDDE9062328F06B
:103ED0002BFE02460B46DDE9020128F049FB0646AF
:103EE0000F4601E0DDE902673C4B1B78032B04D150
:103EF0004FF4D670FCF7A9FC88B9354AA82303FB18
:103F00000525D5E90A233046394628F0E3FCD5E9F2
:103F10000C2328F02DFB58E00020002155E030490B
:103F20003048FCF7E0FC29462E48FCF7E0FC2E491F
:103F30002C48FCF7D8FC21462A48FCF7DCFC02247C
:103F400029492848FCF7CFFC32463B4600942548D7
:103F5000FCF7D7FC24492348FCF7C5FCA82303FB46
:103F600005AA0094DAE91C231E48FCF7CAFC1E4986
:103F70001C48FCF7B8FC0094DAE91E231948FCF74A
:103F8000C0FC19491748FCF7AEFC0094DAE920237D
:103F90001448FCF7B6FC14491248FCF7A4FC009442
:103FA000DAE922230F48FCF7ACFC0F490D48FCF777
:103FB0009AFC0E490B48FCF796FC0D4B09481B6810
:103FC00009930999FCF7ACFC97E70AB0BDE8F087C4
:103FD000008FFF1FACC7FF1F0CCAFF1F04B9FF1FD4
:103FE0009E160300848AFF1FCF1A0300A816030041
:103FF0004CD8FF1F2DE9F04FA44DDFF8949289B003
:1040000005F105084FF0A80A15F8017FA04C0AFB3E
:10401000079696F890306BB14FF48E70FCF715FC54
:1040200001463846FFF786FEC6E90E0101212878D1
:10403000FDF74CFEA845E7D1964E974D32782B7888
:104040009A4219D2262022F0CFFE377840F21D1373
:10405000C0F1D8005843A82606FB074600F6FC002E
:1040600028F0D2FBD6E90A2328F034FCC6E90E0179
:1040700001213846FDF72AFE884B1A78FF2A9B4615
:104080004ED0874B2E7893F80080B04548D201205F
:10409000FCF7DBFB8642814642D90320FCF7D5FBC7
:1040A00086423DD9A82606FB0047D7E90E0100222B
:1040B0007C4B28F09FFE002800F09E80744806FB91
:1040C0000900D0E90E01D7E90E2328F02DFD28F0D4
:1040D000D9FEC0B229F000F87349019029F050F8D8
:1040E000724902904FF000090F680391CA4606FB1F
:1040F00008461BF80A0028F0EFFF804601460298A8
:1041000029F0FAF900285ED10AF101035FFA83FA77
:10411000BAF1050FEDD9B9F1000F01D0039B1F6073
:10412000634B93F800B0BBF1010F20D1614B93F8C2
:1041300000A02B78534539D9A82303FB0A43D3E9C0
:104140000E895D4B186828F071FB06460F46024643
:104150000B464046494628F043FE002865D0574BA1
:104160001A78012A61D083F800B0594674E0BBF197
:10417000030F04D1514F3B78C3B9012107E0BBF1D4
:10418000020F13D14D4F3B78012B0FD100214C4B27
:104190003970187823F032FA4A4B38781E7828F0B4
:1041A00023FBA82303FB0646C6E90E01464B1E78F7
:1041B000FF2E00F0DB800520FCF747FB2D78A8429E
:1041C00007464ED3D2E04149019828F0D9FF014675
:1041D000404629F091F9002896D00AF1010028F014
:1041E00013FBC6E90E013A4B1B680593059F4FF080
:1041F00001094FF0060A87E7D7E90E010022294B93
:1042000028F0E4FD48B9324B284A1B680693069B08
:1042100012689B1AB3F57A7F82D9A82606FB084656
:1042200000220023C6E90E237AE7A82303FB0A4AEB
:10423000DAE90E233046394628F0D2FD10B11F4B83
:104240001A783AB91F4B1E782B78B342AED91B4B64
:104250001878A4E700211970194B187823F0CEF9CB
:10426000F0E70420FCF7F1FA854233D9A82303FBD9
:104270000747D7E90E8903FB0040494603FB064484
:10428000D0E90E23404628F071F961E005B9FF1F1F
:10429000008FFF1F0388FF1F2AC4FF1F20D5FF1FA9
:1042A0004088FF1F000008403333933F18D5FF1F9D
:1042B000B0C5FF1F08CAFF1FB4C7FF1F0D88FF1F2F
:1042C000E08EFF1F4188FF1F0788FF1F9A99593F03
:1042D0004CD8FF1F40F21D10FCF7B7FA012845D15A
:1042E000244A254B12681B680792079A03F5FA7354
:1042F0009A423BD90520FCF7A8FAA82505FB004502
:10430000074600220023D5E90E0128F04BFDDFF817
:104310006CA060B90021DAF8000029F0C5F830B1CE
:10432000D5E90E0128F0CEFDCAF800001EE0A82550
:1043300005FB0747DAF8000028F078FAD7E90E897C
:1043400002460B464046494628F010F905FB064454
:10435000D4E90A2328F0BEFAD4E90C2328F006F9A0
:10436000C4E90E0101213046FDF7B0FC09B0BDE8FB
:10437000F08F00BF4CD8FF1FD88EFF1FEC8EFF1FA1
:1043800010B572B60C4B41241C7003F8010C073BAE
:104390008020187018780006FCD5084B1B788B54C9
:1043A000074B0A441B785370064B1B789370064BDF
:1043B0001B78D37062B610BD070002400B000240AC
:1043C0000A000240090002400800024073B50F498C
:1043D0000F4801AEFCF787FA002231460F20FFF7A5
:1043E000CFFF4FF4C67500242846FCF72EFAA5F53A
:1043F000C6730135F35C83421CBF0134E4B2B5F5EA
:10440000C87FF1D1204602B070BD00BFAF160300D7
:10441000848AFF1FF0B595B02C22002109A822F054
:10442000DDFBA94901A825F0A2F94FF4C6750A27BA
:104430002846FCF70AFA0928044608D8A34901A827
:10444000FCF74FFAA14901A8FCF74BFA22E06328D8
:1044500020D89E4901A8FCF744FAB4FBF7F60A22DB
:10446000F1B205A825F0B6F905A901A8FCF737FABD
:1044700005A825F03CF907FB16410A22C9B205A898
:1044800025F0A8F905A901A8FCF729FA05A825F047
:104490002EF903E0214601A825F06AFA0135B5F5A9
:1044A000C87FC5D12C22002309A901A825F0CCFA88
:1044B00009A821F092FD1021054621F003F90446D8
:1044C000284629F09FFA20222146814829F0B4FA93
:1044D00080B9804905A825F04AF905A94FF4FC6286
:1044E0007D4815F0A5F805A825F001F901214FF444
:1044F0008B7067E0794901A825F0B6F94FF4C675CD
:104500000A272846FCF7A1F90928044608D86F496C
:1045100001A8FCF7E6F96D4901A8FCF7E2F922E0F1
:10452000632820D8694901A8FCF7DBF9B4FBF7F64A
:104530000A22F1B205A825F04DF905A901A8FCF75A
:10454000CEF905A825F0D3F807FB16410A22C9B217
:1045500005A825F03FF905A901A8FCF7C0F905A8B1
:1045600025F0C5F803E0214601A825F001FA013540
:10457000B5F5C87FC5D12C22002309A901A825F0D3
:1045800063FA09A821F029FD1021054621F09AF8C7
:104590000446284629F036FA202221464C4829F0C4
:1045A0004BFAA8B94E4905A825F0E1F805A94FF442
:1045B000FC62494815F03CF805A825F098F801215F
:1045C0004FF48D70FCF7D4F8204629F01BFA75E003
:1045D000444901A825F048F94FF4C6750A27284632
:1045E000FCF733F90928044608D8384901A8FCF734
:1045F00078F9364901A8FCF774F922E0632820D83D
:10460000324901A8FCF76DF9B4FBF7F60A22F1B2C2
:1046100005A825F0DFF805A901A8FCF760F905A8B1
:1046200025F065F807FB16410A22C9B205A825F056
:10463000D1F805A901A8FCF752F905A825F057F80B
:1046400003E0214601A825F093F90135B5F5C87FAF
:10465000C5D12C22002309A901A825F0F5F909A844
:1046600021F0BBFC1021054621F02CF80446284619
:1046700029F0C8F920222146154829F0DDF980B932
:10468000194905A825F073F805A94FF4FC621248F2
:1046900014F0CEFF05A825F02AF802214FF4E770A8
:1046A00090E7124905A825F062F80B484FF47842CC
:1046B00005A914F0BDFF05A825F019F801A825F0FB
:1046C00016F815B0F0BD00BFBD1603006F1903004A
:1046D000CCC4FF1FDB1603005CB9FF1FFC160300F0
:1046E0001A17030038170300561703007D1703003D
:1046F00038B546F22C3112481EF049FC0121104811
:104700001EF03FFC0F490E48FCF7EDF84FF4C6745D
:104710002046FCF79AF80928054601D80A4902E024
:10472000632803D809490648FCF7DDF82946044800
:104730000134FCF7DCF8B4F5C87FE9D138BD00BF1F
:1047400058C6FF1F8B170300FF2103006F190300DA
:104750002DE9F041074688B068B9C34BC34AB3F9A5
:104760000030019012880D3A12B2009201460D22DB
:10477000BF4820F08FFDBF4B00221A70BE4B0022B5
:104780001A60BE4BFF221A703FB93B46DC2228213B
:10479000B7481FF0CFFEFFF7ABFFB924052646F25E
:1047A0002C3300258DE8500002931E22E623282199
:1047B000AF4820F0C7FD8DE85000E6231E2204AC70
:1047C0002821AB4802951FF0D1FBAD49AD4E2046E4
:1047D00024F0CDFF0F2323222D210093AA48029518
:1047E000DC23019414F0FEFF204624F080FF2946CC
:1047F0009F481EF0CCFB01219D481EF0C2FB2B46BA
:10480000272232219A481FF095FE7019143514F0B2
:1048100079FEB5F5027FF8D1002519269B4920467F
:1048200024F0A5FF28233722872199480295019477
:10483000009614F0D7FF204624F059FF95492046F2
:1048400024F095FF28233722B42193480295019440
:10485000009614F0C7FF204624F049FF8F492046F8
:1048600024F085FF28233722E1218D480295019409
:10487000009614F0B7FF204624F039FF89492046FE
:1048800024F075FF2823552287218748029501943B
:10489000009614F0A7FF204624F029FF8349204604
:1048A00024F065FF28235522B42181480295019404
:1048B000009614F097FF204624F019FF7D4920460A
:1048C00024F055FF28235522E1217B4802950194CD
:1048D000009614F087FF204624F009FF7749204610
:1048E00024F045FF282373228721754802950194FF
:1048F000009614F077FF204624F0F9FE7149204617
:1049000024F035FF28237322B4216F4802950194C7
:10491000009614F067FF204624F0E9FE6B4920461C
:1049200024F025FF28237322E12169480295019490
:10493000009614F057FF204624F0D9FE6549204622
:1049400024F015FF28239122B42163480295019495
:10495000009614F047FF204624F0C9FE5F49204628
:1049600024F005FF282337222D215D48029501946C
:10497000009614F037FF204624F0B9FE594920462E
:1049800024F0F5FE282355222D2157480295019445
:10499000009614F027FF204624F0A9FE5349204634
:1049A00024F0E5FE282373222D215148029501941D
:1049B000009614F017FF204624F099FE4D4920463A
:1049C00024F0D5FE282337225A214B480295019422
:1049D000009614F007FF204624F089FE4749204640
:1049E00024F0C5FE282355225A21454802950194FA
:1049F000009614F0F7FE204624F079FE4149204647
:104A000024F0B5FE282373225A213F4802950194D1
:104A1000009614F0E7FE204624F069FE4FF02308CC
:104A20003A49204624F0A3FE4423AF222D213848E2
:104A300002950194CDF8008014F0D4FE204624F0B5
:104A400056FE3449204624F092FE4423AF227621BC
:104A5000314802950194CDF8008014F0C3FE204641
:104A600024F045FE5AE000BF0488FF1F3C88FF1F6A
:104A700058C6FF1F0088FF1FCCC5FF1F0188FF1FFE
:104A8000AB15030020B9FF1F5CB9FF1FF21A03002A
:104A9000E8B9FF1FA8170300FCB9FF1FFA1A0300AB
:104AA00010BAFF1FFE1A030024BAFF1FE51E030001
:104AB00038BAFF1FB61C03004CBAFF1F831903004E
:104AC00060BAFF1F1817030074BAFF1F9417030082
:104AD00088BAFF1F6F1903009CBAFF1F0E1903004D
:104AE000B0BAFF1F02340300D8BAFF1F9E20030094
:104AF00000BBFF1F96170300C4BAFF1FDA33030081
:104B0000ECBAFF1FAD8C030014BBFF1F1618030087
:104B1000ACB9FF1F9817030070B9FF1F1549204655
:104B200024F025FE144802950194CDF80080452319
:104B3000AF22BF2114F056FE204624F0D8FD0FB955
:104B40000E4902E0012F11D10D49204624F00FFE3D
:104B50004FF6E07302930B480194009628239122AC
:104B60002D2114F03FFE204624F0C1FD08B0BDE821
:104B7000F08100BFA017030084B9FF1FA71703002F
:104B8000FE1A030098B9FF1F2DE9F043A14D89B02B
:104B900006460F46904600242819143414F0B2FC3F
:104BA000B4F5027FF8D19C4B9C4800251D709C4BAE
:104BB00000221A609B4BB9241D701E2246F22C3332
:104BC0004FF00509114602938DE810028C2320F066
:104BD000B9FB1E2211468C238DE810028F480295E6
:104BE00004AC1FF0C3F99049204624F0C0FD2322F5
:104BF0000F23114600938D4802958223019414F0EF
:104C0000F1FD204624F073FD294684481EF0BFF9CB
:104C1000012182481EF0B5F92B46272228217F4822
:104C20001FF088FCB8F1000F02D1CDF8008001E040
:104C30000223009332463B46784800261925FBF7AD
:104C400060FE7B49204624F092FD28233722232151
:104C5000784802960194009514F0C4FD204624F093
:104C600046FD7549204624F082FD28233722502135
:104C7000724802960194009514F0B4FD204624F089
:104C800036FD6F49204624F072FD282337227D210E
:104C90006C4802960194009514F0A4FD204624F07F
:104CA00026FD6949204624F062FD28235522232150
:104CB000664802960194009514F094FD204624F075
:104CC00016FD6349204624F052FD28235522502129
:104CD000604802960194009514F084FD204624F06B
:104CE00006FD5D49204624F042FD282355227D2102
:104CF0005A4802960194009514F074FD204624F061
:104D0000F6FC5749204624F032FD28237322232144
:104D1000544802960194009514F064FD204624F056
:104D2000E6FC5149204624F022FD2823732250211D
:104D30004E4802960194009514F054FD204624F04C
:104D4000D6FC4B49204624F012FD282373227D21F6
:104D5000484802960194009514F044FD204624F042
:104D6000C6FCB8F1010F1FD14349204624F0FFFCD7
:104D7000282391222321414802960194009514F0A2
:104D800031FD204624F0B3FC3D49204624F0EFFCE1
:104D90003C48029601940095282391227D2114F02D
:104DA00021FD204624F0A3FC3749204624F0DFFCF7
:104DB0000026192391220093502128230296019462
:104DC000324814F00FFD204624F091FC2325304991
:104DD000204624F0CCFC3E23AF22294602960194C3
:104DE00000952C4814F0FEFC204624F080FC2A4953
:104DF000204624F0BCFC3E23AF226721029601949A
:104E00000095264814F0EEFC204624F070FC09B012
:104E1000BDE8F08320B9FF1F0088FF1F58C6FF1FA1
:104E2000CCC5FF1F0188FF1FAB1503005CB9FF1F36
:104E3000F21A0300E8B9FF1FA8170300FCB9FF1F0F
:104E4000FA1A030010BAFF1FFE1A030024BAFF1F4C
:104E5000E51E030038BAFF1FB61C03004CBAFF1F43
:104E60008319030060BAFF1F1817030074BAFF1FED
:104E70009417030088BAFF1FAA1703009CBAFF1FEC
:104E8000AC170300C4BAFF1F6F190300B0BAFF1FAD
:104E90001618030070B9FF1FA017030084B9FF1F85
:104EA00010B5074C20461EF0E1F8204601211EF007
:104EB00068F820464FF6FF71BDE810401EF067B855
:104EC00058C6FF1F2DE9F04190B00446FFF7E8FFF8
:104ED0000021AE48AE4E1EF05AF8AE4B1878FCF7E3
:104EE0009BFB3278012A33D10A234FF4FC668DE80C
:104EF000480032211F23A548A74D20F0CBF90023FD
:104F000002223821A1481FF015FBA4499F48FBF756
:104F1000EAFCA349A348FBF7E6FC00242B78E1B2A6
:104F2000994204F101040FD2002208A815F0B6F945
:104F300008A99C4824F096FA08A824F0D8FB9A49BE
:104F40009848FBF7D0FCE9E7964824F0ABFAC0E0BC
:104F5000022A03D1954B1B7813B9A2E0092C76D80D
:104F60000A234FF6E0758DE8280001221F23322125
:104F7000864820F08FF98E4B84481D78022200234A
:104F800036211FF0D7FAFF2C18BF254689497F48E4
:104F9000FBF7A9FC29467D48FBF7A9FC864B1B685B
:104FA0000393864B039A1A60854B04AC03F1080205
:104FB000A04618685968274603C7083393423C4601
:104FC000F7D118689A889B793860BA80BB71303500
:104FD0007C488DF819501BF09CFC60B913234246A5
:104FE000794908A81BF0D6FD08A97648FCF7FEFA17
:104FF00008A81BF04BFC73481BF08BFC044600B365
:1050000067497048644DFBF76EFC00242B78E1B2D1
:10501000994204F101040FD2002208A815F03EF9CC
:1050200008A9684824F01EFA08A824F060FB5E492D
:105030006448FBF758FCE9E764496248FBF7B1FABA
:1050400047E063495748FBF7ACFA347041E0032A64
:1050500012D10A234FF6E0748DE8180001221F23B5
:1050600032214A4820F016F9332100230222474812
:105070001FF060FA574929E0042A15D10A204FF49D
:1050800078438DE8090001221F2332213F4820F098
:1050900001F93321002302223C481FF04BFA4E490C
:1050A00014E0092C7FF65CAF0A2146F22C338DE820
:1050B0000A0001221F233221344820F0EBF833216B
:1050C0000023022231481FF035FA44492F48FBF7EC
:1050D0000AFC434B1B78002B51D0424B2B481C88B9
:1050E0006408323421B2A4B20A224FF6E073671C7E
:1050F00002264FF478458DE80C003FB20E230122C2
:1051000020F0C8F8394600960C2308221F48019564
:1051100020F0C0F833463946009606221B48019518
:1051200020F0B8F8A71D04F10B014FF00408334636
:105130000096062209B2154801953FB220F0AAF860
:1051400033463246394611480195CDF8008020F0AB
:10515000A1F8062604EB08013B46424609B20B487B
:10516000019500961EF0A0F9E31D04F109010195D7
:1051700000961BB2424609B204481EF095F903207E
:10518000FCF74AFA10B0BDE8F08100BF58C6FF1F17
:1051900004B9FF1F2688FF1F2AC4FF1FAE17030094
:1051A00013150300848AFF1F5C15030027D5FF1F1A
:1051B0003F88FF1F211903004CD8FF1F34C5FF1F74
:1051C0001E150300F8C4FF1F2CD5FF1FAB150300ED
:1051D000B2170300C0170300C6170300CC17030063
:1051E000B8C7FF1F0488FF1F2DE9F0413B4C07465D
:1051F0002046FBF7DEFB3A4A012313702372394B3A
:10520000394A00261E70394B10781E70384B1978B9
:10521000884215461C4612D2DFF8E080022198F839
:10522000000022F019FA98F80000324B32491E6053
:1052300022284FF0030228BFFF2022F03FFA6A78AD
:1052400023789A420FD22D4C0221607822F004FA82
:105250006078284B2A49002222285A6028BFFF2064
:10526000032222F02BFA274B274D00241C70274BDA
:105270002E681C70264B14201C7024F050FC8046B5
:10528000FBF7B8FB414630461CF0DEFEA7F1640395
:10529000012B07D814202C6824F041FC0546FBF7AD
:1052A000B3FB13E01B4B38461C70FFF70BFE1A4B89
:1052B0001878FCF7B1F9194B1B78042B0CD014208B
:1052C0002C6824F02CFC0546FBF78AFB2946204677
:1052D000BDE8F0411CF0B8BEBDE8F08154C4FF1F2A
:1052E0003A88FF1FC4C7FF1F3788FF1F26D5FF1F3F
:1052F0002AC4FF1F14B9FF1FD9050000B9C7FF1F3B
:10530000E9050000E5C6FF1F98D7FF1FD0C5FF1FA6
:10531000C8C5FF1FE6C6FF1F2688FF1F04B9FF1F71
:1053200037B54FF6E074002808BF00240546FFF7A4
:10533000B7FD154B1B780194032B4FF00B03009323
:105340004FF000024FF0140307D0AA210F481FF0BE
:10535000A1FF00230222AC2106E0E6210B481FF04A
:1053600099FF00230222E82108481FF0E3F8012DED
:1053700007D1002105481DF00AFE05490348FBF747
:10538000B2FA03B030BD00BF2688FF1F58C6FF1F0A
:10539000AE1703002DE9F0438D4F8E4C3B78032B65
:1053A00087B0054609D00C210022B4F900308A48A4
:1053B0008DE8060011461FF06DFF0320FCF72CF965
:1053C00044F208260C22B4F9003083488DE84400EA
:1053D000002211461FF05EFFFFF762FD3DB1032D75
:1053E00000F0F080012D4FF478460BD801E046F232
:1053F0002C360B23009301962E230122052176489B
:105400001FF048FF754902A824F0B1F90523009365
:10541000032202AB1921724815F0A6FA02A824F063
:1054200066F915F0FD0F08D10B23009301962E238A
:105430000122372168481FF02DFF6A4902A824F095
:1054400096F905230093032202AB4B21644815F023
:105450008BFA02A824F04BF9012D73D100215E488C
:105460001DF095FD604B1A78012A1E4607D14FF6B4
:10547000FF7159481DF08BFD4FF4784301E04CF269
:1054800018634FF00B0901220193A8212A235248E7
:10549000CDF800901FF0FEFE4FF00508534902A81A
:1054A00024F065F902AB0322BD214D48CDF8008000
:1054B00015F05AFA02A824F01AF9002146481DF006
:1054C00066FD3378012B56D0FCF732FB4CF21866A0
:1054D000FF2814BF4FF4FC633346012201936F2170
:1054E00034233D48CDF800901FF0D4FE404902A877
:1054F00024F03DF902AB03228B213948CDF800801E
:1055000015F032FA02A824F0F2F83B783248CDF8D0
:105510000090032B18BF4FF4FC662B230122D721E8
:1055200001961FF0B7FE334902A824F020F92C4859
:10553000CDF8008002AB0322ED2115F015FA02A888
:1055400024F0D5F84FF6FF7123481DF020FD032D00
:1055500016D121880B2046F22C3332398DE8090010
:1055600009B22D2301221C481FF094FE24882249F1
:105570001E3CA4B215E04FF6FF7117481DF007FD61
:10558000218815480B2246F22C3332398DE80C0065
:1055900009B22D2301221FF07DFE248817491E3CED
:1055A000A4B202A824F0E3F805230093032202AB7F
:1055B00021460B4815F0D8F902A824F098F807B056
:1055C000BDE8F0834FF6FF7103481DF0E0FCC0E733
:1055D0002688FF1F0488FF1F58C6FF1FD21703002D
:1055E000B8BCFF1F711603000E88FF1FDA170300F7
:1055F000DF170300E8170300461F0300EF1703003F
:105600002DE9F0437E4B1878A7B0002800F0F58014
:105610007C4F7D483988002301937C4B1B88423B9B
:105620001BB2653900932822652309B21FF032FEB0
:105630000123774A774916A81BF0ACFAFFF730FC34
:1056400008230DEB03000A227349FAF74BFF0622E9
:1056500002A912A824F042FA70491EA824F087F883
:105660001EA912A824F017FA04461EA824F03FF839
:1056700012A824F03CF864B90623224602A91EA809
:1056800024F00CFA1EA902A824F0E6F81EA824F0C3
:105690002EF8DFF89C81FF240025012216A91EA800
:1056A0001BF0D4FA1EA81BF034F906461EA8002EE3
:1056B00000F081801BF0EBF8014606A824F057F8B3
:1056C0001EA81BF0E6F8814600286DD154490AA8AF
:1056D00024F04DF80AA906A824F0DDF9002816DB0D
:1056E00001234A4606A90EA824F0D8F94D4912A86C
:1056F00024F03DF812A90EA824F0CDF9B0FA80F6F6
:1057000012A823F0F4FF0EA8760923F0F0FF0AA8F0
:1057100023F0EDFF002E47D198F80020AB1A0C2B98
:1057200001DC954202D20135EDB23DE003EB4302CC
:105730003988354803EB820229325D39334612B28B
:1057400009B205F101091EF0F5FE49462E48FBF7A6
:10575000D2F835492C48FBF7C6F806A92A4823F0A9
:1057600081FE2F4912A824F002F812A906A824F0FD
:1057700092F93246034606A90EA824F08FF90EA826
:1057800024F0B3F9014602A824F030F906460EA829
:1057900023F0ADFF12A823F0AAFF1EB198F8004035
:1057A0002C1BE4B25FFA89F506A823F0A0FF1EA81F
:1057B0001BF06CF871E71BF069F81C4B16A81D7004
:1057C0001BF09BF8FF2C11D0398804EB440204EB4A
:1057D00082020A204FF4784328325E398DE80900AE
:1057E00012B25F2309B208481DF09EFE02A823F002
:1057F0007EFF16A81BF04AF8204627B0BDE8F083CC
:1058000027D5FF1F0488FF1F58C6FF1F3C88FF1FB6
:10581000AC1503002CD5FF1F38C5FF1FCF1A03009E
:10582000F4170300A0180300F81703000BB9FF1FBB
:10583000E88EFF1F2DE9F0414E4B1978A0B00646C7
:1058400019B90A2223F0C6FF8FE001234A4A4B49C7
:105850004B4F10A81BF09EF9FFF722FB00240122FA
:1058600010A918A81BF0F2F918A81BF052F8054669
:1058700018A8002D6DD01BF00AF80146684623F0E9
:1058800076FF18A81BF005F8804600285AD13D493C
:1058900004A823F06CFF04A9684624F0FCF8002853
:1058A00016DB01234246694608A824F0F7F836497A
:1058B0000CA823F05CFF0CA908A824F0ECF8B0FABF
:1058C00080F50CA823F013FF08A86D0923F00FFF43
:1058D00004A823F00CFF002D34D12C490CA823F090
:1058E00046FF0CA9684624F0D6F805460CA823F01C
:1058F000FEFE002DACBF0121FF2107203970FAF711
:1059000037FF234B1A78234B1B7813449C4217D143
:105910001C490CA823F02BFF0CA9684624F0BBF807
:10592000002203466946304624F0B8F80CA823F05C
:10593000DEFE684623F0DBFE18A81AF0A7FF11E090
:105940000134E4B2684623F0D2FE18A81AF09EFF94
:1059500085E71AF09BFF10A81AF0CFFF0E493046DA
:1059600023F005FF10A81AF091FF304620B0BDE8E3
:10597000F08100BF27D5FF1FAC1503002CD5FF1FFA
:10598000A4C6FF1FF4170300A0180300FB170300B1
:10599000A0C5FF1FE88EFF1F6F1903002DE9F0431C
:1059A0008B4C8C4E2288338891B00A210025653BB0
:1059B0000A3A8DE822001BB212B2012180468648C5
:1059C0001FF068FC228884480A3A2B4612B2012153
:1059D0001EF0B0FD814B1B7843B981497E48FAF730
:1059E00082FF4FF47A7021F0ADFFEDE072B6FFF761
:1059F00057FA7C4B02AD03F1100E2A46186859681D
:105A00002F4603C7083373453D46F7D118689B8876
:105A10003860BB807449532308A808F130088DF81A
:105A200018801BF0B7F808A81AF073FF0546002885
:105A300000F09C806D4B6E4A1B7812786D496E4C5D
:105A400008A823F046FD04F5EE670026A04694F86A
:105A50005830002B7DD094F827300B2B05D1A38B29
:105A6000093B9BB2022B40F2A380B4F9101008A8A6
:105A7000FAF741FF614908A8FAF735FFB4F91210A7
:105A800008A8FAF738FF5D4908A8FAF72CFFB4F91F
:105A9000141008A8FAF72FFF584908A8FAF723FFAF
:105AA000B4F9161008A8FAF726FF544908A8FAF71F
:105AB0001AFF94F8271008A8FAF719FF4F4908A809
:105AC000FAF711FFA18B08A8FAF715FF4B4908A8B0
:105AD000FAF709FFE18B08A8FAF70DFF474908A874
:105AE000FAF701FF218C08A8FAF705FF434908A837
:105AF000FAF7F9FE217E08A8FAF7F9FE3F4908A84F
:105B0000FAF7F1FE94F82730ABB94FF07009012590
:105B100009FB068994F82430AB4213D909EB05033D
:105B200008A8197EFAF7E3FE0135344908A8FAF708
:105B3000DAFEEDB2EEE70B2B01D0052B02D1237874
:105B4000002B38D12E4908A8FAF72BFD08A81AF027
:105B500036FE7034A74206F101067FF478AF08A83C
:105B60001AF02DFE08A81AF0C8FE1CE022880A3A96
:105B7000034612B2012118481EF0DCFC338822884B
:105B8000154801950A21653B0A3A00911BB212B2F1
:105B900001211FF07FFB1B490F48FAF7A4FE4FF4C9
:105BA000FA6021F0CFFE62B608A81AF06FFE0BE093
:105BB0000023E38359E7214608A8FAF794FE0F492A
:105BC00008A8FAF790FEBDE711B0BDE8F08300BF6A
:105BD0003C88FF1F0488FF1F58C6FF1F27D5FF1FE3
:105BE00019180300461803002CD5FF1F0E88FF1F4D
:105BF0002688FF1F25180300B8BCFF1F5C15030093
:105C0000AB150300321803002DE9F04FC24EA3B0CC
:105C1000934604AF32883B610A3A002312B28A46A7
:105C200080461946BD4897F8A0901EF083FCFFF708
:105C300037F907F118001AF01BFEB8481DF092F86A
:105C4000824580F2AE81B5481DF08FF80A38834551
:105C500080F2A78101234246B14907F158001AF0AA
:105C600099FF07F1580107F11800FBF7BFFC1AF084
:105C700050FE044607F158001AF008FE2CB94246BF
:105C8000A849A64823F025FC90E107F1180107F187
:105C90005800FBF7B5FF07F15800FDF733FE044647
:105CA00007F158001AF0F2FD44F642539C4240F0CE
:105CB0003F8107F1180107F15800FBF7A1FF07F139
:105CC0005800FDF72EFE07F158001AF0DFFD07F12E
:105CD000180107F15800FBF793FF07F15800FDF793
:105CE00020FE07F158001AF0D1FD07F1180107F165
:105CF0005800FBF785FF07F15800FDF712FEF8602A
:105D000007F158001AF0C2FD07F1180107F1580019
:105D1000FBF776FF07F15800FDF703FE07F1580087
:105D20001AF0B4FD07F1180107F15800FBF768FFFE
:105D300007F15800FDF7F5FD054607F158001AF088
:105D4000A5FD07F1180107F15800FBF759FF07F10E
:105D50005800FDF7E6FD786107F158001AF096FD4E
:105D600007F1180107F15800FBF74AFF07F1580047
:105D7000FDF7C8FD044607F158001AF087FD012C15
:105D800040F0D68007F1180107F13800FBF738FF23
:105D900007F13800FDF7B6FD182811D107F11801F9
:105DA00007F15800FBF72CFF07F15800FDF7B9FD8C
:105DB000B0FA80F407F1580064091AF067FD00E0BA
:105DC000002407F138001AF061FD002C00F0B080CB
:105DD000C7F808D0ADB2BC8ABAF1000F11D1BBF13F
:105DE000000F0ED1504B1A8833881B1B0221521B07
:105DF0000A3B92FBF1F293FBF1F31FFA82FA1FFACE
:105E000083FB3B697C612E467BB1484B702000FBD5
:105E1000093090F82530428A018A029390F82730A1
:105E2000019300942B461AF04BF905F1010909EB97
:105E3000490929F0030339483B611CF093FF55449D
:105E4000854205DD35481CF08DFFCAEB000086B2A7
:105E500032481CF08AFF0BEB0405854206DD2F4813
:105E60001CF083FFCBEB000083B27B6106EB4605A1
:105E7000EB1D23F00703ADEB030DABB2FA687B60BB
:105E80003B69013C564403FB0429B3B20DF11008F1
:105E90000024FB607B69A6B2B34239D907F1180030
:105EA0001AF00DFD484504D0494607F118001AF0D4
:105EB000FDFC7A68414607F118001AF0F2FC0BEB82
:105EC000060292B20092FB68144851461FF0CAFACB
:105ED0000026B54214DD08EB0603104899785B787C
:105EE0000902DB0001F4784103F4FC630B4318F86A
:105EF0000610033643EAD1011DF00AF8B6B2E8E70E
:105F000006481DF011F83B690134C3EB0909C1E7EC
:105F1000D7F808D03FE000BF3C88FF1F58C6FF1FDE
:105F20002CD5FF1F5C1803000488FF1FB8BCFF1F9F
:105F30003288234B0B204FF6E0710B3AB3F9003057
:105F400012B28DE8030000211E481FF0A3F94FF4A0
:105F500078411C481DF01BF841461A48FAF7C3FC6B
:105F600019491848FAF7BFFC414618481AF062FE72
:105F70004FF4FA7021F0E6FC154A702303FB092266
:105F8000938B01339BB2FD2B938304D84A46594629
:105F9000504600F021F807F118001AF0AEFC012479
:105FA00004E00C490748FAF79EFC002407F11800AA
:105FB0001AF06CFC20467C37BD46BDE8F08F00BF70
:105FC0000488FF1F58C6FF1F761803002CD5FF1F3B
:105FD000B8BCFF1F691803002DE9F04F774B1C7800
:105FE000A3B081468A469046002C00F0E280744BB4
:105FF0007449702505FB023502A8AF8B23F0B7FB6F
:1060000095F82730052B01D16F4902E00E2B03D103
:106010006E4902A823F028FC95F82730052B05D1FE
:10602000284627F04AFE012800F2BA80FFB2FF2F6F
:1060300019D10498013023F074FD049A04460146F6
:106040000023013202A823F0FFFC049B234400221A
:106050005A702046CDF80080012352464946FFF78A
:10606000D3FD044698E0DDF808B0594901235A46AB
:1060700012A81AF08FFD0026012212A91AA81AF000
:10608000E5FD1AA81AF045FC044600287BD05946C5
:1060900006A823F06CFB1AA81AF0F9FB014606A823
:1060A000FAF71FFC1AA81AF0F4FB002864D149493A
:1060B0000AA823F05CFB0AA906A823F0ECFC002840
:1060C0000CDB45490EA823F052FB0EA906A823F0CD
:1060D000E2FCC4430EA8E40F23F009FB0AA823F056
:1060E00006FB002C48D1BE4241D10898013023F074
:1060F00018FD089A014601320646234606A823F0F9
:10610000A3FC089B33441AA85C701AF0F6FB12A893
:106110001AF0F3FB2B4906A823F0A6FB1AA81AF0E5
:10612000B6FB014606A8FAF7DCFB0898033823F013
:10613000F8FC089A234607460146033A06A823F0CE
:1061400083FC089A3946033A284620F0ADFC012327
:1061500052464946CDF800803046FFF755FD0446CB
:1061600006A823F0C4FA1AA81AF090FB11E01AA8A6
:106170001AF0C3FB0136F6B206A823F0B8FA1AA843
:106180001AF084FB78E71AA81AF080FB12A81AF01C
:10619000B4FB12A81AF07AFB02A823F0A8FA08E0D0
:1061A000294602A8FAF79DFB0A4902A8FAF799FBCB
:1061B0003FE7204623B0BDE8F08F00BF27D5FF1F83
:1061C000B8BCFF1FAB1503008B1803009118030028
:1061D0002CD5FF1F991803009E18030073B51C4BA4
:1061E0001C4A1D481D4D1E4E00241C701D4BB3F94A
:1061F0000030019412880C3A12B2009221460C220F
:106200001FF048F8184B1878FBF706FA174B0122D5
:106210001A7095F85830E2B26BB195F8273013B97F
:1062200026F8143003E0052B0CD00E2B0AD00021E9
:10623000284619F0F7FE0134112C05F17005E8D15C
:1062400002B070BD698A288AFFF7C6FEF3E700BF77
:10625000C8C5FF1F3C88FF1F58C6FF1FB8BCFF1FE3
:106260002EC4FF1F0488FF1F2688FF1F3A88FF1FC8
:106270002DE9F04FBA4FBB4E3A883388DFF83C9394
:106280009FB000240D46653B0A210A3A80468DE8FE
:1062900012001BB212B20121B3481EF0FBFF3A8874
:1062A000B1480A3A234612B201211EF043F9FEF723
:1062B000F7FDAE4B99F800001C70AD4B1C70FBF75E
:1062C000ABF9B8F10A0F40F09E803A88B6F800901A
:1062D000A84BA94916AD243A4FF00B0B92B24FF0E0
:1062E000050A4FEA5909284683F800B0049223F0C2
:1062F0003EFA2B46049ACDF800A049469F4814F078
:1063000033FB284623F0F3F93A889D491A3A4FF0B7
:106310001A0992B22846049223F029FA049A0294A8
:10632000214628230195CDF80090964813F05AFA9B
:10633000284623F0DCF933883A889349293B1A3AF6
:106340009BB292B228460493059223F010FA059A64
:106350000499029428230195CDF800908B4813F0FE
:1063600041FA284623F0C3F933883A88022044F2E0
:106370000821703B0C3A8DE803001BB212B23321A6
:1063800079481EF087FF824B187833883E3B2246BF
:106390000093FA213223FAF70CFA3F8804901A3F4F
:1063A000BFB27C49284623F0E2F943463A46BDF89D
:1063B000101002940195CDF80090774813F012FA6E
:1063C000284623F094F931886748CDF800B046F2AA
:1063D0002C333239019301222D2309B21EF05AFFCA
:1063E00036886E491E3EB6B2284623F0C0F9CDF875
:1063F00000A02B4603223146604814F0B5FA284627
:1064000023F075F90BE1B8F1080F26D1644E33780B
:106410001BB3DFF8A081594F4FF0140909FB04802A
:1064200013F070F8702303FB047301340025112C62
:10643000524883F85850F1D1012380F85830DC22BB
:1064400010238DE80C0002954FF49B730F22052159
:1064500019F036FE2C463570E1E0524B1C78002CCA
:1064600000F0DD80504B09AA03F1100716461868AA
:106470005968144603C40833BB422246F7D1186852
:106480009B882060A38008F13008314647488DF88A
:1064900034801AF0C3FB28B930238DF83430444BD4
:1064A00001221A7001233246404916A81AF072FBE5
:1064B000032089F80000FBF7AFF816A81AF029FAB4
:1064C0000446002800F09F803A4F2C4E00244FF0E5
:1064D000140808FB047013F015F8702303FB046321
:1064E00001340022112C83F85820F2D1324B0FAA2C
:1064F00003F11806904618685968144603C4083317
:10650000B3422246F7D10026186820603746344649
:10651000B14616A81AF0DEF900286FD016A81AF0B6
:1065200062F95FFA80FA15B1504622F0C1FDBAF166
:106530003B0F45D1072C06D81EAB2344013403F88A
:10654000609CE4B2F6E706A827F0C8F91EAB03EB9F
:106550004603013623F83C0CF6B20024D9E700BF0D
:106560003C88FF1F0488FF1F58C6FF1F10B9FF1F7C
:10657000C5C5FF1FFD87FF1FA2180300B8BCFF1F82
:106580002D1503005CB9FF1F2F15030070B9FF1F05
:1065900070C5FF1FCF1A030084B9FF1FEF17030058
:1065A0003A88FF1F27D5FF1FDD1803002CD5FF1FDA
:1065B0000688FF1F20B9FF1F9C1203002688FF1FBB
:1065C000BAF10D0F02D0BAF10A0F10D17EB1092E27
:1065D000384606AA414694BF8DF818908DF8209051
:1065E000FBF764FC00263844C7B2344691E71EAB83
:1065F0002344013403F860ACE4B28AE716A81AF029
:106600007CF9012408E008490848FAF76CF9324699
:106610000749084822F05DFF16A81AF037F920460E
:106620001FB0BDE8F08F00BFAC18030058C6FF1FB5
:10663000C3180300848AFF1F2DE9F04F8B469FB0DB
:106640000646002840F024830146BB48BB4DDFF8D6
:1066500080A31CF09CFC0121B7481CF092FCB84BB5
:10666000B548B3F9003001962A880C3A12B21AAC38
:10667000314600920C2228271EF00CFEB14920461C
:1066800023F075F83C233A4650210296AE48019417
:10669000009713F0A7F8204623F029F8AB492046CD
:1066A00023F065F83E233A469A210296A8480194C1
:1066B000009713F097F8204623F019F8A5492046D3
:1066C00023F055F83E23E22102963A46A24801946F
:1066D000009713F087F8204623F009F89AF8003065
:1066E0009E49A84612AE16AD2046002B39D04FF475
:1066F000FC6923F03CF83C235A2205219848CDF848
:1067000008900194009713F06DF8204622F0EFFFF7
:106710009249284623F02BF80A229AF80010B1FB80
:10672000F2F10EA823F056F80EA9304623F089F8AE
:106730008C49304623F036F90146204623F081F893
:106740004B4622462946864812F0A8FF204622F0F2
:10675000CEFF304622F0CBFF0EA822F0C8FF28461D
:106760000DE023F004F846F22C3302937C480194A8
:1067700000973C235A22052113F034F8204622F0DA
:10678000B6FF794B79491B78204623B122F0EFFF01
:106790004FF4FC6303E022F0EAFF46F22C3302934D
:1067A000282300935A223C2350217148019413F06E
:1067B00019F8204622F09BFF6E4B1B78012B06D167
:1067C0006D49204622F0D3FF4FF4FC631BE0022BFF
:1067D00001D16A4902E0032B06D16949204622F023
:1067E000C6FF4FF6E0730EE0042B06D16549204644
:1067F00022F0BDFF4FF4784305E06349204622F0C4
:10680000B6FF46F22C33029328235A229A21009392
:106810005E4801943E2312F0E5FF204622F067FF18
:106820004CF218695A492827204622F0A0FF3E233F
:106830005A22E2215748CDF808900194009712F0AF
:10684000D1FF204622F053FF5349204622F08FFF0C
:106850003C2305218C225148CDF8089001940097E3
:1068600012F0C0FF204622F042FF4D4B4D491B78ED
:1068700020462BB122F07BFF4FF6E073029303E03A
:1068800022F075FFCDF808903E238C22E22100977C
:106890004548019412F0A6FF204622F028FF434904
:1068A000284622F064FF4CF2186941492827204607
:1068B00022F05DFF3C23BE2205213E48CDF80C901E
:1068C00002940195009713F032F8204622F00FFF52
:1068D000284622F00CFF3849204622F048FF50217C
:1068E0003C238C223548CDF808900194009712F093
:1068F00079FF204622F0FBFE40F21B10F9F7A5FFBE
:106900002F490A2800F28480DFE800F06E060B10A1
:106910006469828282827800284622F028FF294911
:1069200070E0284622F023FF27496BE0284622F03A
:106930001EFF264966E000BF58C6FF1F3C88FF1FA8
:106940000488FF1FF318030034B9FF1FFB1803006E
:1069500048B9FF1F061903005CB9FF1F1019030097
:1069600070B9FF1F671A03003B88FF1F1619030049
:1069700084B9FF1F04B9FF1F1D1903002519030067
:10698000C0170300C61703002C19030098B9FF1F96
:1069900033190300D4B9FF1F3D190300ACB9FF1F21
:1069A000B8C7FF1F4619030038BAFF1F4F1903006D
:1069B000801D030010BAFF1F5519030074BAFF1F92
:1069C0005D190300661903006B19030071190300B8
:1069D00031C5FF1F284622F0CAFE974912E028461B
:1069E00022F0C5FE95490DE0284622F0C0FE9449EC
:1069F000204622F0BCFE4CF2186312E0284622F03A
:106A0000B6FE9049204622F0B2FE4FF4FC6308E047
:106A1000284622F0ACFE8C49204622F0A8FE4FF614
:106A2000E073039328235021BE22009387480294E9
:106A30003C23019512F07BFF204622F058FE2846A9
:106A400022F055FE824B83491B78012B04D1284646
:106A500022F08DFE804905E0022B09D1284622F064
:106A600086FE7749204622F082FE4CF218630AE047
:106A7000032B18D1284622F07AFE7849204622F0CE
:106A800076FE40F2FF73039328230093BE223C233B
:106A90009A2173480294019512F049FF204622F092
:106AA00026FE28460FE0204622F061FE46F22C33F7
:106AB0000293282300936A4801943C23BE229A2122
:106AC00012F090FE204622F012FE664B1B880BB39C
:106AD0006549304622F04BFE6449284622F047FEC5
:106AE0006349204622F043FE4FF478430493282361
:106AF000BE22E22100935F4803943C230295019655
:106B000012F0B0FE204622F0F2FD284622F0EFFD02
:106B1000304643E0584B1B78022B0AD15249284695
:106B200022F025FE5149204622F021FE4FF6E07367
:106B300025E003F0FD02012A0AD14B49284622F044
:106B400016FE4A49204622F012FE4FF4FC6316E07E
:106B5000042B0AD14949284622F009FE4349204620
:106B600022F005FE40F2FF7309E03F49284622F07B
:106B7000FEFD3E49204622F0FAFD46F22C330393F7
:106B800028230093BE223C23E2213A480294019537
:106B900012F0CDFE204622F0AAFD284622F0A7FDE5
:106BA000B8F800203648083A002312B201211DF03F
:106BB000C1FCFDF79DFD08230A2232493046F9F752
:106BC00091FC06223146284622F088FF2E492046B5
:106BD00022F0CDFD2146284622F05DFF07462046E3
:106BE00022F085FD284622F082FD67B906233A4649
:106BF0003146204622F052FF2146304622F02CFE3C
:106C0000204622F074FD46F22C311D481CF0BFF9DD
:106C1000B8F800201A48083A002312B2C8211DF023
:106C200089FC1A491648F9F75EFE3146144822F0ED
:106C300019FC01F034BE00BF751903007D19030073
:106C400049220300851903002F160300C0B9FF1F56
:106C5000ABC7FF1F8D190300352203001316030075
:106C600060BAFF1FC88EFF1F94190300271B030083
:106C7000E11D03004CBAFF1F6CC5FF1F9A190300EA
:106C800058C6FF1F38C5FF1FCF1A03009E19030007
:106C9000431E012B45F28D81DFF80C83B8F80040CC
:106CA0000328A4F165091FFA89F940F0CF80002775
:106CB000DFF8F8820197B8F80030B3480D3B1BB2FB
:106CC00000930D2223B239461EF0E4FA32463B46C9
:106CD0008221AD481DF02EFC1AADAC49AA48F9F747
:106CE00002FE4FF01A0AAA49284622F040FD64230A
:106CF0000E224946A74802970195CDF800A012F050
:106D000071FD284622F0F3FCB8F80080A249A8F1F2
:106D10001A081FFA88F8284622F029FD4246642303
:106D200049469E4802970195CDF800A012F05AFD01
:106D3000284622F0DCFC4FF6FF719348DFF874829E
:106D40001CF025F932463B4682218F481DF0F2FBAC
:106D50008E498D48F9F7C7FD2A260797904B9DF875
:106D60001C701B78711EBB4289B203D8002105201C
:106D700000F029BC2FB98B4A3B4612784846FBF7F6
:106D800021F8A4F15E0B4FF6FF717F481FFA8BFBD1
:106D90000FFA86FA1CF0FBF8002352460FFA8BF12B
:106DA00079481DF0C7FBD8F8042040F6FF739A42DB
:106DB00014D198F80930032B10D8A4F1570152468A
:106DC000002309B270481DF0B5FB3946032013F0CB
:106DD0003DFA314602465846FCF79AF8724B39465E
:106DE000B3F800A0012013F031FAAAF1140A1FFA37
:106DF0008AFA024631465046FBF79EFF6A4B3946F7
:106E0000B3F800A0002013F021FAAAF10A0A1FFA31
:106E10008AFA024631465046FBF754FF604B0B227C
:106E20001B783946284613F039FA2946564822F08D
:106E300019FB284622F05BFC079B01330D360D2B16
:106E40000793B6B208F1A80888D18FE7042840F06C
:106E5000B3800025554E019533884B48544F423B33
:106E60001BB20FFA89F10093282264231EF012FA54
:106E70004D4B32881B88444801951A21643B1A3ACD
:106E800000911BB2294612B21EF004FA32883E4825
:106E9000DFF80C910A3A2B4612B201211DF04AFB91
:106EA0004FF6FF7138481CF072F83D782A26CB4621
:106EB0003B780C33AB42C5F27C8099F80030AB4292
:106EC00045F27780A4F15E084FF6FF712E481FFA55
:106ED00088F80FFA86FA1CF05AF8002352460FFA87
:106EE00088F129481DF026FB324AA82303FB05231D
:106EF00040F6FF725968914213D15B7A032B10D888
:106F0000A4F157015246002309B21F481DF012FB9D
:106F10002946032013F09AF9314602464046FBF712
:106F2000F7FF214B2946B3F80080012013F08EF9BA
:106F3000A8F114081FFA88F8024631464046FBF7CC
:106F4000FBFE194B2946B3F80080002013F07EF9B0
:106F5000A8F10A081FFA88F8024631464046FBF7B6
:106F6000B1FE9BF800300B2229461AA813F096F9BF
:106F70001AA9054822F076FA01351AA80D3622F032
:106F8000B6FBEDB2B6B293E758C6FF1FF318030085
:106F9000A919030020B9FF1FAC19030034B9FF1F62
:106FA0002AC4FF1FA0C5FF1F0488FF1F3C88FF1FC6
:106FB000E88EFF1F008FFF1F052840F0A5820025E7
:106FC000C34A01951288C348DFF848930D3AA4F1EB
:106FD000660312B21BB2009229460D221EF05AF926
:106FE0004FF6FF71BB48BC4C1BF0D1FF0121B948E3
:106FF0001BF0C7FFB949B7481CF01EF831462B46B5
:107000002422B448B64E1DF095FA99F80030217844
:107010000F221AA813F042F91AA9AE4822F022FA58
:107020001AA822F064FBAB481CF020F84CF218615F
:10703000A8481BF0ACFF2B462D220D21A5481DF0C2
:1070400079FAA849A348F9F74EFC2B462D225F2177
:10705000A0481DF06FFAA4499E48F9F744FC237834
:107060009C48A8274FF00208CDF8008007FB036377
:10707000D3E91023F9F745FC4FF6FF7195481BF053
:1070800086FF2B463A220D2192481DF053FA97496C
:107090009048F9F728FC2B463A225F218D481DF0D5
:1070A00049FA91498B48F9F71EFC2378CDF8008006
:1070B00007FB0363D3E912238648F9F722FC4CF25D
:1070C000186184481BF063FF2B4647220D2181483D
:1070D0001DF030FA86497F48F9F705FC2B46472218
:1070E0005F217C481DF026FA7F497A48F9F7FBFBBF
:1070F0002378CDF8008007FB0363D3E91423754898
:10710000F9F7FFFB4FF6FF7172481BF040FF2B466B
:1071100054220D216F481DF00DFA76496D48F9F79C
:10712000E2FB2B4654225F216A481DF003FA6E49A8
:107130006848F9F7D8FB2378CDF8008007FB036394
:10714000D3E916236348F9F7DCFB2B466E220D21A9
:1071500060481DF0EFF968495E48F9F7C4FB2B461B
:107160006E225F215B481DF0E5F95F495948F9F748
:10717000BAFB2178284613F069F8FBF7DFFE217887
:10718000284613F063F86D2102465120FBF79AFD63
:107190002B467B220D214F481DF0CCF957494D4815
:1071A000F9F7A1FB2B467B2233214A481DF0C2F997
:1071B00053494848F9F797FB7B222B463D21454828
:1071C0001DF0B8F94F4B43481978F9F790FB2B465F
:1071D0007B2247213F481DF0ADF94B493D48F9F767
:1071E00082FB2B467B225F213A481DF0A3F93E49E2
:1071F0003848F9F778FB2178012013F027F8FBF7DE
:107200009DFE2178012013F021F87A2102465120B9
:10721000FBF792FD237807FB036340F6FF72596882
:107220009142B04625D15B7A032B22D82B46882287
:107230000D2128481DF07EF934492648F9F753FB03
:1072400088222B465F2123481DF074F926492148E6
:10725000F9F749FB2178032012F0F8FFFBF76EFEE7
:107260002178032012F0F2FF892102465120FBF71A
:107270004FFE002395220D2116481DF05BF924498D
:107280001448F9F730FB002395225F2111481DF0C7
:1072900051F915490F48F9F726FB217899F8003084
:1072A000A82505FB0181002291F891101AA812F07F
:1072B000F5FF1AA9074822F0D5F81AA822F017FA04
:1072C0000023A2220D2103481DF034F924E000BF61
:1072D0003C88FF1F58C6FF1FA0C5FF1F302B0300AF
:1072E000008FFF1FAF190300B7190300BB1903007C
:1072F000C8190300D0190300DD1903001019030099
:10730000E2190300BBC7FF1FEB330300E4190300BE
:10731000EB1903002AC4FF1FAD49AE48F9F7E3FAA1
:107320000023A2225F21AB481DF004F9AA49A94815
:10733000F9F7D9FA237805FB038393F89120FF2A04
:1073400004D1A649A348F9F7CEFA06E0022200923A
:10735000D3E926239F48F9F7D4FA0023AF220D2161
:107360009C489F4E9F4F1DF0E5F89F499948F9F7BB
:10737000BAFA0023AF225F2196481DF0DBF8964948
:107380009448F9F7B0FA2378A82505FB038393F80E
:107390006800FBF7D3FD237805FB038898F8683075
:1073A000012B36D10023BC220D218A481DF0C2F8E2
:1073B0008E498848F9F797FA0023BC225F21854857
:1073C0001DF0B8F884498348F9F78DFA3B78814875
:1073D000022405FB03630094D3E92023F9F791FA13
:1073E0000023C9220D217B481DF0A4F8804979486B
:1073F000F9F779FA0023C9225F2176481DF09AF83F
:1074000075497448F9F76FFA3B78009405FB0365FA
:1074100073E0022B44F0CD850023BC220D216D4882
:107420001DF088F873496B48F9F75DFA0023BC2218
:10743000172168481DF07EF867496648F9F753FA46
:107440003B786448082405FB03630094D3E91C23BC
:10745000F9F757FA0023C9220D215E481DF06AF89A
:1074600065495C48F9F73FFA0023C92217215948BA
:107470001DF060F858495748F9F735FA3B78009401
:1074800005FB0363D3E91E235248F9F73AFA0023B8
:10749000BC2271214F481DF04DF858494D48F9F76D
:1074A00022FA0023BC227B214A481DF043F84A49B6
:1074B0004848F9F718FA3B78009405FB0363D3E9D1
:1074C00020234448F9F71DFA0023C92271214148BD
:1074D0001DF030F84A493F48F9F705FA0023C92260
:1074E0007B213C481DF026F83B493A48F9F7FBF967
:1074F0003B7805FB036500230093D5E9222335483B
:10750000F9F7FFF904F055BD062840F08D800025FD
:107510003C4E019533882F48443B1BB21AAC2822BD
:1075200000930FFA89F164231DF0B4FE364920461A
:1075300022F01DF934234222494600933348029534
:107540006423019412F04EF9204622F0D0F81A2755
:107550002F49204622F00BF96423AA2249462D48E0
:1075600002950194009712F03DF9204622F0BFF8F1
:107570002949204622F0FBF864230E224946274879
:1075800002950194009712F02DF9204622F0AFF8F1
:10759000368823491A3EB6B2204622F0E8F8642322
:1075A000324649461F4802950194009712F01AF995
:1075B000204622F09CF82C2102202B465A46FAF74E
:1075C00001FC29460720FFF737F804F0F2BC00BFA2
:1075D000F519030058C6FF1FB7190300FE19030071
:1075E000008FFF1FA0C5FF1F021A0300091A030026
:1075F0000C1A0300001A0300B01703006D490300C2
:107600009C1803003C88FF1F1618030048B9FF1F91
:107610000F1A0300D4B9FF1FA919030020B9FF1FD7
:10762000AC19030034B9FF1F072829D161B9114AE9
:10763000128801911A20A4F164031A3A00901BB237
:1076400012B20D481DF026FE00210B481BF09FFCD6
:107650000A4B1A78052A1AAC1D4604F091811A7853
:10766000062A04F08D811A78072A44F0AE8104F0CE
:1076700087B900BF3C88FF1F58C6FF1FE6C6FF1F23
:10768000092840F06F83FF2940F0C2810025DFF810
:1076900078A3BF4EDFF874B3FDF702FCB8F90030F1
:1076A0000195BAF80020BB480D3A12B20092294663
:1076B0000D221DF0EFFDB849B6481BF0BDFC2B466E
:1076C00024220521B3481CF035FFB449B148F9F72D
:1076D0000AF9FDF7E5FBB2481AAC11F013FFB14807
:1076E00011F010FFB049204622F041F83423422225
:1076F000494601940093AD480295642312F072F854
:10770000204621F0F4FFAA49204622F030F8737891
:10771000A8483BF8133002931A276423792249467C
:107720000194009712F05EF8204621F0E0FFA24994
:10773000204622F01CF8642349460E2201949F48FB
:107740000295009712F04EF8204621F0D0FFBAF8CB
:1077500000209B491A3A92B22046079222F007F87D
:107760006423079A0194494696480295009712F0BF
:1077700039F8204621F0BBFFBAF800909249A9F1F0
:107780001A091FFA89F9204621F0F1FF13234A460E
:10779000294601948D480295009712F023F820465F
:1077A00021F0A5FFB8F80090BAF800208849A9F1A7
:1077B0007D091A3A92B21FFA89F92046079221F000
:1077C000D6FF49461323079A0194824802950097F1
:1077D00012F008F8204621F08AFFB8F80030BAF815
:1077E00000206C4844F2082E0221A03B0C3A8DE8A0
:1077F00002401BB212B219211DF04CFDB8F8000076
:10780000963825F001F80022734B24F0AFFE804635
:107810003078894624F0E8FF02460B464046494648
:1078200025F058F800226D4B25F07EF900226A4BB6
:1078300024F09EFE25F026FBBAF800806849A8F1E6
:107840001A081FFA80F91FFA88F8204621F08FFFE6
:107850000A2342464946019462480295009711F076
:10786000C1FF204621F043FFFDF71AFB2D2427B26C
:107870003A4600230D2147481CF05CFE05F1010843
:1078800059494448F9F72FF841464248F9F733F887
:1078900006EB4503621E5B783E483BF813300193CC
:1078A0000923009312B20A2373211DF0F3FC3A4618
:1078B00000233F2137481CF03DFE16F815103548CF
:1078C0006423594345461F460D34F9F714F8082D33
:1078D000A4B2CCD1A22200230D212E481CF02AFEF6
:1078E00042492C48F8F7FFFF414B187824F07CFF01
:1078F0000323002467250293A223019302460B462B
:107900000494039400953B4814F0A6FA2346AF2252
:107910000D2120481CF00EFE37491E48F8F7E3FF02
:10792000364B187810FB07F024F06EFF0526AF23C6
:10793000019302460B4604940394029600952D4849
:1079400014F08AFA2346BC220D2112481CF0F2FDE5
:107950002B491048F8F7C7FFBC2301930494039404
:107960000296009500220023224814F075FA23465F
:10797000C9220D2107481CF0DDFD22490548F8F712
:10798000B2FF234622462D210220FAF71BFABCE162
:107990002788FF1F58C6FF1F302B0300FB1803006A
:1079A000ACB9FF1FC0B9FF1F1F1A030048B9FF1F62
:1079B000241A030098B9FF1FA919030020B9FF1F5B
:1079C000AC19030034B9FF1F2D1503005CB9FF1F6C
:1079D0002F15030070B9FF1F0000394000005E4002
:1079E000CF1A030084B9FF1F2A1A03002F1A0300BD
:1079F000FC87FF1FB8BCFF1F3B1A03003988FF1F1D
:107A0000471A03004F1903003C88FF1F1088FF1F0F
:107A1000012940F07A81C14D2E78082E5ED8C04FE2
:107A2000963C17F816000094192378220021F8F7E5
:107A3000C0FEBC4EA3B281B2192206F1640011F05F
:107A4000C7FFFDF72DFA2B78B74803EB430203EB92
:107A5000820200240A232D328DE8180012B21E2360
:107A60003F211DF017FC2B78AF4803EB430203EBDB
:107A700082022D3212B223463F211CF05BFD2B788F
:107A8000A94817F81310642359431AACF8F733FFC9
:107A9000A649B6F88080B6F88290B6F884A0B6F809
:107AA00086B0204621F063FE2B7807EB4307A04BFE
:107AB0007A7833F8123002934A465346414606F12B
:107AC00078000194CDF800B011F08CFE204621F032
:107AD0000EFE06F18C00F8F741FF88E0092E27D151
:107AE000944E963C307800941923FF220021F8F739
:107AF00060FEA3B281B219228F4811F069FFFDF731
:107B0000CFF92B78884803EB430203EB8202002471
:107B10000A232D328DE8180012B21E2367211DF0B2
:107B2000B9FB307824F060FE0494039403234EE004
:107B30000A2E21D1814F963C38780094192378225F
:107B40000021F8F736FEA3B281B219227A4811F06B
:107B50003FFFFDF7A5F92B787348009603EB43022E
:107B600003EB82022D32002401941E2312B26721FE
:107B70001DF090FB387823E00B2E38D1704E963CE8
:107B800030780094192378220021F8F712FEA3B26E
:107B900081B21922684811F01BFFFDF781F92B789B
:107BA000614803EB430203EB82022D320A230024D7
:107BB0008DE8180012B21E2367211DF06BFB307890
:107BC0006423584324F020FE049403940523029375
:107BD0002B7803EB430203EB82032D339BB201931B
:107BE0006723009302460B46564814F035F92B786C
:107BF0000C2B40F08A804FF4D470F8F726FE494CE5
:107C00005149B4F88060B4F88270B4F88480B4F854
:107C1000869001281AAD0CBF4FF01F0A4FF4FC6A82
:107C2000284621F0A4FD3A4643463146CDF808A047
:107C3000CDF8009004F17800019511F0D3FD2846AD
:107C400021F055FD4149B4F88690B4F88080B4F82D
:107C500084A0B4F8826016A821F089FD3C4B12A8DC
:107C6000197821F0A4FD12A916A821F093FE4E4424
:107C700003360146B6B20027284621F0E2FD32461F
:107C800053464146CDF8009004F18C0002970195CF
:107C900011F0A8FD284621F02AFD12A821F027FDA9
:107CA00016A821F024FDB4F89A30B4F89660B4F820
:107CB0008080B4F88490B4F886A01E44254B12A8A6
:107CC000197821F074FD12A916A821F0BAFD2249F5
:107CD00016A821F067FE03360146B6B2284621F009
:107CE000B0FD4B463246414604F1A0000297019593
:107CF000CDF800A011F076FD284621F0F8FC16A87A
:107D000021F0F5FC12A803F0AABF1448F8F726FEEC
:107D10001348F8F723FE04F04CB900BFA0C5FF1FBD
:107D20002788FF1F20B9FF1F58C6FF1F241A030012
:107D30001088FF1FFC87FF1F84B9FF1F3988FF1FB2
:107D4000368EFF1FB8BCFF1F531A03005D1A0300D5
:107D5000F08EFF1F2BC4FF1F631A0300ACB9FF1F77
:107D6000C0B9FF1F0A286FD100220C2044F208235B
:107D700011468DE8090023B2AF481DF08BFAFDF7DC
:107D80008FF8002303228221AB481CF0D3FBAB49C0
:107D9000A948F8F7A8FDB8F80010A7480B2646F246
:107DA0002C3732392D23012209B28DE8C0001DF095
:107DB00071FAB8F80040A2491E3C0525A4B21AA8E1
:107DC00021F0D5FC1AAB032221469E48009512F003
:107DD000CBFD1AA821F08BFCBBF1000F0CBF3B467A
:107DE0004FF478430122019329462E2392480096AE
:107DF0001DF050FA94491AA821F0B9FC1AAB0322DD
:107E000019219048009512F0AFFD1AA821F06FFCDF
:107E1000BBF1000F0CBF4FF478433B4601220193A6
:107E200037212E23844800961DF034FA87491AA87A
:107E300021F09DFC834800951AAB03224B2112F0E0
:107E400093FD1AA803F00BBF0B2804F0B2800C2896
:107E500040F0A68100267E4F01963B8876480D3B78
:107E60001BB20D220093314623B21DF013FA4FF6D8
:107E7000FF7171481BF08BF801216F481BF081F8EE
:107E800074496D481BF0D8F83346242205216A480E
:107E90001CF050FB70496848F8F725FD66481BF058
:107EA000E5F83A8864480A3A334612B205211AAC1A
:107EB0001CF040FB69496048F8F715FD08230A22C9
:107EC00067492046F8F70EFB21465B4821F0CAFAC5
:107ED000204621F00CFC3A8857480A214FF4784399
:107EE0000B3A12B28DE80A0016AD782331461BF02A
:107EF0001BFB5C49284621F03AFC40F29F10F8F742
:107F0000A4FC24F071FC02460B4600204FF0804197
:107F100021F0E8FF544B002224F0DCFC24F0D2FFD7
:107F20004FF0280801460222204621F0A6FC3C23FF
:107F3000912205214D48039602940195CDF80080C9
:107F400011F0F5FC204621F0D2FB284621F0CFFBB2
:107F50004749204621F00BFC05213C232D224548B2
:107F600002960194CDF8008011F03CFC204621F0EF
:107F7000BEFB4FF4E570F8F768FCBA463E493F4F48
:107F800048B1284621F0F3FB3D49204621F0EFFBA4
:107F90004FF4FC6308E0284621F0E9FB384920460D
:107FA00021F0E5FB46F22C335F2205210393CDF847
:107FB00000803C2307F164000294019511F0B7FCA6
:107FC000204621F094FB284621F091FB2D492846BC
:107FD00021F0CDFB2C49204621F0C9FB4FF02808A9
:107FE0004CF2186350215F220393284802943C23EB
:107FF0000195CDF8008011F09AFC204621F077FB26
:10800000284621F074FB4FF4D870F8F75AFC12AEF2
:1080100083461F493046BBF1000F3FD021F0A7FB3C
:108020001C49284621F0A3FB1B49204621F09FFB59
:108030004FF4FC6304933DE058C6FF1F061903008C
:10804000691A0300B8BCFF1F391903006E1A030038
:108050003C88FF1F302B03003D190300751A0300F5
:1080600038C5FF1F881A030000405F4048B9FF1F52
:10807000921A03005CB9FF1F971A030020B9FF1F73
:108080009F1A0300EE190300BE1A030098B9FF1FE0
:10809000141D0300F41D03005521030021F067FBAC
:1080A0003649284621F063FB3549204621F05FFB25
:1080B000CDF810B03C239122502102950196CDF8C5
:1080C000008003942F4811F0CDFB204621F00FFBD8
:1080D000284621F00CFB304621F009FB40F2191034
:1080E000F8F7B3FB2D239B220821FAF7F9FC264968
:1080F000204621F03CFB002628235F2200939B2191
:108100003C2302960194214811F06CFB204621F09B
:10811000EEFA4FF01A081E49204621F028FB64238E
:108120000E22494602960194CDF80080194811F0BC
:1081300059FB204621F0DBFABAF8005016491A3DE7
:10814000ADB2204621F013FB2A464946642302962D
:108150000194CDF80080114811F044FB204621F035
:10816000C6FAFDF74DFAFB897989388919443246F8
:10817000334689B2F9F726FE03F01BBFF41D030056
:10818000A71A0300ACB9FF1FB01A0300D4B9FF1F30
:10819000A919030020B9FF1FAC19030034B9FF1F50
:1081A0000D2840F00485FF2940F0DD83BC4D0024FC
:1081B0002819143411F0A6F9B4F5027FF8D1B94B9F
:1081C000B94AB3F90030B948B94EBA4F0024019406
:1081D00012880D3A12B2009221460D221DF05AF873
:1081E00046F22C35032202238DE82C0005214FF4A2
:1081F0009B738C22AD481DF0A5F84FF6FF71AB487C
:108200001AF0C5FE0121A9481AF0BBFEAA49A748E9
:108210001AF012FF234624220521A4481CF08AF9F3
:10822000A649A248F8F75FFBA0481AF01FFF2946AD
:108230009E481AF0ACFE3068716832890EAB03C3F9
:1082400001201A80F8F701FB3B7883420CD99C4B44
:10825000A82202FB003000F110030EAA53F8050F0C
:1082600059681B7A03C2137016AC1AAD4FF00008A0
:1082700094498DF84180204621F079FA0EA92846CC
:1082800021F075FA28232D22052100938448CDF88A
:108290000C803C230295019411F049FB284621F003
:1082A00026FA204621F023FA30687168327A0EAB44
:1082B00003C303201A70F8F7C8FA3B7883420CD93D
:1082C0007F4BA82202FB003000F110030EAA53F8E6
:1082D000050F59681B7A03C213704FF000087A49E2
:1082E0008DF84180204621F042FA0EA9284621F05F
:1082F0003EFA28232D22502100937448CDF80C809B
:108300003C230295019411F012FB284621F0EFF96D
:10831000204621F0ECF930687168327A0EAB03C365
:1083200004201A70F8F791FA3B7883420CD9644B19
:10833000A82202FB003000F110030EAA53F8050F2B
:1083400059681B7A03C213704FF0000860498DF81A
:108350004180204621F00BFA0EA9284621F007FAA9
:1083600028232D229B2100935A48CDF80C803C23D2
:108370000295019411F0DBFA284621F0B8F9204665
:1083800021F0B5F930687168327A0EAB03C305206D
:108390001A70F8F75AFA3B7883420CD9484BA82256
:1083A00002FB003000F110030EAA53F8050F5968C4
:1083B0001B7A03C213704FF0000847498DF84180C3
:1083C000204621F0D4F90EA9284621F0D0F928231F
:1083D0002D22E62100934148CDF80C803C230295E4
:1083E000019411F0A4FA284621F081F9204621F0E9
:1083F0007EF930687168327A0EAB03C306201A70BA
:10840000F8F723FA3B7883420CD92D4BA82202FBC4
:10841000003000F110030EAA53F8050F59681B7ABB
:1084200003C2137000272E498DF84170204621F0B9
:108430009EF90EA9284621F09AF9039728273C2394
:108440005A220521274802950194009711F06FFAEE
:10845000284621F04CF9204621F049F9306871682E
:10846000327A0EAB03C31A701F4B20491E78012EBF
:10847000204603D121F07BF91D4958E0022E03D19B
:1084800021F075F91B4952E0032E03D121F06FF959
:1084900019494CE0042E33D121F069F9174946E01F
:1084A00020B9FF1F0488FF1F3C88FF1F58C6FF1F0D
:1084B000C71A03002AC4FF1F302B0300B71A03009A
:1084C000008FFF1FC31A03008C1A030048B9FF1F57
:1084D000D11A03005CB9FF1FD81A030070B9FF1F3F
:1084E000DF1A03004CBAFF1F348DFF1FE41A03008C
:1084F000F01A0300F41A0300F81A0300FC1A030030
:10850000052E0FD121F033F9B349284621F02FF978
:108510004FF4FC6303930295019400973C23962249
:10852000314619E0062E08D121F021F9AB49284641
:1085300021F01DF94FF4FC6307E021F018F9A84978
:10854000284621F014F946F22C3303930295019446
:1085500000973C2396220521A24811F0E8F928460D
:1085600021F0C5F8204621F0C2F89F4B9F491B78A7
:1085700012AE012B304607D121F0F9F89C49204674
:1085800021F0F5F89B4930E0022B07D121F0EFF8FC
:108590009749204621F0EBF8974926E0032B07D1B5
:1085A00021F0E5F89249204621F0E1F893491CE0DA
:1085B000042B07D121F0DBF88D49204621F0D7F8B4
:1085C0008F4912E0052B07D121F0D1F888492046C8
:1085D00021F0CDF8804908E0062B0CD121F0C7F836
:1085E0008349204621F0C3F87C49284621F0BFF892
:1085F0004FF4FC630BE021F0BAF87D49204621F0EE
:10860000B6F87749284621F0B2F846F22C330493A5
:1086100028239622E62100937A4803953C2302946E
:10862000019611F01FF9284621F061F8204621F04B
:108630005EF8304621F05BF8734BDFF8E4911A786E
:1086400099F80080FF2A4FF4CD709A464FF6E077F4
:1086500018BF4FF4FC67F8F7F8F8804505D16B496F
:10866000204621F084F863493EE040F29B10F8F781
:10867000ECF8804505D16549204621F078F85E493F
:1086800032E04FF4CE70F8F7E0F8804505D15F494D
:10869000204621F06CF8594926E040F29D10F8F789
:1086A000D4F880455949204603D121F060F8544957
:1086B0001AE0B8F1000F03D121F059F8464913E050
:1086C000B8F1010F03D121F052F844490CE0B8F1A0
:1086D000090F03D121F04BF84D4905E0B8F10A0F1D
:1086E00007D121F044F84B49284621F040F8039780
:1086F00008E021F03CF83A49284621F038F846F2E3
:108700002C3303932823962250210093424802954C
:108710003C23019411F00BF9284620F0E8FF204695
:1087200020F0E5FF9AF8013099F80180FF2B4FF413
:10873000CD704FF6E07718BF4FF4FC67F8F785F877
:10874000804505D13549204621F011F829493EE000
:1087500040F29B10F8F779F8804505D12F49204663
:1087600021F005F8244932E04FF4CE70F8F76DF8A7
:10877000804505D12949204620F0F9FF1F4926E010
:1087800040F29D10F8F761F880452449204603D156
:1087900020F0EDFF1A491AE0B8F1000F03D120F0E4
:1087A000E6FF0D4913E0B8F1010F03D120F0DFFF20
:1087B0000A490CE0B8F1090F03D120F0D8FF1449A1
:1087C00005E0B8F10A0F2DD120F0D1FF114928465C
:1087D00020F0CDFF03972EE03B1603003716030071
:1087E0000C1D030034B9FF1FECC4FF1F001B030066
:1087F000E91A0300F01A0300F41A0300F81A030040
:10880000FC1A0300E8B9FF1F3788FF1F0B1B03008A
:108810003F1603004316030010BAFF1F131B03008B
:10882000B9C7FF1F20F0A3FF6849284620F09FFF2B
:1088300046F22C33039328239B219622009364480D
:1088400002953C23019411F072F8284620F04FFF66
:10885000204620F04CFF5F4B5F491F78012F3046C8
:1088600020D120F084FF5D49204620F080FF5C4944
:10887000284620F07CFF4FF4FC63049328230093E8
:108880000395029401963C23C3220521554810F01C
:10889000E9FF284620F02BFF204620F028FF304635
:1088A00003F0DDB9022F07D120F061FF4B492046CC
:1088B00020F05DFF4C49DBE7032F07D120F057FF85
:1088C0004649204620F053FF4849D1E7042F07D1FD
:1088D00020F04DFF4149204620F049FF4449C7E7B9
:1088E000052F15D120F043FF3C49204620F03FFFE3
:1088F0004049284620F03BFF4FF4FC6304932823B3
:1089000000930395029401963C23C3223946BDE7A8
:10891000062F07D120F02BFF3049204620F027FFFB
:108920003549A5E7072F07D120F021FF2B49204625
:1089300020F01DFF31499BE7082F07D120F017FFDA
:108940002649204620F013FF2D4991E720F00FFF24
:108950002249204620F00BFF1C49284620F007FF43
:1089600046F22C3389E72749274B0A781B78DFF832
:108970009C90501E9842884616D00AB9FF2B13D0FF
:108980009A4217D099F800108A4201D1FF2B11D0DA
:10899000501C834213D08A4200D183B101398A42EC
:1089A00036D1FF2B34D10AE044F208252E464FF48D
:1089B000FC6731E044F208254FF4FC662BE044F2FA
:1089C00008264FF4FC65374626E000BF0C1D030067
:1089D00024BAFF1FE4C6FF1F1B1B03007916030008
:1089E000F01A030038BAFF1FF41A0300F81A030044
:1089F000FC1A03003B160300371603003F16030062
:108A000043160300A0C5FF1FE88EFF1F2AC4FF1FE7
:108A100044F208252E462F46DFF860A28A49BAF8AC
:108A200000B01AACABF11A0B204620F0A0FE1FFAE2
:108A30008BFB02971A275A46332337218348019428
:108A4000009710F0CFFE204620F051FEBAF800202B
:108A50007F48113A002312B239211BF06BFD98F8C0
:108A6000001099F8003001390822C9B2204611F0EF
:108A700015FC2146764820F0F5FC204620F037FE14
:108A8000BAF800B07049ABF11A0B1FFA8BFB204605
:108A900020F06DFE33235A46702102966D480194F2
:108AA000009710F09FFE204620F021FEBAF800202B
:108AB0006748113A002312B273211BF03BFD99F86D
:108AC000003098F800100822204611F0E7FB2146FC
:108AD0005F4820F0C7FC204620F009FEBAF800608D
:108AE00059491A3EB6B2204620F041FE32463323A1
:108AF000A921029558480194009710F073FE204672
:108B000020F0F5FDBAF800205148113A002312B2C6
:108B1000AC211BF00FFD98F8001099F800300131DE
:108B20000822C9B2204611F0B9FB2146484820F07E
:108B300099FC204620F0DBFDBAF8005047491A3D69
:108B40000026ADB2204620F012FE2A4633233146DD
:108B5000434802960194009710F044FE204620F00E
:108B6000C6FDBAF800503F491A3DADB2204620F08C
:108B7000FEFD2A463323E2213B48029601940097EA
:108B800010F030FE204620F0B2FDBAF80050374910
:108B90001A3DADB2204620F0EAFD029601940097FE
:108BA00027232A464FF48C71314801F09ABC1428CF
:108BB00040F03984FF29DFF8C8804FF0000600F04C
:108BC00032812D22631F009201961BB2C322052120
:108BD0001F481CF05FFB08EB0600143610F092FCF7
:108BE000B6F5027FF7D12349234B0A781B78DFF8CB
:108BF0009490501E9842884615D00AB9FF2B12D087
:108C00009A4216D099F800108A4201D1FF2B10D059
:108C1000501C834212D08A4200D17BB1884233D1AA
:108C2000FF2B31D10AE044F208252E464FF4FC67B1
:108C30002EE044F208254FF4FC6628E044F20826B2
:108C40004FF4FC65374623E0CF1A030084B9FF1FB9
:108C500058C6FF1F98B9FF1FACB9FF1F2D150300A1
:108C6000C0B9FF1F2F150300D4B9FF1F161803004A
:108C7000FCB9FF1FA0C5FF1FE88EFF1F3C88FF1F28
:108C800020B9FF1F2AC4FF1F44F208252E462F4695
:108C9000DFF82CA3BF49BAF800B01AACABF11A0B3D
:108CA000204620F064FD1FFA8BFB02971A275A46D4
:108CB00033233721B8480194009710F093FD2046E4
:108CC00020F015FDBAF80020B448113A002312B282
:108CD00039211BF02FFC98F8001099F80030013969
:108CE0000822C9B2204611F0D9FA2146AB4820F03B
:108CF000B9FB204620F0FBFCBAF800B0A549ABF167
:108D00001A0B1FFA8BFB204620F031FD33235A4605
:108D100070210296A2480194009710F063FD20464E
:108D200020F0E5FCBAF800209C48113A002312B26A
:108D300073211BF0FFFB99F8003098F8001008220F
:108D4000204611F0ABFA2146944820F08BFB2046D8
:108D500020F0CDFCBAF800608E491A3EB6B220462B
:108D600020F005FD32463323A92102958D48019458
:108D7000009710F037FD204620F0B9FCBAF800202B
:108D80008648113A002312B2AC211BF0D3FB98F8AD
:108D9000001099F8003001310822C9B2204611F0C4
:108DA0007DFA21467D4820F05DFB204620F09FFCA7
:108DB000BAF800507C491A3D0026ADB2204620F09A
:108DC000D6FC2A4633233146784802960194009710
:108DD00010F008FD204620F08AFCBAF800507449D3
:108DE0001A3DADB2204620F0C2FC2A463323E221D0
:108DF000704802960194009710F0F4FC204620F091
:108E000076FCBAF800506C491A3DADB2204620F00D
:108E1000AEFC02960194009727232A464FF48C71EA
:108E2000664801F05EBB664B01961B885B480D3BB4
:108E30001BB20D220093314623B21CF02BFA4FF6E1
:108E4000FF7156481AF0A3F8012154481AF099F816
:108E50005C4952481AF0F0F83346242205214F4865
:108E60001BF068FB58494D481AADF7F73CFD4B48DD
:108E70001AF0FCF85549284620F079FC544B16AC02
:108E8000282719880A22204620F0A4FC2D223C2302
:108E900005214046039602940195009710F047FD86
:108EA000204620F024FC284620F021FC4949284691
:108EB00020F05DFC484B20461978F9F7DFFE2D22A3
:108EC0003C23502108F11400039602940195009769
:108ED00010F02DFD204620F00AFC284620F007FC6B
:108EE0003E49284620F043FC3D4B2046197820F0AF
:108EF0005EFC2D223C239B2108EB07000396029485
:108F00000195009710F013FD204620F0F0FB284655
:108F100020F0EDFB3349284620F029FC324B204657
:108F2000197820F044FC3C2308EB03002D22E621B5
:108F3000039602940195009710F0F9FC204620F06A
:108F4000D6FB284620F0D3FB284A1378012B914604
:108F50000AD12749204620F00AFC2649284620F05D
:108F600006FC4FF4FC6355E0032B05D12049204655
:108F700020F0FDFB204906E0042B41D11F4920468B
:108F800020F0F5FB1B49284620F0F1FB40F2FF736F
:108F900040E000BFCF1A0300E8B9FF1F58C6FF1F0B
:108FA000FCB9FF1F10BAFF1F2D15030024BAFF1FC5
:108FB0002F15030038BAFF1F161803004CBAFF1F05
:108FC0003C88FF1F302B0300211B03002F1B0300D5
:108FD000EEC4FF1F391B03000EB9FF1F3E1B030029
:108FE00000B9FF1F491B0300EAC9FF1F6CC5FF1F23
:108FF000541B0300FA1C03005B1B03009A190300B7
:10900000A749204620F0B3FBA649284620F0AFFB35
:109010004FF6E0735A220521039308F150003C23D8
:1090200002950194009710F082FC284620F05FFB27
:10903000204620F05CFB9C4B1E7876B9314640F20E
:10904000CF10F7F795FB9949204620F090FB954902
:10905000284620F08CFB03960FE0012140F2CF1050
:10906000F7F786FB9149204620F081FB904928467E
:1090700020F07DFB4FF4FC63039328235A225021F8
:1090800000938C4802953C23019410F050FC284634
:1090900020F02DFB204620F02AFB99F80030032B0E
:1090A00040F081808449204620F061FB002728267B
:1090B0008249284620F05BFB3C235A229B218048B2
:1090C000039702950194009610F031FC284620F099
:1090D0000EFB204620F00BFB7A49284620F047FB88
:1090E000794B0A221988204620F074FB3C23872202
:1090F00005217648039702940195009610F017FC1D
:10910000204620F0F4FA284620F0F1FA704928466B
:1091100020F02DFB6F4B0A221988204620F05AFBC5
:109120003C23872250216C480397029401950096B6
:1091300010F0FDFB204620F0DAFA284620F0D7FA9E
:109140006649284620F013FB654B0A221988204601
:1091500020F040FB3C2387229B2162480397029426
:109160000195009610F0E3FB204620F0C0FA284657
:1091700020F0BDFA5C49284620F0F9FA5B4B0A2240
:109180001988204620F026FB3C238722E6215848F8
:10919000039702940195009610F0C9FB204620F039
:1091A000A6FA284617E05349204620F0E0FA524933
:1091B000284620F0DCFA00230393282300935A2248
:1091C0003C239B213E480295019410F0B0FB2846B9
:1091D00020F08DFA204620F08AFA4849484F204670
:1091E00020F0C5FA0026444928464FF0280820F010
:1091F000BEFA3C235A22E621039642480295019486
:10920000CDF8008010F093FB284620F070FA20463D
:1092100020F06DFA46F22C390A234FF0030B8DE84B
:109220000808B6224FF49B7305213748CDF8089003
:109230001CF088F83346B7222D2133481BF07AF909
:10924000FBF72EFE31493048F7F74DFB0722B721D7
:109250002520FAF727FBB721FA200722FAF722FB8D
:109260003E782B492046002E58D020F080FA29491C
:10927000284620F07CFA4FF4FC630393C7223C237A
:10928000052102950194CDF80080234810F04FFB92
:10929000284620F02CFA204620F029FA5CE000BF96
:1092A000541B03000C1D030028C4FF1F5F1B030099
:1092B000FA1C030084B9FF1F661B03009419030006
:1092C00060BAFF1F9C1803006AC5FF1F88BAFF1F02
:1092D0009C190300368DFF1F9CBAFF1F591E030007
:1092E00028D5FF1FB0BAFF1F6D1B03000CB9FF1F6D
:1092F000C4BAFF1F791B0300A6490300811B0300AA
:10930000B0C5FF1F74BAFF1F58C6FF1F881B03009C
:10931000B81B03005521030098B9FF1F20F027FA5E
:10932000BC49284620F023FA3C23C7220521BA482D
:10933000CDF80C9002950194CDF8008010F0F7FA6A
:10934000284620F0D4F9204620F0D1F931464FF4D8
:10935000E870F7F70DFA3E70B049284620F007FA9A
:10936000AF4B20461978F9F789FC00262823C7223D
:1093700050210093AB4803963C230294019510F0D2
:10938000D6FA204620F0B3F9284620F0B0F9A64AD4
:1093900051681068128912AB03C3A4491A80A44B08
:1093A00009781A78914202D2FF221A700DE0A14B7F
:1093B000A82101FB0233103312AA53F8050F596894
:1093C0001B7A03C213708DF851609B49204620F030
:1093D000CEF9002712A92826284620F0C8F93C23F8
:1093E000C7229B219548039702950194009610F09F
:1093F0009EFA284620F07BF9204620F078F9904923
:10940000204620F0B4F98F4B02221968284620F03C
:1094100034FA03970295019400963C23C722E62173
:10942000894802F070B8162840F08E82FF294FF06C
:10943000000440F04581854D2819143410F062F87D
:10944000B4F5027FF8D10A240025C02601944FF418
:109450009B73302205217E48029500961BF072FF17
:109460004CF218633022029301944FF49B73052150
:10947000774800961AF07AFD4FF6FF71744819F09C
:1094800086FD0121724819F07CFD7249704819F07F
:10949000D3FD2B464A2221466D486F4C1BF04AF8FB
:1094A0006E496B48F7F71FFA694819F0DFFD022192
:1094B000674819F0BFFC2378694AD25C5B4B1B7884
:1094C0009A424ED227262378DFF894912178227889
:1094D000584F19F80110DBB20793237819F80330BD
:1094E0004FF0A80808FB037308FB017193F814A060
:1094F00019F8023008FB0373D3E91223D1E91601EE
:1095000023F034F80022574B23F00EFBCDE908017D
:10951000284623F079F902460B46DDE9080123F0DD
:10952000D9F9079B19F8033008FB0377D7E9122311
:1095300023F01EF823F0C6FC1AAB524601211DF0A1
:1095400053FE32B200231A2141481AF0F3FF0135CD
:109550001AA93F48F7F7C7F918360B2DB6B2B2D1A2
:1095600005E02078FF2100F5F770F7F701F90321F6
:109570003748DFF80481DFF8B490DFF800A119F074
:1095800059FC46F22C31324819F001FD00236522C6
:109590000C212F481AF0CEFF33492D48F7F7A3F9D5
:1095A00000237A2210212A481AF0C4FF2F492848A4
:1095B000F7F799F900238F221E2125481AF0BAFFE8
:1095C00000212348F7F797F90023A3221021204810
:1095D0001AF0B0FF26491E48F7F785F90023B72295
:1095E0000C211B481AF0A6FF22491948F7F77BF90E
:1095F00007250024184B1A78E3B29A4208D198F84C
:10960000013099F800209A423AD98AF8003037E0C0
:10961000002737E0A71A030098B9FF1F391B030082
:10962000E08EFF1FACB9FF1FC71A03002AC4FF1F3B
:1096300008CAFF1F008FFF1FEE190300C0B9FF1FEC
:10964000F8190300B4C7FF1FD4B9FF1F20B9FF1FCB
:1096500058C6FF1F302B0300E6C6FF1FC01B0300C8
:10966000D08EFF1F00002440D21B0300D81B030034
:10967000DD1B0300E21B0300CF8EFF1FA0C5FF1FF1
:109680004FF4FC671AAE99F8003018F8011F0A224F
:10969000304610F003FE9F4A142303FB04202946A2
:1096A0008DE8C8004D223A233C3010F09BF801347D
:1096B000304620F01CF83E35052CADB29AD108E0BA
:1096C0005C2300930194F8236422272192481BF025
:1096D000E1FD672441F2A20522B215340095F12381
:1096E0002A218D48A4B21BF037FFD02CF4D12A24B4
:1096F00041F2A20521B2183400955423682286480D
:10970000A4B21BF0CBFEB4F5997FF3D1834C844E09
:109710002378844DF25C2B789A4206D3BBF10B0F71
:10972000DFF820825FD902F0B8BA22787E4F0B238F
:109730005A434FF00B08BA56642AC1BF22785343EC
:109740000022FA54237808FB03F34FF02A09FA5653
:109750006FF0530364325A43C92392FBF3F2BC32D5
:1097600092B24FF0010A237808FB037313F90A3011
:10977000642B02F38A82694B6B491B7808FB031345
:1097800013F90A306433C2F28082237808FB037332
:109790006FF0530113F90A3064334B43C92193FB33
:1097A000F1F3BC33662B03DDBC2BA8BFBC2300E068
:1097B000672399B207910FFA89F109F118091FFA85
:1097C00089F94FF478401BB20190009312B20FFA5E
:1097D00089F3514819F068FEB9F58D7F0AF1010A45
:1097E0009CD0079ABFE723784C4FF25C2B789A42C3
:1097F00082F053823B784C4C47480B2505FB0343D2
:109800000BEB4B0113F90B206FF0530364324FF451
:1098100078465A43C900C92392FBF3F2BC32009642
:10982000032312B22A311AF037FB4FF003090296D4
:10983000152632233522F92137488DE840021BF0E6
:1098400081FD4FF6FF71344819F0A1FB37493248CA
:1098500019F0F2FB4A220023FA212F481AF06AFE7F
:109860003B782D4805FB03441AAD14F90B10F7F7AC
:1098700042F8294819F0FAFB00242D4928462427EC
:109880001FF075FF182364224FF49371019521484E
:10989000029400970FF0A6FF28461FF028FF2549E5
:1098A00028461FF064FF1823CC224FF493710195D2
:1098B0002148029400970FF095FF28461FF017FFEC
:1098C0001E4928461FF053FF3C238C224FF493710E
:1098D000019500931A48029418230FF083FF28463D
:1098E0001FF005FFB8F800200B480294183A8DE8E5
:1098F00040024FF48A7312B211211BF023FD054D73
:1099000004F1C800284414340FF0FCFD642CF7D196
:1099100002F04FBB20B9FF1F58C6FF1FE6C6FF1F4E
:10992000D08EFF1F2AC4FF1FA6C6FF1F302B0300C7
:10993000A9190300AC19030034B9FF1F0D1C030063
:1099400048B9FF1F3C88FF1F182840F06283FF2999
:109950004FF0000440F08281B24D281914340FF00A
:10996000D1FDB4F5027FF8D10024AC250A2640F2DF
:109970002B1330221421AC4802948DE860001BF0B8
:10998000E1FC4CF2186330220293142140F22B13B5
:10999000A5488DE860001AF0E9FA4FF6FF71A24879
:1099A00019F0F5FA0121A04819F0EBFA9F499E48F9
:1099B00019F042FB23464A2219219B481AF0BAFDAE
:1099C0009B499948F6F78FFF9A4A9B4910780B7884
:1099D0000891984292460BD211781AA8082210F0EA
:1099E0005DFC1AA990481FF03DFD1AA81FF07FFEEC
:1099F0008D4819F03BFB02218B4819F01BFA00231C
:109A00001A22582188481AF095FD8C498648F6F7A5
:109A10006AFF27270026089A9AF800301278DFF8A4
:109A200014829A4240F2C58000233AB216217E4841
:109A3000834C1AF07FFD98F80030A82505FB0343FE
:109A40001B7D8BBB98F8001098F8003098F8002028
:109A500005FB014105FB0343D2B20792D1E9160190
:109A6000D3E9122322F082FD0022764B23F05CF82A
:109A700080463046894622F0C7FE02460B464046E5
:109A8000494622F027FF079B05FB0344D4E9122334
:109A900022F06EFD23F016FA23F04EFD6A4902B261
:109AA0001AA824F0B7F880E098F8003098F8001071
:109AB00005FB034305FB01411B7D012B98F800309A
:109AC00098F8002005FB0343D2B20792D1E91601B2
:109AD000D3E9122333D122F049FD0022594B23F060
:109AE00023F880463046894622F08EFE02460B4619
:109AF0004046494622F0EEFE079B05FB0344D4E9AD
:109B0000122322F035FD23F0DDF90021054623F074
:109B1000D5FC10B105F1004000E028464B4923F088
:109B20002FFB23F009FD0A2390FBF3F404FB13043D
:109B3000284623F001FD234602B2454932E022F0D7
:109B400015FD00223F4B22F0EFFF8046304689464C
:109B500022F05AFE02460B464046494622F0BAFE23
:109B6000079B05FB0344D4E9122322F001FD23F0F7
:109B7000A9F90021054623F0A1FC10B105F1004030
:109B800000E02846334923F0FBFA23F0D5FC642398
:109B900090FBF3F404FB1304284623F0CDFC2E497C
:109BA000234602B21AA824F035F81AA91E48F6F77F
:109BB0009AFE013618370B2EBFB27FF42CAF03216B
:109BC000194819F037F946F22C31174819F0DFF926
:109BD00000234D22172114481AF0ACFC64211248CE
:109BE000F6F789FE002362221A210F481AF0A2FC20
:109BF00050210D48F6F77FFE0023A4221A210A48BF
:109C00001AF098FC14210848F6F775FE0023BA22D2
:109C1000202105481AF08EFC00210348F6F76BFE60
:109C200025E000BF20B9FF1F58C6FF1F302B0300DF
:109C3000E81B030029C4FF1F2AC4FF1FF41B0300F5
:109C4000008FFF1F00002440EB490300000020416B
:109C5000FB1B03000000C842041C03007523009393
:109C60000194F8234D2227219A481BF013FB50241E
:109C700041F2A20522B216340095F1232A2195481B
:109C8000A4B21BF069FCD42CF4D12A2441F2A20521
:109C900021B2183400956D2351228E48A4B21BF0D6
:109CA000FDFBB4F5997FF3D18B4D2E46502716F866
:109CB000010B0097BE2364220021F6F77AFD2A24C7
:109CC0001FFA80F916F8010B0097BE2364220021C9
:109CD000F6F76FFD80B24F2803DDBE28A8BFBE2077
:109CE00000E0502021B21834A4B21FFA80FA4FF4D9
:109CF000784800B20090CDF8048023B20FFA89F2C0
:109D0000744819F0D1FBB4F58D7F01D0D146D9E765
:109D1000ABF16503DBB2992B00F2FA806F4B0BF1CC
:109D20003807FFB21B787A1E9A4216D00FB9FF2B64
:109D300013D09F4217D06A4A1278974201D1FF2B65
:109D400011D0791C8B4213D0974200D183B1013AD4
:109D5000974213D1FF2B11D10AE044F20824264682
:109D60004FF4FC690EE044F208244FF4FC6608E06E
:109D700044F208264FF4FC64B14603E044F20824A0
:109D80002646A146DFF88481B8F800201920052373
:109D90000025303A8DE8290012B2DB234F214D48CF
:109DA0001BF0D0FA4FF0030C4FF0000E94238DE817
:109DB00008503C2218234FF4937146481BF0C2FA16
:109DC000B8F800A0464B1AAD0BF137011B780822FA
:109DD000C9B22846AAF1300A10F060FA1FFA8AFACE
:109DE000CDF808904FF01A09524633234F213D48D1
:109DF0000195CDF800900FF0F5FC28461FF077FC98
:109E0000B8F800A0364BAAF1300A1B780822394670
:109E100028461FFA8AFA10F041FA33235246872166
:109E2000029631480195CDF800900FF0DBFC2846F2
:109E30001FF05DFCB8F80060294B303E0BF1390192
:109E40001B780822C9B22846B6B210F027FA33238D
:109E50003246BF21029425480195CDF800900FF0BD
:109E6000C1FC28461FF043FCB8F800402049303CB4
:109E700028461FF07CFCA4B200232246172102933F
:109E80001C4801953323CDF800900FF0ABFC284619
:109E90001FF02DFCB8F800401749303C28461FF051
:109EA00066FCA4B200232246F721029313480195D1
:109EB0003323CDF800900FF095FC28461FF017FCD7
:109EC0000F480FF01FFB0F480FF01CFB0E4800F06F
:109ED000BCBD00BF58C6FF1F84C5FF1FE88EFF1F13
:109EE0002AC4FF1F84B9FF1F98B9FF1FACB9FF1F19
:109EF0002D150300C0B9FF1F2F150300D4B9FF1F94
:109F000020B9FF1F34B9FF1F48B9FF1F3C88FF1F4E
:109F1000BBF1C70F02F24D80502315F80B000093E0
:109F20006422BE230021F6F744FC0BEB4B01C90071
:109F300002B203232A31C048CDF8008019F0ACFFEB
:109F40001521032335228DE80A00BB48CDF808808F
:109F50002A23F9211BF0F6F94FF6FF71B64819F0E4
:109F600016F8B649B44819F067F800234A22FA21D6
:109F7000B1481AF0DFFA15F80B10AF481AACF6F733
:109F8000B6FCAD4819F072F80025AD4924262046EC
:109F90001FF0EDFB18233C224FF49371A948029562
:109FA000019400960FF01EFC20461FF0A0FBA6496E
:109FB00020461FF0DCFB1823AC224FF49371A3481A
:109FC0000295019400960FF00DFC20461FF08FFBC8
:109FD0009F4920461FF0CBFB442364224FF493712A
:109FE00000939C480295182301940FF0FBFB204638
:109FF0001FF07DFB98480FF085FA98480FF082FA21
:10A0000097480FF07FFA97480FF07CFA964800F0D7
:10A010001CBD152840F08882FF294FF0000440F055
:10A020006781884D281914340FF06CFAB4F5027F5B
:10A03000F8D1AC240A25002640F22B13302214213B
:10A040007D488DE870001BF07DF94CF218633022DA
:10A050000293142140F22B1377488DE8300019F059
:10A0600085FF4FF6FF71744818F091FF0121724887
:10A0700018F087FF7149704818F0DEFF33464A2216
:10A0800019216D481AF056FA784916A81FF06FFB8F
:10A09000774B1A78032A9A4617D176496648F6F71D
:10A0A00022FC754B75491B78097832461AA810F0C6
:10A0B000F5F81AA960481FF0D5F91AA81FF017FB88
:10A0C0006F4916A81FF0D0FB03E06E495A48F6F717
:10A0D0000AFC594818F0CAFF0221574818F0AAFE96
:10A0E00000231A22532154481AF024FA16A9524880
:10A0F0001FF0B8F9272500272AB2002316214E4861
:10A10000614E1AF017FA0120F6F79FFBA82404FB12
:10A11000006000225D4BD0E9160122F005FD80466B
:10A120003846894622F070FB02460B4640464946B7
:10A1300022F0D0FB22F0A6FE013781B23E48F6F7AE
:10A14000DAFB18350B2FADB2D6D103213A4818F0FF
:10A1500071FE46F22C31384818F019FF9AF8003099
:10A16000032B4FF04D024FF0000340F09780434F18
:10A1700031481A211AF0DEF93B782F48012504FBFB
:10A1800003630095D3E91623F6F7BBFB0023622295
:10A190001A2129481AF0CEF9397804FB0161D1E976
:10A1A0001289D1E9160142464B4622F0DFF900221E
:10A1B000374B22F08FFB0022364B22F0B5FC424693
:10A1C0004B4622F0D5F9009502460B461A48F6F7A1
:10A1D00098FB0023A4221A2117481AF0ABF939780A
:10A1E00004FB0161D1E91289D1E9160142464B46CF
:10A1F00022F0BCF90022284B22F06CFB0022254BF8
:10A2000022F092FC42464B4622F0B2F900950246FB
:10A210000B460948F6F775FB0023BA221A210648B7
:10A220001AF088F93B78009504FB0364D4E9122303
:10A230000148F6F766FB57E058C6FF1F302B0300B6
:10A24000A919030020B9FF1FAC19030034B9FF1F7F
:10A250000D1C030048B9FF1F84B9FF1F98B9FF1FE9
:10A26000ACB9FF1FC0B9FF1FD4B9FF1F101C0300FA
:10A270006CC5FF1F1A1C03002AC4FF1FFE87FF1FA7
:10A28000661B0300281C0300008FFF1F00002440F2
:10A290000000544000005940000034401721964807
:10A2A0001AF048F964219448F6F725FB002362224E
:10A2B0001A2191481AF03EF950218F48F6F71BFBFE
:10A2C0000023A4221A218C481AF034F914218A4858
:10A2D000F6F711FB202188480023BA221AF02AF948
:10A2E00000218548F6F707FB16A81FF000FA08E0E2
:10A2F000752300930194F8234D2227217E481AF0FC
:10A30000C9FF502441F2A20522B216340095F12370
:10A310002A217948A4B21BF01FF9D42CF4D12A24A5
:10A3200041F2A20521B2183400956D2351227248E2
:10A33000A4B21BF0B3F8B4F5997FF3D16F4B704D15
:10A340001A7807932E46032A16F8012B6FF06C0734
:10A3500014BF4FF065094FF480797A4392FBF9F20C
:10A36000BE3292B22A2416F8013B7B4393FBF9F3E9
:10A37000BE339BB24F2B03DDBE2BA8BFBE2300E034
:10A38000502321B21834A4B21FFA83FA4FF478484C
:10A390001BB20093CDF8048023B212B2564819F0D4
:10A3A00083F8B4F58D7F01D05246DCE7BBF1FF0F97
:10A3B00001F0FF8515F80B204F48CDF800806FF0B5
:10A3C0006C030BEB4B015A43C90092FBF9F2BE320E
:10A3D000032312B22A3119F05FFD152203238DE801
:10A3E0000C00EF21342335224348CDF808801AF0C1
:10A3F000A9FF4FF6FF71404818F0C9FD41493E489A
:10A4000018F01AFE00234A22F0213B481AF092F875
:10A41000079B15F80B401B78032B29D13A4B3B4A7D
:10A420001B78A82101FB0321D1E91267D1E91601AC
:10A4300032463B4622F09AF880462046894622F072
:10A44000D3F902460B464046494622F043FA28A378
:10A45000D3E9002322F068FB32463B4622F088F81D
:10A460000223009302460B462348F6F74AFA03E01C
:10A4700021462148F6F73BFA1AAC1F4818F0F6FDC2
:10A4800000252349242620461FF071F918233C2279
:10A490004FF493711F480295019400960FF0A2F9B2
:10A4A00020461FF024F91C4920461FF060F91823AC
:10A4B000AC224FF4937119480295019400960FF065
:10A4C00091F920461FF013F9154920461FF04FF966
:10A4D00044231448009302950194182364224FF4F6
:10A4E00093710FF07FF901F0B9BB00BFAFF30080AB
:10A4F0000000000000E06F4058C6FF1F6CC5FF1F42
:10A50000C1C4FF1F302B0300FE87FF1F008FFF1FFA
:10A51000A919030020B9FF1FAC19030034B9FF1FAC
:10A520000D1C030048B9FF1F172840F0E480A04D20
:10A530000024281914340EF0E5FFB4F5027FF8D199
:10A540000026AC240A258DE8700040F22B1330223F
:10A5500014219848DFF8B4821AF0F4FE4CF2186324
:10A5600030228DE830000293142140F22B139148E1
:10A5700019F0FCFC4FF6FF718E4818F008FD012120
:10A580008C4818F0FEFC8C498A4818F055FD33467B
:10A590004A221921874819F0CDFF88498548F6F7E6
:10A5A000A2F9844818F062FD3346BE221921814881
:10A5B00019F0C0FF82497F48F6F795F93346CB2260
:10A5C00019217C481AAC19F0B5FF7E49794816ADBF
:10A5D000F6F789F97C4920461FF0C9F8282798F832
:10A5E000001028461FF0E3F83C234D221921704843
:10A5F00003960295019400970FF099F928461FF0F1
:10A6000076F820461FF073F8704920461FF0AFF827
:10A6100098F8011028461FF0CAF83C234D22692102
:10A620006B4803960295019400970FF080F9284635
:10A630001FF05DF820461FF05AF8664920461FF0CB
:10A6400096F898F8021028461FF0B1F83C234D22E6
:10A65000B921614803960295019400970FF067F9BC
:10A6600028461FF044F820461FF041F85B49204679
:10A670001FF07DF898F8031028461FF098F83C2347
:10A680007F221921564803960295019400970FF0F6
:10A690004EF928461FF02BF820461FF028F85149A4
:10A6A00020461FF064F898F8041028461FF07FF841
:10A6B0003C237F2269214C48039602950194009720
:10A6C0000FF035F928461FF012F820461FF00FF85A
:10A6D000464920461FF04BF898F8051028461FF011
:10A6E00066F803960295019400973C237F22B921D6
:10A6F0003F4800F008BF0E2840F0EE820026FF29F8
:10A700003C4FDFF80C9101961AAD40F0A2813B88D6
:10A7100028480D3B1BB20D223146009323B21AF09C
:10A72000B9FD4FF6FF71234818F031FC0121214893
:10A7300018F027FC20491F4818F07EFC33462422DD
:10A7400005211C4819F0F6FE2B491A48F6F7CBF8FC
:10A7500016AC184818F08AFC284920461FF007F864
:10A76000254928461FF003F828232D22502103965F
:10A770000093234802953C2301940FF0D8F8284613
:10A780001EF0B5FF20461EF0B2FF40F2AB10F6F708
:10A790005CF81C4B1C4E187019781A46002901F001
:10A7A00075833378022B41F0C18301F06FBB00BF8A
:10A7B00020B9FF1F58C6FF1F302B03003B1C0300AE
:10A7C0004C1C0300791C0300941C03009A1C03001A
:10A7D00034B9FF1FA01C030048B9FF1FA61C0300CB
:10A7E0005CB9FF1FAC1C030070B9FF1FB21C030053
:10A7F00084B9FF1F3C88FF1F8D190300791B0300DC
:10A80000E8B9FF1FF18EFF1FABC7FF1F20D5FF1F49
:10A810002AC4FF1F1F78FFB2052F41F0A283A84969
:10A8200028461EF0A4FF4FF4FC63029328230093F4
:10A8300001953C232D223946A2480EF0D3FF28462D
:10A840001EF055FF4FF0000828279F4928461EF0AC
:10A850008EFF3C235F2205219C48CDF8088001959E
:10A8600000970EF0BFFF28461EF041FF984928468A
:10A870001EF07DFF3C235F2250219648CDF80880D2
:10A88000019500970EF0AEFF28461EF030FF92496A
:10A8900028461EF06CFF3C23912205218F48CDF8FD
:10A8A0000880019500970EF09DFF28461EF01FFFBF
:10A8B0008B4928461EF05BFF3C235021912289489A
:10A8C000CDF80880019500970EF08CFF28461EF009
:10A8D0000EFF337884497D4E022B204641F0F182F1
:10A8E0001EF045FF814928461EF041FF4CF21863D7
:10A8F000C3220521039306F1F0003C230295019445
:10A9000000970FF014F828461EF0F1FE20461EF0C6
:10A91000EEFE774B1B78002B41F0E982754920460B
:10A920001EF025FF744928461EF021FF4CF21863E3
:10A9300003932823C3225021019400936F4802956A
:10A940003C230EF0F4FF28461EF0D1FE20466C4C4E
:10A950001EF0CDFE99F800302178092228460FF02C
:10A960009DFC05237A22009323212B4665480FF096
:10A97000FBFF28461EF0BBFE227899F800309A4271
:10A9800019D2F28BB18B60481B32193112B20023FD
:10A9900009B219F0CFFD5D4B186821F047FF22780E
:10A9A0005B4BA82707FB023302461B7D00935648EA
:10A9B0000B46F5F7A6FF99F8003061780922284682
:10A9C0000FF06CFC0523AC22009323212B464D484D
:10A9D0000FF0CAFF28461EF08AFE627899F8003010
:10A9E0009A421CD2B6F84620B6F8441046481B32AC
:10A9F000193112B2002309B219F09CFD434B58687B
:10AA000021F014FF3E4B5A78414BA82404FB02333B
:10AA100002461B7D00933C480B46F5F772FF64200D
:10AA2000FAF7E2FB3B4B3C4801221A700EF06AFD3C
:10AA30003A480EF067FD3A480EF064FD39480EF0D2
:10AA400061FD39480EF05EFD38480EF05BFD01F007
:10AA5000B0BA28230093C3229A2305212A481AF06A
:10AA600019FC334B1A78334B1B78511E994215D081
:10AA70000AB9FF2B12D09A4216D099F800108A42D8
:10AA800001D1FF2B10D0501C834212D08A4200D13A
:10AA90007BB1884250D1FF2B4ED10AE044F208240A
:10AAA00026464FF4FC684BE044F208244FF4FC6661
:10AAB00045E044F208264FF4FC64B04640E000BF95
:10AAC000CE1C030070B9FF1FEC1C030020B9FF1F50
:10AAD000F51C030034B9FF1FFD1C030048B9FF1F1C
:10AAE000071D03005CB9FF1F541B0300492203002C
:10AAF00002B9FF1F101D0300181D030024BAFF1F19
:10AB00002488FF1FB8BCFF1F58C6FF1F98C5FF1F32
:10AB1000008FFF1F3A88FF1F84B9FF1F98B9FF1FDE
:10AB2000ACB9FF1FC0B9FF1FD4B9FF1FFCB9FF1F8D
:10AB3000A0C5FF1FE88EFF1F44F208242646A0464A
:10AB4000B7F800A08D492846AAF11A0A1EF00FFE98
:10AB50001FFA8AFACDF808804FF01A0852463323BC
:10AB600037210195CDF800808548DFF85CA20EF012
:10AB700039FE28461EF0BBFD3A888248113A002370
:10AB800012B2392119F0D6FC9AF8001099F8003069
:10AB9000013908222846C9B20FF080FB29467948BE
:10ABA0001EF060FC28461EF0A2FDB7F800B0734905
:10ABB000ABF11A0B1FFA8BFB28461EF0D8FD5A4644
:10ABC0000296332370210195CDF800806E480EF077
:10ABD00009FE28461EF08BFD3A886A48113A002388
:10ABE00012B2732119F0A6FC99F800309AF80010FF
:10ABF000082228460FF052FB294662481EF032FC1C
:10AC000028461EF074FD3E885C491A3EB6B22846BE
:10AC10001EF0ADFD324602943323A9210195CDF8F3
:10AC200000805A480EF0DEFD28461EF060FD3A888E
:10AC30005448113A002312B2AC2119F07BFC9AF867
:10AC4000001099F80030013108222846C9B20FF0EF
:10AC500025FB29464B481EF005FC28461EF047FD03
:10AC60003C884B491A3C0026A4B228461EF07FFDC2
:10AC700022463323314602960195CDF8008045489F
:10AC80000EF0B0FD28461EF032FD3C8842491A3CC9
:10AC9000A4B228461EF06BFD22463323E221029621
:10ACA0000195CDF800803D480EF09CFD28461EF031
:10ACB0001EFD3C883A491A3CA4B228461EF057FDB6
:10ACC00002960195CDF80080272322464FF48C711F
:10ACD00034480EF087FD1BE1102840F0EF81FD297C
:10ACE00040F21981FF2926D100252F4B01951B88A1
:10ACF00024480D3B1BB20D220093294623B21AF0C3
:10AD0000C9FA4FF6FF711F4818F041F901211D489B
:10AD100018F037F925491B4818F08EF92B462422E4
:10AD20000521184819F006FC21491648F5F7DBFD06
:10AD3000144818F09BF940F21B10F5F786FD1AAC89
:10AD40000A2843D8DFE800F0060D0F1142424242C4
:10AD500042421300174920461EF009FD46F22C33EB
:10AD60003AE0154904E0154902E0154900E01549AB
:10AD700020461EF0FCFC4FF4FC632DE0CF1A0300CC
:10AD800084B9FF1F58C6FF1F98B9FF1FACB9FF1F3A
:10AD90002D150300C0B9FF1F2F150300D4B9FF1FE5
:10ADA00016180300FCB9FF1F3C88FF1F302B03005F
:10ADB0005D1903000C1D0300661903006B190300E5
:10ADC0007119030085190300A0C5FF1FA44920467F
:10ADD0001EF0CDFC4FF6E073029328232D220521AF
:10ADE0000093A04801943C2316AD0EF0FBFC2046D6
:10ADF0001EF07DFC9C4928461EF0B9FC0027282641
:10AE00009A4920461EF0B3FC3C235F220521984856
:10AE100003970294019500960EF089FD20461EF0DE
:10AE200066FC28461EF063FC924928461EF09FFCF3
:10AE3000914920461EF09BFC3C23912205218F481E
:10AE400003970294019500960EF071FD20461EF0C6
:10AE50004EFC28461EF04BFC894928461EF087FC14
:10AE6000854920461EF083FC05213C23C3228548EA
:10AE700003970294019500960EF059FD20461EF0AE
:10AE800036FC28461EF033FC4FF4D770F5F7DDFC96
:10AE90007D4948B928461EF06AFC7C4920461EF0D0
:10AEA00066FC46F22C3308E028461EF060FC774929
:10AEB00020461EF05CFC4FF4FC63C3226421039324
:10AEC000734802943C23019500960EF030FD204615
:10AED0001EF00DFC28461EF00AFC6E4928461EF0A6
:10AEE00046FC4FF48A70F5F7B0FC014620461EF090
:10AEF0005EFC002303932823009367480294019586
:10AF00003C23C3229B210EF012FD20461EF0EFFBD6
:10AF1000284600F0A4BE002944D1604B0A4643F8FD
:10AF20002B200BF1010BBBF1080F4FF00004F6D101
:10AF3000C823272250215A4800930194DC231AF099
:10AF4000A9F9F9F7ADFF234628228C21544819F0BE
:10AF5000F1FA54495248F5F7C6FC234632228C21B7
:10AF60004F4819F0E7FA50494D48F5F7BCFC3E4907
:10AF700016A81EF0FCFB3D491AA81EF0F8FB1F2383
:10AF80001AAA16A93A480EF089FB1AA81EF0AFFBC0
:10AF900016A81EF0ACFB454B14221A70444B1C70D3
:10AFA00001F007B801292DD100233C4A194642F887
:10AFB00023100133082B4FF00004F8D1C8232722B7
:10AFC0005021374800930194DC231AF063F9F9F714
:10AFD00067FF284916A81EF0CAFB27491AA81EF0C9
:10AFE000C6FB23461AAA16A924480EF057FB1AA836
:10AFF0001EF07DFB16A81EF07AFB284B02221A6178
:10B0000000F0D7BF022940F0D487244B24481961AF
:10B010000024C823272250218DE81800DC231AF0D1
:10B0200039F9F9F73DFF164916A81EF0A0FB1249A1
:10B030001AA81EF09CFB23461AAA16A911480EF066
:10B040002DFB1AA81EF053FB16A81EF050FB194B3F
:10B050001B681A93184B1A9A1A6000F0AABF00BF17
:10B060002F16030020B9FF1F1D1D0300221D030022
:10B0700034B9FF1F2C1D0300311D030048B9FF1F09
:10B08000351D03005CB9FF1F661903003B1D03005B
:10B0900070B9FF1F411D030084B9FF1F18C6FF1FB1
:10B0A00058C6FF1F491D0300611D0300E6C6FF1FB0
:10B0B0000188FF1F4CD8FF1FE48EFF1F112840F0AE
:10B0C00043824FF00008B54BCDF804801B88B4488C
:10B0D0000D3B1BB20D220093414623B21AF0DAF861
:10B0E0004FF6FF71AE4817F052FF0121AC4817F040
:10B0F00048FFAC49AA4817F09FFF43462422052188
:10B10000A74819F017FAA849A548F5F7ECFB16ADC2
:10B11000A34817F0ABFFA54928461EF028FB4FF4C3
:10B120008E70F5F792FB1AAC0146282720461EF0D8
:10B130003EFB50213C233A469D48CDF80C800294BA
:10B14000019500970EF0F3FB20461EF0D0FA28463A
:10B150001EF0CDFA4FF4D670F5F777FB12AE01284A
:10B160009449304620D11EF002FB934928461EF038
:10B17000FEFA924920461EF0FAFA4FF4FC633A4672
:10B180009B21049303943C230295019600978C48DD
:10B190000EF068FB20461EF0AAFA28461EF0A7FA19
:10B1A00030461EF0A4FA24E01EF0E1FA8249284657
:10B1B0001EF0DDFA814920461EF0D9FA46F22C3302
:10B1C0009B213A4604937E4803943C2302950196C2
:10B1D00000970EF047FB20461EF089FA28461EF025
:10B1E00086FA30461EF083FA41464FF4D670F5F7E2
:10B1F000BFFA40F2AD10F5F728FB724928B120469E
:10B200001EF0B5FA4FF4FC6304E020461EF0AFFADE
:10B2100046F22C3328220092052102936A480194B9
:10B220003C230EF0DFFA20461EF061FA6749204603
:10B230001EF09DFA664B282719784CF218682846AC
:10B240001EF0B5FA3C233A46EB216248CDF80C805B
:10B250000295019400970EF06AFB28461EF047FA0B
:10B2600020461EF044FA5C4920461EF080FA4FF456
:10B27000D270F5F7EAFA014628461EF098FA3C2308
:10B280005F2205215548CDF80C8002950194009766
:10B290000EF04DFB28461EF02AFA20461EF027FA33
:10B2A0004F4920461EF063FA002350215F2202938B
:10B2B0004C4801943C2300970EF094FA20461EF06F
:10B2C00016FA40F2AF10F5F7C0FA4749C8B9304650
:10B2D0001EF04DFA454928461EF049FA44492046D9
:10B2E0001EF045FA46F22C3304934248039402952B
:10B2F000019600973C235F229B210EF0B3FA204673
:10B300002EE030461EF033FA384928461EF02FFA58
:10B3100040F2AF10F5F799FA01460AA81EF047FA75
:10B320000AA90EA81EF08DFA33490EA81EF03AFBAA
:10B33000014620461EF085FA4FF4FC635F229B21F4
:10B3400004932C4803943C230295019600970EF039
:10B3500089FA20461EF0CBF90EA81EF0C8F90AA8FB
:10B360001EF0C5F928461EF0C2F930461EF0BFF99E
:10B3700040F21D10F5F769FA01282049304643D103
:10B380001EF0F5F91E4928461EF0F1F91D49204628
:10B390001EF0EDF94FF4FC6342E000BF3C88FF1F54
:10B3A00058C6FF1F302B03007A1D0300891D0300C0
:10B3B00034B9FF1F21190300921D03000B1903006C
:10B3C0005CB9FF1F9B1D030084B9FF1FA31D030071
:10B3D000FF87FF1F70B9FF1FAB1D030098B9FF1F48
:10B3E000B41D0300ACB9FF1FBA1D0300C11D03004B
:10B3F0000C1D0300C0B9FF1F671A0300C81D03001E
:10B40000CD1D0300FA1C03001EF0B1F94149284686
:10B410001EF0ADF9404920461EF0A9F946F22C3342
:10B42000049328235F22EB2100933C4803943C23A0
:10B43000029501960EF016FA20461EF058F928469D
:10B440001EF055F930461EF052F9354B354F1B783A
:10B45000F3B9354928461EF08AF9344920461EF0D2
:10B4600086F939880A2230461EF0B4F946F22C33A8
:10B470000493282300930396029401953C2396227B
:10B4800005212B480EF0EEF930461EF030F91FE092
:10B490003B882549284643B11EF069F925492046D5
:10B4A0001EF065F94FF4784307E01EF060F9224979
:10B4B00020461EF05CF94FF4FC63039328230093AD
:10B4C000029401953C239622052119480EF02FFA8B
:10B4D00020461EF00CF928461EF009F917492046AF
:10B4E0001EF045F9164B19780A22013128461EF044
:10B4F00071F90023039313480295282300930194C4
:10B500003C23962250210EF012FA28461EF0EFF846
:10B51000A4E300BFCD1D03000C1D0300D4B9FF1F21
:10B520006CC5FF1FC88EFF1F94190300D21D0300B6
:10B53000E8B9FF1FD81D0300DF1D0300E81D03004D
:10B54000E1C7FF1FFCB9FF1F122840F0328500271A
:10B55000B54B01971B88B5480D3B1BB20D223946F0
:10B56000009323B219F096FE4FF6FF71AF4817F023
:10B570000EFD0121AD4817F004FDAD49AB4817F0B1
:10B580005BFD3B4624220521A84818F0D3FFA949BA
:10B59000A648F5F7A8F9A54817F068FD4FF4D9704B
:10B5A000F5F78FF916AD82B2A34912A81AAC22F0B2
:10B5B00031FBA249284628261EF0D9F812A92046B8
:10B5C0001EF0D5F83C232D22052103979C480294B8
:10B5D000019500960EF0ABF920461EF088F828463B
:10B5E0001EF085F84FF4DA70F5F76BF9924982B2E4
:10B5F00012A822F00FFB934928461EF0B8F812A9B2
:10B6000020461EF0B4F83C232D22502103978E488B
:10B610000294019500960EF08AF920461EF067F814
:10B6200028461EF064F84FF4DB70F5F74AF98249BA
:10B6300082B212A822F0EEFA844928461EF097F84A
:10B6400012A920461EF093F83C232D229B2103973C
:10B650007F480294019500960EF069F920461EF08D
:10B6600046F828461EF043F84FF4DC70F5F729F948
:10B67000714982B212A822F0CDFA764928461EF00E
:10B6800076F812A920461EF072F83C232D22E621FE
:10B69000039771480294019500960EF048F92046F0
:10B6A0001EF025F828461EF022F84FF4DD70F5F75D
:10B6B00008F9614982B212A822F0ACFA674928461B
:10B6C0001EF055F812A920461EF051F83C235F22C7
:10B6D0000521039762480294019500960EF027F920
:10B6E00020461EF004F828461EF001F84FF4DE70E4
:10B6F000F5F7E7F8504982B212A822F08BFA5949BF
:10B7000028461EF034F812A920461EF030F83C23DB
:10B710005F225021039754480294019500960EF041
:10B7200006F920461DF0E3FF28461DF0E0FF4FF428
:10B73000DF70F5F7C6F8404982B212A822F06AFA23
:10B740004A4928461EF013F812A920461EF00FF8A9
:10B750003C235F229B210397454802940195009664
:10B760000EF0E5F820461DF0C2FF28461DF0BFFF91
:10B770004FF4E070F5F7A5F82F4982B212A822F035
:10B7800049FA3C4928461DF0F2FF12A920461DF057
:10B79000EEFF3C235F22E621039737480294019590
:10B7A00000960EF0C4F820461DF0A1FF28461DF0BB
:10B7B0009EFF4FF4D870F5F784F8B8424FF4D87074
:10B7C000C8BF4FF4FC67F5F77CF81B4982B212A89A
:10B7D00022F020FA294928461DF0C9FF12A9204667
:10B7E0001DF0C5FF05213C239122254803970294B3
:10B7F000019500960EF09BF820461DF078FF284634
:10B800001DF075FF4FF4E270F5F71FF801281D4990
:10B8100028463BD11DF0ABFF1B4920461DF0A7FF7A
:10B820004FF4FC633AE000BF3C88FF1F58C6FF1F7F
:10B83000302B0300F01D0300FB1D0300021E03005C
:10B8400020B9FF1F0A1E030034B9FF1F121E030098
:10B8500048B9FF1F1A1E03005CB9FF1F221E030018
:10B8600070B9FF1F2A1E030084B9FF1F321E030098
:10B8700098B9FF1F3A1E0300ACB9FF1F421E030018
:10B88000C0B9FF1F471E0300552103001DF06FFFC5
:10B89000684920461DF06BFF46F22C33912250215F
:10B8A000039300963C230294019563480EF03FF801
:10B8B00020461DF01CFF28461DF019FF5F49284651
:10B8C0001DF055FF002628275D4920461DF04FFF3B
:10B8D0003C23BE2205210396029401950097594806
:10B8E0000EF025F820461DF002FF28461DF0FFFE51
:10B8F000554920461DF03BFF3C23BE2250210296B5
:10B900000194009751480DF06DFF20461DF0EFFEA9
:10B910004F4920461DF02BFF3C23BE229B2102965F
:10B92000019400974B480DF05DFF20461DF0DFFEAF
:10B93000494928461DF01BFF484920461DF017FFC6
:10B940003C23BE22E62103960294019500974448C9
:10B950000DF0EDFF20461DF0CAFE28461DF0C7FE83
:10B960004CF218613F4817F012FB3346E7220A21D8
:10B970003C4818F0DFFD3C493A48F4F7B4FF18E3BF
:10B980002B78052B07D1394B002019780EF05EFC7F
:10B99000002840F056812B78062B04D02B78072BFB
:10B9A00040F0518108E0314B012019780EF04EFC37
:10B9B000002840F04681F1E72C4B032019780EF067
:10B9C00045FC002840F03D813DE11A780A2A59D112
:10B9D000274920461DF0CBFE002221461D480DF0D0
:10B9E00027FE20461DF083FE224920461DF0BFFEA3
:10B9F00046F22C3302931A23494601940093832282
:10BA0000642317480DF0EEFE20461DF070FE1A4A22
:10BA100000231370194A1370194B14201C681EF070
:10BA20007EF80546F4F7F0FF2946204616F00CFB99
:10BA3000BFE200BFA71A0300FCB9FF1F501E03009E
:10BA4000571E030010BAFF1F5B1E030024BAFF1F1E
:10BA5000611E0300D4B9FF1F351D03006C1E0300D7
:10BA6000E8B9FF1F58C6FF1F701E0300A0C5FF1FC7
:10BA7000161A0300AB150300D0C5FF1FC8C5FF1F72
:10BA800098D7FF1F1E78F6B2082E40F0D4808F4D55
:10BA90008F49B5F80080DFF87CB2DFF88492A8F116
:10BAA0001A0820461DF063FE1A271FFA88F844F290
:10BAB00008234246192102938648019433230097B4
:10BAC0000DF090FE20461DF012FE2A888248DFF815
:10BAD0005482113A002312B21B2118F02BFD9BF85F
:10BAE00000304FF0A80A0AFB0393324693F89110F6
:10BAF00098F800300139C9B220460EF0CFFB21463C
:10BB000075481DF0AFFC20461DF0F1FD2A887049F4
:10BB10001A3A92B2204607921DF029FE4FF4FC63B8
:10BB2000079A0293522133236C48019400970DF039
:10BB300059FE20461DF0DBFD2A886748113A002394
:10BB400012B2552118F0F6FC9BF8001098F800305E
:10BB50000AFB0191324691F8911020460EF09EFBAF
:10BB600021465D481DF07EFC20461DF0C0FD2A8860
:10BB700057491A3A92B2204607921DF0F8FD44F256
:10BB80000823079A02938B21332355480194009789
:10BB90000DF028FE20461DF0AAFD2A884E48113AD5
:10BBA000002312B28E2118F0C5FC9BF800300AFB6E
:10BBB0000399324699F8911098F800300131C9B2D2
:10BBC00020460EF06BFB214643481DF04BFC2046FF
:10BBD0001DF08DFD2E8843491A3E4FF00008B6B285
:10BBE00020461DF0C4FD3246132341463E48CDF8A1
:10BBF0000880019400970DF0F5FD20461DF077FDBB
:10BC00003A4B2D881E883A497D3E1A3DB6B2ADB2F8
:10BC100020461DF0ACFD13232A4631463548CDF8A9
:10BC20000880019400970DF0DDFD20461DF05FFDBA
:10BC30003148FCF76EB81A783AB11B78022B11D153
:10BC400003E02E4902E02E4900E02E4920461DF077
:10BC50008EFD0022214628480DF0EAFC20461DF00A
:10BC600046FDA6E1284920461DF081FD002221461F
:10BC700021480DF0DDFC20461DF039FD2348F4F786
:10BC80006DFE234B01221A7093E1237808FB0373A6
:10BC9000002103F80A10FDF778BD1E4B93F80090C1
:10BCA0002378F35C09F1FF329A4208D0B9F1000F12
:10BCB0003AD1194B194A1B78D35CFF2B34D144F28B
:10BCC000082427464FF4FC6A48E000BF3C88FF1F69
:10BCD000CF1A030098B9FF1F58C6FF1F5CB9FF1F9A
:10BCE000ACB9FF1F2D15030070B9FF1F0488FF1F9B
:10BCF0002F15030084B9FF1FD4B9FF1F611E030075
:10BD00009D1E0300AE1D03000F1A0300E8B9FF1FBC
:10BD1000D0C5FF1FA0C5FF1FE6C6FF1FD08EFF1FA7
:10BD2000008FFF1F2AC4FF1F2378F35C4B4500F0F0
:10BD300097802A78914500F08C802178715C09F118
:10BD400001038B4200F09C80914500F08E8093426D
:10BD500000F0918044F208242746A246B8F800B0CB
:10BD60002B781AAE09F1FF3130460822C9B2ABF187
:10BD7000180B0EF093FA1FFA8BFBCDF808A04FF0CA
:10BD8000150A5A4633234A210196CDF800A08A4865
:10BD90000DF028FD30461DF0AAFCB8F800B02B7855
:10BDA000ABF1180B494630461FFA8BFB08220EF008
:10BDB00075FA5A460297332382210196CDF800A0E6
:10BDC0007E480DF00FFD30461DF091FCB8F8007074
:10BDD0002B7809F10101183F3046BFB20822C9B2E1
:10BDE0000EF05CFA3A4633230294BA210196CDF85C
:10BDF00000A073480DF0F6FC30461DF078FCB8F852
:10BE000000407049183C0025A4B230461DF0AFFC3C
:10BE100022463323112102950196CDF800A06A48ED
:10BE20000DF0E0FC30461DF062FCB8F800406749B8
:10BE3000183CA4B230461DF09AFC02950196CDF84C
:10BE400000A033232246F22161480DF0CBFCFCF721
:10BE500026BD604B60491B78CB5CFF2B7FF46DAF38
:10BE600044F208244FF4FC6777E75A495A480978A6
:10BE7000415C29B16BE72378F35CFF2B7FF46AAF59
:10BE800044F208274FF4FC64BA4667E7534920465A
:10BE90001DF06DFC524928461DF069FC4CF21863F8
:10BEA0000393282300932D223C2305214D4802951E
:10BEB00001940DF03CFD28461DF019FC2046FEF7CC
:10BEC000BFBC032B09D11DF052FC474928461DF089
:10BED0004EFC40F2FF73FEF70BBD1DF048FC4349DA
:10BEE00028461DF044FC4FF4FC63FEF701BD022B15
:10BEF0000BD13F4920461DF03AFC3E4928461DF033
:10BF000036FC4FF6E073FEF713BD01214FF4D570F8
:10BF1000F4F72EFC384920461DF029FC3349284609
:10BF20001DF025FC4FF4FC63FEF702BD1278334B85
:10BF3000012A06D1324928461DF019FC4FF6E0735C
:10BF40002EE01A78022A01D12E491DE01A78032A20
:10BF500001D12D4918E01A78042A7EF45BAC2B49F4
:10BF600012E01A78062A01D129490DE01A78072A29
:10BF700001D1284908E01A78082A01D1264903E0AE
:10BF80001B78092B06D1254928461DF0F0FB4FF4FC
:10BF9000FC6305E0224928461DF0E9FB4FF4784395
:10BFA00002932823009301953C232D220521FEF7BF
:10BFB00043BC1FB0BDE8F08FE8B9FF1FFCB9FF1FFD
:10BFC00010BAFF1F2D15030024BAFF1F2F15030001
:10BFD00038BAFF1FE6C6FF1FD08EFF1F0C1D0300DF
:10BFE000D51B030070B9FF1F131603003522030091
:10BFF000181D030055210300101D0300F18EFF1FC3
:10C00000B81C0300BD1C0300C21C0300C91C0300B4
:10C01000D21C0300D61C0300DA1C0300DE1C030044
:10C02000E61C03002DE9F04F8BB004ABB84E83E85B
:10C0300003003778BDF91040BDF91250AFB90DF1CA
:10C040001808B44940461DF092FB23220F230093A9
:10C0500011468223B0480297CDF804800DF0C2FB50
:10C0600040461DF044FBAD4B1F700021AC4816F05C
:10C070008EFF0121AA4816F084FF3178A84801EB11
:10C080004101490000232722323118F053FAA54B11
:10C090001F7899462FB17B1C89F800304FF00108BA
:10C0A00001E04FF00A08A4B2ADB201232A462146AE
:10C0B0009D480DF02FFA38B33378DFF854B2062BD1
:10C0C00022D8DFF8B4A29949DAF8000021F0F6F995
:10C0D000D0B197499248F4F706FC404620F0FCFFA7
:10C0E000DAF8001021F04CF8CAF80000384620F0C9
:10C0F0007BFB02460B4600208E491DF0F3FE0246F4
:10C100000B4600208C490AE201232A4621468B482F
:10C110000DF000FA40B33378DFF8F4B1062B23D8E2
:10C12000DFF854A28149DAF8000021F0C7F9D8B14C
:10C1300083497B48F4F7D7FB404620F0CDFFDAF87F
:10C14000001021F01DF8CAF80000384620F04CFB22
:10C1500002460B46002077491DF0C4FE02460B46FE
:10C1600000204FF08041DAE101232A46214675483C
:10C170000DF0D0F938B33378DFF894B1062B22D81C
:10C18000DFF8F4A16949DAF8000021F097F9D0B19D
:10C190006D496348F4F7A7FB404620F09DFFDAF8AD
:10C1A000001020F0EDFFCAF80000384620F01CFB1C
:10C1B00002460B4600205F491DF094FE02460B46E6
:10C1C00000206249ABE101232A46214660480DF078
:10C1D000A1F938B33378DFF838B1062B22D8DFF86D
:10C1E00098A15249DAF8000021F068F9D0B1594914
:10C1F0004B48F4F778FB404620F06EFFDAF8001069
:10C2000020F0BEFFCAF80000384620F0EDFA0246E2
:10C210000B46002047491DF065FE02460B460020F4
:10C220004D497CE101232A4621464C480DF072F924
:10C2300038B33378DFF8D8B0062B22D8DFF838A12E
:10C240003A49DAF8000021F039F9D0B144493448CC
:10C25000F4F749FB404620F03FFFDAF8001020F0E9
:10C260008FFFCAF80000384620F0BEFA02460B469F
:10C27000002030491DF036FE02460B4600203949A9
:10C280004DE101232A46214637480DF043F968B1B4
:10C290003378DFF87CB0062B08D8DFF8DCA0234920
:10C2A000DAF8000021F00AF9002867D101232A46B4
:10C2B00021462E480DF02EF900287AD03378DFF889
:10C2C00050B0062B75D8DFF8B0A01849DAF8000096
:10C2D00021F0F4F800286CD025491148F4F703FB4D
:10C2E000404620F0F9FEDAF8001020F049FFCAF8C5
:10C2F0000000384620F078FA02460B4600200D492F
:10C300001DF0F0FD02460B4600201A4907E100BF70
:10C310000088FF1FAB1503005CB9FF1FE18EFF1FF4
:10C3200058C6FF1F0188FF1FE8B9FF1F003C1C46CD
:10C33000F21A0300000024400000F03FFCB9FF1F88
:10C34000A817030010BAFF1FFA1A030000000840E4
:10C3500024BAFF1FFE1A03000000104038BAFF1F66
:10C36000E51E0300000014404CBAFF1F60BAFF1F17
:10C370008319030000001C40CCC5FF1FB949BA480F
:10C38000F4F7B1FA404620F0A7FEDAF8001020F0EA
:10C39000F7FECAF80000384620F026FA02460B469F
:10C3A0000020B2491DF09EFD02460B460020B04918
:10C3B000B5E001232A462146AE480DF0ABF838B36C
:10C3C0003378DFF8FCB2062B22D8DFF8D8A2AA49CE
:10C3D000DAF8000021F072F8D0B1A849A248F4F7C9
:10C3E00082FA404620F078FEDAF8001020F0C8FE0D
:10C3F000CAF80000384620F0F7F902460B46002044
:10C400009A491DF06FFD02460B4600209C4986E0CC
:10C4100001232A4621469B480DF07CF838B3337837
:10C42000DFF89CB2062B22D8DFF878A29249DAF81E
:10C43000000021F043F8D0B193498B48F4F753FA48
:10C44000404620F049FEDAF8001020F099FECAF8C4
:10C450000000384620F0C8F902460B460020834908
:10C460001DF040FD02460B460020884957E001239D
:10C470002A46214686480DF04DF878B199F80030EB
:10C48000844C43B984497848F4F72DFA3378013362
:10C490003370012300E0013B237063E37F480123F5
:10C4A0002A46214600F5C8700DF034F860B13378A3
:10C4B000DFF80CB2062B07D8DFF8E8A16E49DAF8EE
:10C4C000000020F0FBFF80B901232A462146744872
:10C4D0000DF020F800283AD0724B0021186820F0A7
:10C4E000E3FF074600283FD031E06F495E48F4F78C
:10C4F000FAF9404620F0F0FDDAF8001020F040FE96
:10C50000CAF80000384620F06FF902460B460020BA
:10C5100056491DF0E7FC02460B460020002120F0A2
:10C5200003FB0446DAF800000D4620F07FF90B46C5
:10C5300002462946204620F01BF820F0C3FC9BF859
:10C540000030CAF8000001338BF800300AE3012301
:10C550002A46214655480CF0DDFF002841D0544FB3
:10C560003B780C2B4CD93CE0524C237883F00103F0
:10C5700023702722034628213B4817F0DBFF25784C
:10C5800006AC4DB14C493848F4F7ADF94A4920465C
:10C590001DF0EDF802970FE008224CF218638DE8C9
:10C5A0000C002821052327222F4818F073FE42494A
:10C5B00020461DF0DCF802951923009391222823D0
:10C5C0007D21374801940DF00DF920461DF08FF8BC
:10C5D00099F80030002B00F0C5822E4A013B137001
:10C5E000C0E201232A46214630480CF093FFA8B14F
:10C5F0002F4B1A780D2A0FD01A780E2A0ED10BE085
:10C6000000210520FAF718F839780620FAF714F80F
:10C610002A4B06221A70A5E20E2070E001232A465A
:10C62000214622480CF076FF40B1214B1A780E2AA1
:10C6300004D91A78112A01D8142060E001232A466F
:10C6400021461A480CF066FF00283BD0184B1A7898
:10C65000122A37D1194A1420107000221A70FF21B3
:10C6600052E000BFB61C030058C6FF1F0000244064
:10C670000000184074BAFF1F003C1C461817030046
:10C680000000204088BAFF1F9417030000002240DA
:10C690009CBAFF1F0188FF1FAA17030020B9FF1FC4
:10C6A000C4BAFF1FCCC5FF1F6F19030084B9FF1F59
:10C6B000E6C6FF1FE18EFF1FAC170300FD87FF1FBB
:10C6C0000088FF1F01232A46214697480CF022FFCD
:10C6D00030B1964B1A78122A02D91A78182A0DD935
:10C6E00001232A46214690480CF014FF78B18F4B65
:10C6F0001A781C2A0BD91A781E2A08D811208C4ABD
:10C700001070FF221A701978F9F796FF2AE20123B8
:10C710002A46214687480CF0FDFE08B133787BB9E4
:10C72000002327225921844817F004FF4FF4784151
:10C73000814816F02CFC81497F48F4F7D4F811E2C7
:10C740007F4B1B7823B17F4A136803F100431360CA
:10C75000764C2378012B14D17B4B7C4A1B78A8257F
:10C7600005FB0325774B186820F060F8C5E9120136
:10C7700000210520F9F760FF6D4B06221A70002595
:10C78000C5E02378032B0CD16F4B704A1B78A8258A
:10C7900005FB03256B4B186820F048F8C5E9160126
:10C7A000E6E723780B2B0CD1674B684A1B78A8254A
:10C7B00005FB0325634B186820F038F8C5E9200114
:10C7C000D6E723780C2B0CD15F4B604A1B78A82549
:10C7D00005FB03255B4B186820F028F8C5E922010A
:10C7E000C6E72378092B0CD1574B584A1B78A8254C
:10C7F00005FB0325534B186820F018F8C5E92601FE
:10C80000B6E723780D2B08D14E4B51491B680B60BE
:10C810001520F3F7EEFF0E2260E02578EDB20E2D25
:10C820000CD1484B4A491B6841F8043F1A20F3F7E2
:10C83000E0FF3F4B1D70FF232370A0E723780F2BF1
:10C8400022D1404D43492E68304620F055FE20B994
:10C850000021304620F028FE08B13E4B2B602868AE
:10C860003D4E20F08FFE30803C481CF09DFD33880B
:10C870003B493A484FF47A7292FBF3F2F4F75AF8D4
:10C88000317840F2CD1026E02378102B10D12D4DB9
:10C890003449286820F030FE08B1324B2B602868FC
:10C8A00020F070FE304BC1B2197040F2CB1012E094
:10C8B0002378112B15D1234D2A4E2868314620F0BC
:10C8C0001BFE00B12E60286820F05CFE274BC1B231
:10C8D00019704FF4E670F3F74BFF1422144B1A70E3
:10C8E000A9E72378114D122B09D1164B20491B685B
:10C8F0000B6040F2D310F3F77CFF14222DE12B786C
:10C90000122B39D92B78182B40F2168134E0194BB1
:10C91000581914350CF0F6FDB5F5DC7FF7D1044B52
:10C9200021781878F0E600BF84B9FF1FE6C6FF1F24
:10C93000FD87FF1F70B9FF1F58C6FF1FE61C0300CD
:10C94000E18EFF1FCCC5FF1FA0C5FF1F008FFF1F7B
:10C9500098C5FF1F00007F43EEC4FF1FD8C7FF1F0D
:10C96000F90500000000C84200B9FF1FEAC9FF1F17
:10C97000B4C7FF1F20B9FF1F23787C4D192B1DD191
:10C980007B4D7C4E2868314620F0B6FD00B12E600C
:10C990002868794D20F0F6FD81B2298040F22710F9
:10C9A000C9B2F3F7E5FE754B297814221A70FF23FC
:10C9B0002370734A734B12781B783EE02B781A2B46
:10C9C0001BD16B4D6B4E2868314620F095FD00B1B0
:10C9D0002E6028686A4D20F0D5FD81B229804FF481
:10C9E0009470C9B2F3F7C4FE644B14221A70FF238B
:10C9F0002370644B2A781B781DE02B781B2B21D1E8
:10CA00005B4D5C4E2868314620F076FD00B12E600B
:10CA100028685C4D20F0B6FD81B2298040F22910D3
:10CA2000C9B2F3F7A5FE554B14221A70544AFF23DE
:10CA3000237012782B785049097853480190534855
:10CA4000009023E02B781C2B24D1494D494E2868B7
:10CA5000314620F051FD00B12E6028684B4D20F08A
:10CA600091FD81B229804FF49570C9B2F3F780FE31
:10CA7000424B41494448097814221A70FF2323701D
:10CA80003F4A404B12781B7801900095404819F0BE
:10CA900009FB74E62B781D2B0AD1354B186820F062
:10CAA00071FD3C4B1A8880B2904213D100200EE0F9
:10CAB0002B781E2B16D12E4B37491D68284620F0A7
:10CAC000FDFC38B1284620F05DFD324B80B2188065
:10CAD000F3F798FE294B11221A70304AFF23237076
:10CAE00013704CE62B781F2B7FF449AE204B2B4F55
:10CAF0001868DFF8888020F045FD264B1A8880B240
:10CB000090424FF000060ED130461E80F3F77AFEB9
:10CB1000234B1E70142388F80030224B1E70FF2315
:10CB20002B703B702BE6032388F800302E70FF2318
:10CB30003B7029783046E7E50D4B2E78186820F0D9
:10CB400021FD194BC1B2F6B228781E4400F587705A
:10CB500006F8131CF3F70CFE1722084B1A70FF237C
:10CB60002B700CE60BB0BDE8F08F00BFE6C6FF1FD0
:10CB7000CCC5FF1F00007F436AC5FF1FFD87FF1F55
:10CB8000368DFF1F28D5FF1F0F88FF1F0CB9FF1F11
:10CB9000D4C5FF1FC88EFF1F00401C460188FF1F21
:10CBA000A0C5FF1FE88EFF1F20D5FF1F2DE9F74FFF
:10CBB0000120F3F74AFE344EA82303FB006600224F
:10CBC000324BD6E916011FF0AFFFD6E90E890246B7
:10CBD0000B4604460D46404649461FF0A5FF20F08F
:10CBE00051F95FFA80F8B8F1090FDFF8A49045D841
:10CBF000D6E90E2329462046CDE9002320F042F94C
:10CC00001FFA80FB0BFB08FA50461FF0FDFD06469D
:10CC100019F808000F461FF0E7FDC84404460D460A
:10CC200098F801001FF0E0FD22462B461FF09EFC05
:10CC30003246804689463B46DDE900011FF096FCFE
:10CC400002460B46404649461FF044FE80460BEB29
:10CC50000A0089461FF0D8FD32463B461FF086FC8D
:10CC600002460B46404649461FF05EFF22462B46D1
:10CC70001FF07EFC20F006F9C0B201E099F80A002E
:10CC800003B0BDE8F08F00BF008FFF1F00002440FD
:10CC9000C1C4FF1F37B500244FF4D8708DF8004091
:10CCA0008DF801400194F3F70CFE00283CD0234995
:10CCB0002348F3F718FE4FF4E270F3F7C6FD01289E
:10CCC000054609D01F491E48F3F70DFE21464FF4D3
:10CCD000E270F3F74DFD25461B491948F3F703FEB3
:10CCE000002404F1D900400080B28DF80150F3F720
:10CCF000E8FDE2B201906946144815F0A5FA013446
:10CD0000019A13490E481CF0E4FB082CE9D14FF4BA
:10CD1000D8708DF80050F3F7D4FD0E49019002460B
:10CD200007481CF0D6FB03E00B490548F3F739FC34
:10CD30006946064815F04CFA03B030BDA61E030044
:10CD4000848AFF1FB21E0300B71E03003CC5FF1FED
:10CD5000C11E0300C71E0300D31E03002DE9F04FC0
:10CD60005D4B5E4A1B7889B04FF00B0B06935C4B12
:10CD70001B780BFB03234FF0000A00250793594B48
:10CD80001AF80340069B9C4280F08280564BA822F2
:10CD900002FB0434D4E916010022544B1FF0C4FEF8
:10CDA000D4E90E8902460B4606460F4640464946E0
:10CDB0001FF0BAFE20F066F85FFA80F8B8F1090FAC
:10CDC0005CD83946304620F07DF8D4E90E3406466A
:10CDD0004046CDE9023420F07FF9314620F0D0F909
:10CDE0001FF024FD3D4B0BFB0A34CDE9000114F983
:10CDF00008001FF009FD08F1010780463846894602
:10CE000020F06AF9314620F0BBF91FF00FFDDDE993
:10CE100000231FF0ABFB00220023E457CDE90401FF
:10CE20001FF0C0FF00BB20461FF0EEFC42464B4601
:10CE30001FF09CFBDDE9002306460F46DDE90201F9
:10CE40001FF094FB02460B46304639461FF042FD68
:10CE5000DDE904231FF068FE02460B4640464946C2
:10CE60001FF086FB8046894628461FF0DFFC4246BD
:10CE70004B461FF07DFB20F025F808E0079B93F957
:10CE80000A0020F029F90146284620F071F80546ED
:10CE90000AF1010ABAF1050F7FF471AF144B28466D
:10CEA0001C7820F049FB00B210F1640F03DB64280A
:10CEB000A8BF642001E06FF063001FF0A5FC0A4BDF
:10CEC000A82202FB0433C3E90E01D3E90E011FF0CF
:10CED000F9FF09B0BDE8F08F2AC4FF1FA6C6FF1FE7
:10CEE000E88EFF1FD08EFF1F008FFF1F0000244021
:10CEF0000288FF1FFFFFFFFF2DE9F04F9A4B9B4C6D
:10CF00001A7889B0032A059360D126887822B3B2B3
:10CF100093FBF2F602FB1636002E57D1944D954B3B
:10CF20002B6008236B71944BDFF87C921B78022BEB
:10CF30000CBF022300234FF001082B7240466423EC
:10CF40006B7285F80480F3F780FCA82707FB00903C
:10CF5000D0E90E011FF096FFC0F30720A8724046EB
:10CF6000F3F773FC07FB0090D0E90E011FF08AFF76
:10CF70002E73E8726E73AE73EE73009695E80F0031
:10CF8000F3F74CFD7D4A13784344DBB213701378FA
:10CF900003F0FF020BB97A4B1A702A6879497A4874
:10CFA0007A4E1CF096FA06F1080716F8012F784918
:10CFB00075481CF08EFAB742F7D1764B6A791B6838
:10CFC0000793079B744970481CF083FA734B1B78D6
:10CFD000032B40F08380724B1B78FE2B7ED1714E69
:10CFE000714D3178A82707FB0151D1E90E010022CC
:10CFF00000231FF0FFFE002870D0FFF7AFFE82462F
:10D00000FFF7D4FD367807FB0651D1E91289834634
:10D0100042464B46D1E916011FF0A8FACDE90201BC
:10D0200058461FF0E1FB02460B46DDE902011FF006
:10D0300051FC4BA3D3E900231FF076FD42464B463B
:10D040001FF096FA594B00221FF044FC1FF01AFF04
:10D0500080B220F041F856498046504620F044F90D
:10D0600001464FF07E501FF081FF0146404620F000
:10D0700087F820F087FA4F4B80B218804E4B93F818
:10D0800000804E4B1B7843450AD920F021F84849CF
:10D0900020F02AF91FF0CAFB07FB0857C7E90E0169
:10D0A000A82707FB0655414B0022D5E90E011FF0CA
:10D0B00011FC1FF0BFFE424B1860424818F0A6FF5B
:10D0C00060B1414B1D78414B1888414B18801FF0CF
:10D0D0008BFB354B07FB0535C5E90E01059B1B781E
:10D0E000012B07D1238828219BB293FBF1F201FB8E
:10D0F000123333B340F21910F3F7A7FB092826D1F6
:10D1000023884FF4FA619BB293FBF1F201FB1233D7
:10D11000D3B12388C8219BB293FBF1F201FB1233F8
:10D1200093B1238801339BB22380238842F6E061C8
:10D130009BB293FBF1F201FB12335BB90B4A1380F4
:10D1400008E0F4F77DF8D5E7F3F7AEFCE9E700284F
:10D15000E7D0DEE709B0BDE8F08F00BFAFF3008095
:10D160000000000000E06F40ABC7FF1FF28EFF1F02
:10D1700074C5FF1F00D1CC1CF18EFF1F30C5FF1FEF
:10D18000E28EFF1FDC140300848AFF1F7BC5FF1F94
:10D19000E21403004CD8FF1FE81403006CC5FF1F06
:10D1A0000FB9FF1FFE87FF1F008FFF1F00005940B0
:10D1B0000000C842E8C9FF1F0A88FF1F2AC4FF1FDA
:10D1C000E4C9FF1FD4C5FF1F0988FF1F6EC5FF1FDD
:10D1D000C6C5FF1FFFFFFFFF2DE9F04186B019F024
:10D1E00093FED34AD3480023FF2151825372138206
:10D1F00013751946C21819500833B3F5007F117121
:10D20000CC4AF7D1CC4B402100261A601971334625
:10D21000935191190836B6F5007F4FF000040B7159
:10D22000F6D140F29F10F3F710FB1FF0DDFA024633
:10D230000B4600204FF080411CF054FEBAA3D3E906
:10D2400000231FF047FB1FF01DFE23460146224628
:10D250000094BA4814F028FFB948BA4ABA490460A1
:10D26000802505711FF06AF9B848B64AB6490571BC
:10D2700004601FF063F9B648B24AB349057104600F
:10D280001FF05CF940F2C710F3F7DFFAB14B1870EA
:10D290004FF4E470F3F7D9FAAF4B187040F2C510B1
:10D2A000F3F7D3FAAD4B1870AD4813F0E1FAA54A85
:10D2B000AC49AB481FF042F9AB4813F0D9FAA14A88
:10D2C000A849A9481FF03AF9A84818F0C1FF9D4A9B
:10D2D000A749A6481FF032F940F29910F3F7B5FAC2
:10D2E000D22302460821A34819F06BFB954AA249B4
:10D2F000A0481FF023F94FF4C870F3F7A6FA0546CB
:10D3000040F29110F3F7A1FA0B210D220C238DE8C6
:10D310000E0002462946FF239848994D15F0D2FC8D
:10D32000984815F06FF840F2A910F3F78EFA964B73
:10D33000187040F27710F3F788FA944B18704FF496
:10D34000CD70F3F782FA287040F29B10F3F77DFA64
:10D3500068704FF4CE70F3F778FAA87040F29D1021
:10D36000F3F773FAE87040F2C310F3F76EFA28711E
:10D3700040F2A510F3F769FA854B864D187040F21C
:10D38000A710F3F762FA844B187040F21710F3F706
:10D390005CFA824B187040F21510F3F756FA804B86
:10D3A00018700720F3F751FA7E4B18704FF4907005
:10D3B000F3F74BFA287040F21F10F3F746FA687043
:10D3C00040F2CB10F3F741FA774B784D18704FF4D9
:10D3D000E670F3F73AFA764B187040F2C910F3F79B
:10D3E00034FA744B187040F2CD10F3F72EFA724BEA
:10D3F00018804FF4E770F3F728FA704B187040F27A
:10D40000CF10F3F722FA6E4B001B18BF01201870E3
:10D410004FF4E870F3F719FA6A4B187040F2D11024
:10D42000F3F713FA684B18704FF4E970F3F70DFA3D
:10D43000664B187040F2D710F3F707FA28704FF4D4
:10D44000EC70F3F702FA687040F2D910F3F7FDF9C7
:10D45000A8704FF4ED70F3F7F8F9E87040F2DB10C4
:10D46000F3F7F3F928714FF4EE70F3F7EEF9687102
:10D4700040F2DD10F3F7E9F9A8714FF4EF70F3F71C
:10D48000E4F9E87140F2DF10F3F7DFF928724FF4A6
:10D49000F070F3F7DAF9687240F2E110F3F7D5F9BA
:10D4A000A8724FF4F170F3F7D0F9494B494D187059
:10D4B0004FF4F770F3F7C9F9287040F2EF10F3F763
:10D4C000C4F968704FF4F870F3F7BFF9A87040F230
:10D4D000F110F3F7BAF9E8704FF4F970F3F7B5F912
:10D4E00028714FF49570F3F7B0F93B4D288040F266
:10D4F0002710F3F7AAF9394B074618804FF49470B8
:10D50000F3F7A3F9364B8046188040F22910F3F761
:10D510009CF9344B344A1880344B354904900193BC
:10D52000009567E0AFF30080000000008084FE40BB
:10D5300054C4FF1FE4C7FF1FECC9FF1F3CC5FF1FFA
:10D54000BCC7FF1FF887FF1FC1060000D8C7FF1F19
:10D55000388EFF1F01B9FF1FDD8EFF1FDE8EFF1FFC
:10D5600048C5FF1F8D080200F8C4FF1F388DFF1F3C
:10D570004161020018C5FF1F8D67020058C6FF1FDA
:10D58000ACC7FF1FA2C5FF1F2BC4FF1FF08EFF1FDC
:10D5900031C5FF1FB9C7FF1F70C5FF1F348DFF1FA7
:10D5A000ECC4FF1FA4C6FF1F00B9FF1FC1C4FF1FAB
:10D5B000EAC9FF1F0EB9FF1FEEC4FF1F6CC5FF1F96
:10D5C00028C4FF1FB0C5FF1FE08EFF1F08CAFF1F42
:10D5D0000FB9FF1FD08EFF1F0CB9FF1F6AC5FF1FB9
:10D5E000368DFF1F28D5FF1F6EC5FF1F0F88FF1F39
:10D5F000E4C9FF1F5F4B0594CDF80C8002975E488D
:10D600005E4D18F075FD40F22110F3F71EF92870F9
:10D610004FF49170F3F719F9687040F22310F3F7A3
:10D6200014F9A8704FF49270F3F70FF9E87040F214
:10D630002510F3F70AF928714FF49370F3F705F901
:10D64000687140F25F10F3F700F94D4D28704FF408
:10D65000B070F3F7FAF8687040F26110F3F7F5F87C
:10D66000A8704FF4B170F3F7F0F8E87040F263106F
:10D67000F3F7EBF828714FF4B270F3F7E6F868713E
:10D6800040F2FB10F3F7E1F83E4B3F4D18703F4876
:10D6900014F0BBFE4FF48A70F3F7D7F83C4B1870C8
:10D6A00040F2A110F3F7D1F83A4B18704FF48B7099
:10D6B000F3F7CBF8384B187040F2AB10F3F7C5F81E
:10D6C000364B18704FF4D570F3F7BFF8344B187021
:10D6D0004FF4FE70F3F7B9F8287040F2FD10F3F73D
:10D6E000B4F868704FF4FF70F3F7AFF8A87040F229
:10D6F000FF10F3F7AAF8E8703046F3F7A6F82871A0
:10D7000040F20120F3F7A1F8687140F20220F3F72C
:10D710009CF8A87140F20320F3F797F8E8714FF4F2
:10D720000170F3F792F8287240F20520F3F78DF8B4
:10D73000687240F20620F3F788F8A87240F20720DA
:10D74000F3F783F8174B1870174B2246E252143444
:10D75000B4F5027FFAD1154B002203F5EE6123F8F0
:10D76000662C23F8022C70338B42F8D106B0BDE84A
:10D77000F08100BFE8C9FF1FD4C5FF1F20D5FF1FE0
:10D78000F48EFF1FE4C6FF1F84C5FF1FD0C7FF1F15
:10D79000A5C6FF1F68C5FF1FABC7FF1FF18EFF1F88
:10D7A00002B9FF1F29C4FF1F20B9FF1F28BDFF1F9B
:10D7B0002DE9F041074688B08846002408EB0403B1
:10D7C00004AA03F1100E164618685968154603C5D9
:10D7D000083373452A46F7D132466946094818F09E
:10D7E00019FF6D463A192B4603CBB34210605160C6
:10D7F0001D4602F10802F6D11034C02CDED108B06B
:10D80000BDE8F081388DFF1F2DE9F04FCDB0064601
:10D81000B4491CA81BF0ABFF1CA930461CF03BF917
:10D8200004461CA81BF063FF74BB08230A22AE4900
:10D830001CA8F2F757FE1CA930461CF00DF81CA8D6
:10D840001BF055FF062231461CA81CF047F9A749DA
:10D8500014A81BF08CFF14A91CA81CF01CF904468A
:10D8600014A81BF044FF1CA81BF041FF64B9062359
:10D87000224631461CA81CF011F91CA930461BF0A9
:10D88000EBFF1CA81BF033FF99491CA81BF06FFF8E
:10D8900031461CA81CF07EF896491CF083F801461E
:10D8A00004A81BF0CEFF1CA81BF021FF049C92498A
:10D8B00014A80123224613F06DF914A813F029F8D7
:10D8C000002867D114A813F018F822468B498C4819
:10D8D0001BF0FFFD86491CA81BF049FF31461CA820
:10D8E0001CF058F887491CF05DF8014604A81BF0AD
:10D8F000A1FF1CA81BF0FBFE224601237E49049DCC
:10D900001CA813F047F91CA914A8F3F76FFE1CA874
:10D9100012F0BCFF14A812F0FCFF0446002839D115
:10D920002A46794D794976481BF0D3FD2A887848F4
:10D930000A3A234612B20A2116F0FCFD754B2A88DA
:10D940001B8873480B214FF6E075693B0B3A1BB2FD
:10D9500012B28DE82200214617F09CFC4FF478416A
:10D960006B4815F014FB6C491CA81BF000FF3146F6
:10D970001CA81CF00FF8014665481BF073FD1CA89D
:10D980001BF0B5FE14A812F0B8FF4FF4FA6019F0BE
:10D99000D9FFBEE14FF48C70F2F757FFFF284FF02C
:10D9A000000405D121464FF48C70F2F7E1FEB0E19E
:10D9B0005A4B5B4A1C705B4B5B4D1C70FF23137012
:10D9C00053709370D3701371584A2B701370584A68
:10D9D0006B701370574A1370574A1370574A13707D
:10D9E000574A1370574A1370574A14A8137012F00D
:10D9F00090FF039570B1DFF85CB1DFF854A12746C2
:10DA0000A0462546A14614A812F064FF80B1002F5D
:10DA100032D076E14D491CA81BF0A9FE1CAA0A21B0
:10DA20003148F2F789FD1CA81BF061FE052742E191
:10DA3000B8F10A0F14D9002F40F06781444B1B78CE
:10DA4000012B12D021461CA8F4F76AFB81450CD0AB
:10DA5000404B1B682DB203EBC50243F8350014712F
:10DA600014A812F04AFF1FB125E114A812F045FFD7
:10DA7000002C00F01F81ACE014A812F0B4FEC0B27C
:10DA80000D2807D19AF80020012A03D0B8F1320FEF
:10DA9000B9D90A204CAB03EB08020A2802F8C00CE3
:10DAA0005AD19AF80020012A00F08280402C00F21E
:10DAB0008880B8F10A0F40F2858021461CA8F4F74F
:10DAC0002FFB484509D0DBF800302AB203EBC20136
:10DAD000013543F83200EDB20C710134E4B28146F5
:10DAE00070E000BFE31E030038C5FF1FCF1A03001C
:10DAF000AC150300B71503002CD5FF1FE71E03006C
:10DB0000848AFF1FB21503003C88FF1F051F030016
:10DB100058C6FF1F0488FF1F141F0300AAC7FF1F5A
:10DB200006B9FF1FBBC7FF1F3788FF1F4188FF1FB4
:10DB30003E88FF1F0388FF1F0788FF1F0988FF1FFC
:10DB40000288FF1F0A88FF1F4088FF1F291F03004C
:10DB5000A4C6FF1FECC9FF1FB8F1BF0F2BD19AF865
:10DB60000020012A30D11CA96F48FFF721FEC022F6
:10DB70006D491CA818F098FF402C03D902274FF0DC
:10DB8000BF0840E721461CA8F4F7CAFA814509D02E
:10DB9000DBF800302AB203EBC201013543F8320052
:10DBA000EDB20C710134E4B281464FF0FF080BE096
:10DBB000B8F1BF0FD7D0B8F1C00F34BF002703278B
:10DBC00002E002274FF0000808F101035FFA83F832
:10DBD00019E7039B1B78FF2B07D0544AA82101FBB0
:10DBE00003239A7A0AB902229A72039B5A78FF2A6F
:10DBF00007D04E4BA82101FB02339A7A0AB90222C0
:10DC00009A7230461BF071FF014608A81BF019FEFE
:10DC100047490CA81BF0ABFD0CA930461BF03BFF9D
:10DC20000022034608A910A81BF038FF10A908A875
:10DC30001BF012FE10A81BF05AFD0CA81BF057FD9C
:10DC40000A9B062B03D83B4908A8F2F74AFE082393
:10DC50000A22394910A8F2F745FC10A908A81BF0C0
:10DC60001AFF054610A81BF042FDBDB133493448E8
:10DC7000F2F739FE08A932481BF0F4FB08A910A8F6
:10DC80001BF0DFFD0A2110AA2B48F2F755FC10A863
:10DC90001BF02DFD2B492A48F2F783FC2A4B1978FB
:10DCA00001B101214FF48C70F2F762FD08A81BF05E
:10DCB0001EFD2EE00427254C254822880A3A002321
:10DCC00012B20A2116F036FC224B22881B880B2048
:10DCD0004FF6E071693B0B3A8DE803001BB212B2BC
:10DCE00000211B4817F0D6FA4FF47841184815F078
:10DCF0004EF93B463246184915481BF0EAFB002412
:10DD000007E0B8F10A0F7FF6ABAE14A812F0F5FDEC
:10DD1000D1E714A812F0BAFD04A81BF0E8FC2046D5
:10DD20004DB0BDE8F08F00BFE7C6FF1F008FFF1F9B
:10DD3000311F0300CF1A030038C5FF1F351F030032
:10DD4000848AFF1F421F030005B9FF1F3C88FF1F85
:10DD500058C6FF1F0488FF1F4B1F0300034B1B788F
:10DD60000BB1FFF751BD1846704700BF27D5FF1F05
:10DD70002DE9F04F02218FB040F29F10F2F7F8FC2E
:10DD80000820F2F762FDFF2808D0012119F064FC99
:10DD90000820F2F75AFD002119F030FC8D4C8E4D11
:10DDA00021788E48F2F707FC29788C48F2F703FCBB
:10DDB00069788A48F2F7FFFB4FF4CD70F2F745FD22
:10DDC000002119F049FC40F29B10F2F73EFD0021C2
:10DDD00019F042FC4FF4CE70F2F737FD002119F034
:10DDE0003BFC40F29D10F2F730FD002119F034FCAD
:10DDF0004FF4C870F2F729FD012119F02DFC4FF402
:10DE0000C870F2F722FD012119F0F8FB4FF4CB7036
:10DE1000F2F71BFD012119F01FFC4FF4CB70F2F754
:10DE200014FD012119F0EAFB4FF4CA70F2F70DFD61
:10DE3000012119F011FC4FF4CA70F2F706FD01211F
:10DE400019F0DCFB4FF4D770F2F7FFFC012804D97E
:10DE500000214FF4D770F2F78BFC2078062808D900
:10DE6000002140F21710F2F783FC5A4B00221A707F
:10DE700006E0042804D905380221C0B219F0ECFBF1
:10DE8000574C2078062807D9002140F21510F2F7E8
:10DE90006FFC0023237006E0042804D90538022112
:10DEA000C0B219F0D9FB4F4C2378322B06D91E2172
:10DEB00040F2A510F2F75CFC1E2323704A4E0025A9
:10DEC0004FF4CA780127B1464FF0650A08FB05F305
:10DED0000124F7500AFB05FB4FF48E70F2F7B5FCF6
:10DEE000844206D20BEB0403013449F82370E4B2F8
:10DEF000F2E70135072DE9D11420F2F7A6FC3B4CDF
:10DF00003B4E20701920F2F7A0FC3A4960701520B2
:10DF1000F2F78DFC38491A20F2F789FC374940F2B4
:10DF2000D310F2F784FC002404F5167504F263277D
:10DF30002846F2F78AFCA5F516730135AF42F05476
:10DF4000F6D10B34372CEFD140F2C310F2F77DFC41
:10DF5000FF2802D0002119F07FFB4FF4E370F2F7A5
:10DF600074FC012119F078FB4FF4E570F2F76DFCB9
:10DF700004464FF4E3702CB9F2F767FC214619F020
:10DF80003DFB09E0F2F761FC012119F037FB0121AB
:10DF90004FF4E570F2F7ECFB194C1A4922780F4860
:10DFA0001BF097FA2278A046B2B3174B1978642970
:10DFB0001D462BD94FF4FE74002740F20726204659
:10DFC0000021F2F7D5FBA4F5FE730134B442EF54FF
:10DFD000F5D121E0348DFF1FB9C7FF1F848AFF1FD1
:10DFE000ECC4FF1F31C5FF1F0CCAFF1F2488FF1F91
:10DFF000A6C6FF1F98C5FF1F9CC5FF1FB4C7FF1F04
:10E00000ABC7FF1F6B1F030084C5FF1F032A03D983
:10E01000AB49AC48F2F7C5FAAB48AC4CDFF82493F7
:10E0200018F0C4FB40F27710F2F70FFCA84B187001
:10E03000F3F75CFD082140F2A9102170F2F798FB7C
:10E040002178A14818F0C3FB4FF4B370F2F7FDFB41
:10E05000A04B187040F26510F2F7F7FB9E4B064696
:10E06000187040F2671440F26F172046F2F7EDFB8C
:10E0700009EB44056FF43372AB18A5F2CE25187086
:10E0800004F10800F2F7E1FB0134BC422870ECD146
:10E0900031468D4818F0E2FC0220F5F793FB002191
:10E0A0000246894818F0A3FC874818F0D3FB0820E3
:10E0B000F2F7CBFBFF2802D0012119F09FFA874C21
:10E0C000874E642019F03EFC0021864816F0FAFACB
:10E0D000FF2320783370F3F79FFA2278824979483A
:10E0E000824C1BF0F6F97F4814F0C0FF40F2071095
:10E0F000F2F7ABFB7E4B18704FF48370F2F7A5FB81
:10E100007C4B003018BF012018704FF4BC70F2F740
:10E110009CFB0128207002D0C31E012B02D80023D3
:10E1200023700CE002280AD14FF4D070F2F78DFB77
:10E13000714B092888BF0022187088BF1A70227896
:10E140006E4960481BF0C5F94FF4D370F2F77DFBC0
:10E150006B4902465B481BF0BCF94FF4CB70F2F7F9
:10E1600074FB6849024657481BF0B3F940F2971018
:10E17000F2F76BFB6449024652481BF0AAF92022D1
:10E180006249634817F0F6FF03244FF4CB70F2F7AF
:10E190005CFB01465F4812F05BFC18B15E4B01224C
:10E1A0001A700AE0642019F0CDFB013C5B49454838
:10E1B000F2F7F7F914F0FF04E7D1574B03931A78FD
:10E1C000002A65D140F29510F2F73FFB012119F0CA
:10E1D00043FA4FF4D370F2F738FB012840F2951060
:10E1E00005D0F2F732FB012119F008FA0CE0F2F742
:10E1F0002CFB4B4919F08CF940F29510F2F725FBF6
:10E20000484B197819F0AAFA474C36484FF4784130
:10E2100014F0BDFE0121334814F0B3FE22883148CA
:10E22000093A002312B2012116F084F922883F4BEB
:10E230002C48B3F900304FF6E0710A240A3A12B2C2
:10E2400001910094002117F025F839492548F2F78B
:10E250004AFB37491B48F2F7A4F90321214814F07F
:10E2600090FE0023142221461E4816F063F94FF653
:10E27000FF711C4814F08BFE2E491A48F2F733FB4D
:10E280004FF4FA6019F05EFB00232B4C15485BE05D
:10E290002A490C48F2F785F940F2AF10F2F7D5FAA7
:10E2A0000028F1D026491B4812F0B8FC0028EBD01A
:10E2B000002300931A4619462148F7F7A5FCE3E727
:10E2C0007E1F0300848AFF1F18C5FF1F2BC4FF1F7A
:10E2D000F08EFF1F3988FF1FFC87FF1F2688FF1F56
:10E2E000FD87FF1F58C6FF1F911F030004B9FF1FC2
:10E2F000FF87FF1F3B88FF1F3F88FF1FA11F0300F1
:10E30000B11F0300C11F0300D11F0300D53003005C
:10E31000388DFF1F2CD5FF1F27D5FF1FE11F0300DE
:10E32000001BB74870C5FF1F3C88FF1F0488FF1FF4
:10E33000EA1F0300FC1F0300B8BCFF1F0E200300F0
:10E340001C2003002788FF1FE2187033B3F5EE6F1F
:10E35000D060B949F8D1B9480023C2181433B3F5D5
:10E36000027F5160F9D10020F2F76FFAB44BB54C3F
:10E370001870B54BB54F01301870F6F791FD228833
:10E38000B7F90030AC4800250A210A3A8DE822008E
:10E3900012B2294616F07EFF2288A7480A3A2B4679
:10E3A00012B2052116F0C6F8A949A348F2F79BFA64
:10E3B00040F29510F2F749FA012119F04DF94FF4A6
:10E3C000D370F2F742FA012807D040F29510F2F725
:10E3D0003CFA012119F012F914E0FF2540F29510E2
:10E3E000F2F733FA294619F0B9F9012019F0AAFA1F
:10E3F000013DF3D140F29510F2F727FA954B1978C9
:10E4000019F0ACF92288B7F900308B4800250A21B1
:10E410000A3A8DE8220012B2294616F03BFF228804
:10E4200085480A3A2B4612B2052116F083F88A492C
:10E430008148F2F758FA0121884814F0AFF8F3F751
:10E44000C1F8874A13680593864B0599196092466F
:10E450009946DAF800300693069BD9F800209B1AFB
:10E46000632B3BD8142019F06DFA4FF4CC70F2F7FF
:10E47000ECF919F0E3F805460028EAD1228801906A
:10E480004FF00A090A3A0146642312B26A48CDF8ED
:10E49000009016F0FFFE228867480A3A2B4612B217
:10E4A000052116F047F870496348F2F71CFA6E49E7
:10E4B0006E48F2F776F86E490AA81BF058F90AAAD6
:10E4C00049466C48F2F738F80AA81BF010F94FF4E7
:10E4D0007A7019F037FA4FF0010A01E04FF0000AA4
:10E4E000F5F774FF0546F8B1228853480B21002543
:10E4F0000B3A8DE82200642312B216F0CBFE22887C
:10E500004D480A3A2B4612B2052116F013F84FF483
:10E510007841494814F03BFD57494748F2F7E3F981
:10E520000A2019F00FFAFBE754495048F2F739F87E
:10E530002288B7F90030404801954FF00B090B3A9B
:10E54000CDF8009012B2294616F0A4FE22883A486F
:10E550000A3A12B22B46052115F0ECFF484936481D
:10E56000F2F7C1F947490AA81BF001F90AA8FFF719
:10E57000F5FB454B18700AA81BF0B9F8F6F790FCAC
:10E580002288B7F900302C48CDF800900B3A12B22F
:10E590002946019516F07EFE22882748DFF89890DC
:10E5A0000A3A2B4612B2052115F0C4FF374922481A
:10E5B000F2F799F936492048F2F795F92288398817
:10E5C0001D480A3A43392B4612B209B215F0B2FF80
:10E5D00030491948F2F787F998F8003083B1194BA0
:10E5E0001A881A4B198849080A3A0F3909B248465D
:10E5F0002B4612B215F09EFF27494846F2F773F9F1
:10E6000026491A48F2F76FF9254A1378042B144665
:10E6100006D124491548F2F766F94FF4164107E090
:10E62000052B45D120491148F2F75DF94FF4E1314E
:10E630001E481AF001FE63E058C6FF1F20B9FF1FF5
:10E64000E1C7FF1F3C88FF1F0688FF1F0488FF1FCC
:10E650002520030070C5FF1F39200300A2C5FF1F3E
:10E660004CD8FF1FD88EFF1F47200300848AFF1F4E
:10E67000291F030038C5FF1F592003001618030087
:10E6800078200300E31E03002AC4FF1F8920030033
:10E690008833030092200300A0200300A72003007A
:10E6A00005B9FF1FB9200300BF2003005C8AFF1FCC
:10E6B000062B01D1B149B6E7072B05D1B049B148C6
:10E6C000F2F711F9B049B3E7092B0DD1AF49AD48C5
:10E6D000F2F709F9AE4819F09DF9062019F002FA8F
:10E6E000AC4B00229A720BE033B1AB49A548F2F76C
:10E6F000FAF84FF496419BE7A849A248F2F7F3F8DD
:10E700002178A048DFF82083A54FF1F754FF40F2AD
:10E710001B10F2F79AF8A34902469A481AF0D9FE5C
:10E720000024E3B2A346013422469F499548029350
:10E730001AF0CFFE4FF4CD70F2F787F818F8015FAA
:10E74000854217D040F29B10F2F77FF8854211D036
:10E750004FF4CE70F2F779F885420BD040F29D105D
:10E76000F2F773F8854205D0012D03D9093D012D3B
:10E7700000F23F828D4B39781B788B4240F2398210
:10E780008048F2F7B4F8022198F8000018F064FF0E
:10E79000874B002243F82B20029B012B854B05D091
:10E7A0001878854922284FF0030204E058788349FD
:10E7B00022284FF0030228BFFF2018F07FFF98F8AF
:10E7C00000207F496F481AF084FE3A787D4BA821DB
:10E7D00001FB0233002283F89020022C07F101078D
:10E7E0009FD1794D2A78531E072B2F4626D877497B
:10E7F00064481AF06EFE2B785A1E032A05D8744816
:10E800000344002113F8010C0AE0581FC0B201288C
:10E8100009D8002118F020FF287805382146C0B219
:10E8200018F01AFF11E0DA1F012A07D8981CC0B2AD
:10E83000002118F011FF28780230EFE7FF2140F2A5
:10E84000FB10F1F793FF00233B70624D62494D4886
:10E85000F2F749F82B7803F0FD02012A66D15F4BED
:10E860001A78642A05D9322140F2CB101970F1F7D9
:10E870007FFF5B4B1A78642A05D964214FF4E67058
:10E880001970F1F775FF574F3B88042B03DDFF2B01
:10E89000A8BFFF2300E005234FF4FA723B80524CDF
:10E8A00092FBF3F3514A137022780A2A04D840F2FB
:10E8B0008363D340DB0705D4002140F2C9102170E7
:10E8C000F1F756FF0121207818F0C6FE484B374A71
:10E8D0001B7892F80080434502D2464A137006E046
:10E8E0000520F1F7B2FF804584BF424B18702B78AA
:10E8F000042B0CD140492348F1F7F5FF20783F491C
:10E9000018F006FE0021207818F028FF08E03B8868
:10E910003B493C484FF47A7292FBF3F2F2F70AF863
:10E920002278394917481AF0D4FD0FE00BB937495E
:10E9300002E0022B04D136491248F1F732FE05E01D
:10E9400034491048F1F72DFE00232B7032490D4851
:10E95000F1F7C9FF314B1B78002B67D0304C3149A0
:10E96000227808481AF0B5FD2078012118F074FECD
:10E970000021207818F042FE5CE000BFC7200300B1
:10E98000CD200300848AFF1F6EDC0200D320030029
:10E9900006800100488EFF1FDC200300E1200300F9
:10E9A0003788FF1FE7200300F12003002AC4FF1F60
:10E9B00014B9FF1FB9C7FF1FD9050000E905000002
:10E9C00006210300008FFF1FE4C6FF1F172103006D
:10E9D000ACC7FF1F6CC5FF1F2821030000B9FF1F34
:10E9E000EAC9FF1FEEC4FF1F0EB9FF1F0F88FF1FEC
:10E9F0000788FF1FFE87FF1F3B21030000907B4617
:10EA0000F9050000D8C7FF1F40210300682103005B
:10EA1000512103005C21030073210300B0C5FF1FD7
:10EA2000E08EFF1F7C210300B8C7FF1F7A497B4897
:10EA3000F1F7B7FD4FF4D170F1F743FF784B80B297
:10EA400042F20F72904218801C4601D82B7823B9ED
:10EA50000020F1F7D7FE00232380724D724F2B6800
:10EA60000793079B3B604FF47A783378FF2B17D1DD
:10EA70002B680893089B3C6840F2AF101C1BF1F711
:10EA8000E4FE08FB00F0844200F2BA804FF4CC7040
:10EA9000F1F7DBFE18F0D2FD002800F0B180E4E7CA
:10EAA0000021624815F0CAFD039B1B786BB1604BD7
:10EAB0001B7853B9BAF1000F07D15E4B18780138B3
:10EAC0005146C0B2F7F7D4FB01E0002333700120B8
:10EAD000F4F77EFA584B594E00241C7096F82730F4
:10EAE000052BE2B201D00E2B04D196F85830002B42
:10EAF00040F089800134112C06F17006EED1504BA4
:10EB000050491A784548504C1AF0E3FC40F29F10E7
:10EB1000F1F79BFE1DF068FE02460B4600204FF009
:10EB200080411BF0DFF93AA3D3E900231DF0D2FEA8
:10EB30000B460246454939481AF0CBFCFEF7AAF8C5
:10EB40004FF48A70F1F781FE4149024620460AF0EF
:10EB500083FF2046F1F72DFFC4F804903D492F486C
:10EB60003D4CF1F7C0FEFA223C493D48F1F7E2FE88
:10EB7000142026681AF0D3FF8046F1F73BFF414688
:10EB8000304613F061FA142024681AF0C8FF0646D4
:10EB9000F1F726FF3146204613F056FA4FF4CC70B9
:10EBA000F1F753FE0322212888BFFF202D4918F0DA
:10EBB00085FD2D491948F1F7F4FC2B680A930A9B4F
:10EBC0002A4916483B60F1F78EFE2B680993099994
:10EBD0001248F1F7A5FE0020F4F7F4FD00210246EB
:10EBE000234817F004FF224817F034FE0FB0BDE8A9
:10EBF000F08F20490948F1F7D4FCFF233B70ECE586
:10EC00000023337031E7718A308AF7F7E5F971E74D
:10EC1000000000008084FE4049220300848AFF1F18
:10EC2000C88EFF1F4CD8FF1FD88EFF1F58C6FF1F6E
:10EC3000FD87FF1F0688FF1FC8C5FF1FB8BCFF1F49
:10EC400068C5FF1F8D21030054C4FF1FA7210300C7
:10EC50003CC5FF1FB821030098D7FF1FF9CE000065
:10EC6000BCC7FF1F256F0100CE210300D521030083
:10EC700018C5FF1F0C1D03002DE9F04FA7B006AF0C
:10EC800007F1200381464FF4CC7083E80600F1F7CA
:10EC9000DCFDB34CB7F92050B7F922A0212888BF7A
:10ECA000FF2018F007FC01232370AE4B7B6118781E
:10ECB00008B9F4F7D3FDABB2AB4D3B612B68BB6237
:10ECC000AA4BBA6A1A604FF4E170F1F7BEFDBD615C
:10ECD00040B10021F02300911A463869F1F779FD1F
:10ECE00003B210E04FF6C1661AFB06F640F241137C
:10ECF00096FBF3F63B6906F5A07603F101080FFADF
:10ED000086FA0FFA88F39A48FB6114F0AFF9994A32
:10ED10001578FF2D934611D197490988183900239A
:10ED20005145237006DCF969182903DC01231370AF
:10ED300002F099BC8BF8003002F095BC012D40F236
:10ED4000A980162D04D88D4BEB40DA0700F14581E0
:10ED5000894B1B88313B534578DCFA69132A75DCF3
:10ED6000874E96F80080B8F1FF0F40F03381854C54
:10ED70002078F2F751FC86F80080F2F7EBFE9BF862
:10ED800000300B2B09D1804B40F2A7101978F1F716
:10ED9000EFFC7E4B1A787E4B1A709BF80030022BEA
:10EDA00006D17B4B18780138C0B2F6F7F7FD07E0C3
:10EDB00006D9774B187801380021C0B2F7F758FA16
:10EDC000744B10225A72744B1B78042B03D101210F
:10EDD0000846F3F707FE714BDFF8EC81DFF8EC91A2
:10EDE0006F4E01221A704FF0000A6E4B504683F8A6
:10EDF00000A0F4F7EDF80A2018F0A4FD20786A4C82
:10EE0000F2F70AFC554694F82730052B5FFA8AF290
:10EE100002D00E2B42F0498494F85810002902F0D9
:10EE20006284618A208AF7F7D7F80AF1010ABAF1F9
:10EE3000110F04F17004E6D15C4BFF201870002321
:10EE40008BF80030F6F7D0F902F00DBC022D40F03F
:10EE5000C480534500F3C380FB69132B00F3BF80CC
:10EE6000474E3378FF2B00F0BA804F48702404FBE4
:10EE700003000122FF210BF0B9FDF2F76BFE012028
:10EE8000F6F788FAF7F7AAF9484AFF2333701370A8
:10EE900002F0E9BB002D40F0A08001231370444A2A
:10EEA00033481370434A404CDFF82491137014F038
:10EEB000DDF87D6194F8583097F8148033B31FFA69
:10EEC0008AF60123BA8B314620460BF03BFA18B183
:10EED0002C4B1B78032B0DD03B69C3F1F00132465C
:10EEE000012389B220460BF02DFA78B1254B1B780F
:10EEF000032B0BD094F82730092B42F087842E4B3C
:10EF00001B7803F0FD03012B02F0C2847B690133FF
:10EF1000112B7B6104F17004CCD1002D42F0A3834E
:10EF2000264A274B10781978884215461C4606D287
:10EF3000244B1878222828BFFF2018F0BBFA6A78E3
:10EF400023789A4206D21F4B5878222828BFFF20E8
:10EF500018F0B0FA0020F6F71DFA02F084BB00BFEB
:10EF6000C8C5FF1FE18EFF1F4CD8FF1F2CC5FF1F18
:10EF700058C6FF1FFD87FF1F0488FF1F0045610063
:10EF80004288FF1F2688FF1F70C5FF1F0888FF1FCC
:10EF90000688FF1F54C4FF1F04B9FF1F3A88FF1FD4
:10EFA0000FB9FF1F03B9FF1FB8BCFF1F0188FF1F68
:10EFB000D0C5FF1FE5C6FF1FABC7FF1F3788FF1F68
:10EFC0002AC4FF1FB9C7FF1F01B9FF1FB0C5FF1F2C
:10EFD000DD8EFF1F022D3FF443AF142D33D8C24BFB
:10EFE000EB40DE0708D5C14B1B78FF2B04D1AAF1FB
:10EFF00038039BB22B2B09D90A2D24D1BC4B1B887B
:10F00000313B534547F3C98602F02DBBFB69132BF7
:10F0100019DCB84B00251D70B44BFF221A70B64A9C
:10F0200001231370B54A237002201370F6F7B2F96A
:10F0300003238BF80030F2F78DFD29462846F7F7B9
:10F04000FBFA02F010BB022D7DD1DFF8A08298F808
:10F050000030FF2B41F0DE81AAF16E039BB2362B0C
:10F060000CD8FB69132B09DCF2F762FDFF288346FD
:10F0700004D0A34B1B78012B42F0CD85AAF1A70346
:10F080009BB22C2B14D8FB69132B11DC9C4B1A78E8
:10F09000012A14BF0122002201201A70F6F77AF922
:10F0A000984B18780138C0B2F6F778FC02F0DBBA5A
:10F0B000AAF1D6039BB22D2B01F2AC81FB69132B75
:10F0C00001F3A8818E4B1B78012B01F0A381032053
:10F0D000F2F7A2FA01218C4813F053FF00218A486D
:10F0E00013F055FF894B1A78032A05D102221A70B2
:10F0F0004CF21863019308E0022A08BF04214CF285
:10F10000186218BF0321197001920B23009301228A
:10F110002B23D7217C4816F0BDF87D4907F17000FC
:10F120001AF025FB05230093032207F17003ED215C
:10F1300078480BF019FC07F170001AF0D8FAF7F7CD
:10F140004DF802F090BA012D06F0A987032D06F0C4
:10F150004984042D06F09787052D12D0072D06F05F
:10F1600086870C2D06F095870D2D06F08687112DCC
:10F1700006F07787122D07F03381142D16D105F094
:10F18000BBBFBAF1310F00F3AA85BAF1000F40F30B
:10F19000A685FB69272B47F30686012D06F083879A
:10F1A000032D06F02384142D05F0AA87182D30D1E5
:10F1B000FB69322B10DD584BFA691B88323B9A42AF
:10F1C0000ADA564B1A78FF2A06D100212846197010
:10F1D000F7F732FA02F047BABC8B51481FFA8AF6A9
:10F1E0000123224631460AF095F9002802F05485A1
:10F1F0004A4B1978FF2902F04F854A4A535C632B2A
:10F2000002F24A85013318205354F7F715FA02F039
:10F210002ABA162D3CD1FB69692B13DD3E4BFA69E6
:10F220001B881E3B9A420DDA3F4B1A78FE2A09D002
:10F230003A4A002111702846FE221A70F7F7FCF9AD
:10F2400002F011BABC8B36481FFA8AF60123224617
:10F2500031460AF05FF9002802F064862F4B1978D6
:10F26000FF2902F05F86314D314B2A780B2000FBDD
:10F2700002325256632A02F355862A7800FB023383
:10F2800016205A5C01325A54F7F7D6F902F0EBB95E
:10F29000152D51D1FB69214C322B09DD2378FF2B31
:10F2A00006D1002128462170F7F7C6F902F0DBB934
:10F2B000BE8B1B481FFA8AF50123324629460AF005
:10F2C00029F9002802F0D6872178FF2902F0D28799
:10F2D000184A535C632B02F2CD8701331520535437
:10F2E000F7F7AAF902F0BFB9B6F217000188FF1FBD
:10F2F0000488FF1FC0C4FF1FD0C5FF1FE5C6FF1F46
:10F300000E88FF1F0688FF1F58C6FF1F2688FF1F95
:10F31000E8170300B8BCFF1F3C88FF1FA0C5FF1FF4
:10F3200020B9FF1F84C5FF1FE88EFF1FE6C6FF1F21
:10F33000A6C6FF1FC1C4FF1F112D73D1B7F81C80D3
:10F34000C4481FFA8AF60123424631460AF0E2F821
:10F3500050B34FF48E70F1F778FA0130C4B2292C13
:10F3600028BF022421464FF48E70F1F701FABA4902
:10F3700007F160001AF0FBF9214607F170001AF05E
:10F3800016FA4CF2186307F1700207F16001B148F8
:10F390000AF084F907F170001AF0A9F907F160008A
:10F3A0001AF0A5F902F05FB9012342463146AB4895
:10F3B0000AF0B0F8002803F007804FF4D670F1F798
:10F3C00044FA002843F00080A54907F150001AF0E4
:10F3D000CEF9A44907F160001AF0C9F9A24907F172
:10F3E00070001AF0C4F94FF4FC6307F1500107F103
:10F3F00060020093994807F170030AF097F907F14A
:10F4000070001AF074F907F160001AF070F907F152
:10F4100050001AF06CF901214FF4D670F1F7A8F9F9
:10F4200002F021B9172D40F09F80FB692C2B0EDCD8
:10F430008E4A002313708E4A13708E4A1120FF21CA
:10F4400013708BF80000F7F7F7F802F00CB9B7F873
:10F450001C8089481FFA8AF60323424631460AF087
:10F4600059F8054670B1834B13221A7009238BF8A3
:10F470000030824B18781DF0B7F90022F5F784FBB5
:10F4800002F0F1B803234246314672480AF042F8CE
:10F49000044670B1774B14221A7009238BF80030A0
:10F4A000764B58781DF0A0F92A46F5F76DFB02F06F
:10F4B000DAB803234246314671480AF02BF870B19E
:10F4C0006C4B15221A7009238BF800306B4B98781F
:10F4D0001DF08AF92246F5F757FB02F0C4B8032362
:10F4E000424631465D480AF015F870B1614B16226C
:10F4F0001A7009238BF80030604BD8781DF074F92E
:10F500000022F5F741FB02F0AEB803234246314634
:10F510005C4809F0FFFF044670B1564B17221A7081
:10F5200009238BF80030554B18791DF05DF9002246
:10F53000F5F72AFB02F097B80323424631465248BA
:10F5400009F0E8FF002802F08E804A4B18221A705A
:10F5500009238BF80030494B58791DF045F92246B4
:10F56000F5F712FB02F07FB8122D40F04181002127
:10F57000464813F00CFDB7F81C803F481FFA8AF686
:10F5800001234246314609F0C5FF054668B1404BAC
:10F5900000221A80364B022201201A70F5F7D8F8A3
:10F5A00013238BF8003002F05EB801234246314647
:10F5B000284809F0AFFF044660B1354B1D802C4B45
:10F5C000042201201A70F5F7C3F813238BF80030DA
:10F5D00002F049B8012342463146294809F09AFF12
:10F5E000054660B12A4B1C80214B062201201A706F
:10F5F000F5F7AEF813238BF8003002F034B801238E
:10F6000042463146154809F085FF044660B1204B5B
:10F610001D80174B082201201A70F5F799F8132363
:10F620008BF8003002F01FB80123424631461548DE
:10F6300009F070FF054668B3154B1C800C4B0A227D
:10F6400001201A70F5F784F813238BF8003002F0CC
:10F650000AB800BF34B9FF1F891D03005CB9FF1F42
:10F6600021190300921D03000B190300A0C5FF1F01
:10F67000E88EFF1FE6C6FF1F20B9FF1F20D5FF1F22
:10F6800048B9FF1F70B9FF1F84B9FF1F58C6FF1F7D
:10F69000A8C7FF1F012342463146C54809F03AFF7B
:10F6A000044660B1C34B1D80C34B0C2201201A706D
:10F6B000F5F74EF813238BF8003001F0D4BF012387
:10F6C00042463146BD4809F025FF054660B1B94BB9
:10F6D0001C80B94B0E2201201A70F5F739F813235C
:10F6E0008BF8003001F0BFBF012342463146B448D9
:10F6F00009F010FF044660B1AE4B1D80AE4B1022E6
:10F7000001201A70F5F724F813238BF8003001F06C
:10F71000AABF012342463146AA4809F0FBFE58B170
:10F72000A44B1C80A44B01201C70F5F711F8132387
:10F730008BF8003001F097BF012342463146A248C2
:10F7400009F0E8FE50B100214FF4D870F1F71EF82F
:10F7500000211220F6F770FF01F085BF0123424619
:10F7600031469A4809F0D6FE044678B14FF4D87471
:10F77000204600210134F0F7FBFFB4F5E17FF7D11B
:10F7800000211220F6F758FF01F06DBF0123424619
:10F7900031468F4809F0BEFE002803F0B2804FF4D6
:10F7A000E270F1F752F8012843F0AB80894907F184
:10F7B000600019F0DCFF884907F1700019F0D7FFED
:10F7C00007F1600146F22C3307F17002804809F01E
:10F7D00065FF07F1700019F08AFF07F1600019F06A
:10F7E00086FF21464FF4E270F0F7C0FF01F03BBF07
:10F7F000132D5AD1794C267896B907F170057849BE
:10F80000284619F0B4FF0F2300937648029601951D
:10F81000DC2323222D2109F0E5FF284619F067FF9C
:10F82000002171486D4D13F0B2FB01216E4813F0B9
:10F83000A8FB21786C4801EB4101490000232722F5
:10F84000323114F077FEB7F81C8060481FFA8AF650
:10F8500001234246314609F05DFE002803F0FF8097
:10F860002B78032B03F2FB8060495F48F1F73BF8EC
:10F87000504A2978138801311B010133C9B2138022
:10F8800029700A22C1F1040107F1700019F0A2FFEA
:10F890004FF6E07207F17001484809F0C9FE07F120
:10F8A000700019F024FF01F0DEBE082D4FD1504B3F
:10F8B000504C1B88313B534519DCFB69132B16DC7C
:10F8C0004D4BFF221A704D4B01251D704C4B0220F1
:10F8D0001D70F5F75FFD03238BF80030F2F73AF95E
:10F8E000002108462570F6F7A7FE01F0BCBEBAF16C
:10F8F000330F10DCFB69132B0DDC3F4B0022012181
:10F900000A201A70F6F798FE012364202370F5F799
:10F910006BFC01F0A8BEAAF13606B6B2322E4FF04B
:10F9200001050ED8FB69132B0BDC334B00210A2099
:10F930001D70F6F781FE64202570F5F755FC01F087
:10F9400092BE64202570F5F74FFC01F08CBE072DA8
:10F9500040F0C2817A69BD8B2A4800231FFA8AF4DD
:10F960001370214601232A4609F0D4FD064660B1F2
:10F97000254A1378591EC9B2FF29117001D10C21F3
:10F9800049E0082948D1072145E001232A462146BC
:10F990001E4809F0BFFD8046002844D01A4A13785B
:10F9A000591CC9B20C29117032D9167034E000BF4D
:10F9B00084B9FF1FA8C7FF1FE88EFF1F98B9FF1F5C
:10F9C000ACB9FF1FC0B9FF1FD4B9FF1FE8B9FF1FB3
:10F9D000FCB9FF1F471E0300A71A03000088FF1F82
:10F9E000AB1503005CB9FF1F58C6FF1FF21A0300D6
:10F9F0000488FF1F3A88FF1F0188FF1FD0C5FF1F23
:10FA0000E5C6FF1F20B9FF1FA0C5FF1F34B9FF1FA8
:10FA1000082901D10921117012782D210220F2F755
:10FA2000D1F903F00BBC01232A462146BF4809F057
:10FA300071FD002857D0BE4DBE482988DFF81493C9
:10FA40005F393722434609B214F074FDF5F728FAFE
:10FA5000B949B848F0F747FFB84B4FF4B37019787D
:10FA6000F0F786FEB64B40F265101978F0F780FE8D
:10FA700040F2671440F26F1663006FF4337B5B440F
:10FA8000204619F80310DFF8CC820134F0F770FE3D
:10FA9000B442F1D140F277166300A3F2DE23204690
:10FAA00018F803100134F0F763FEB442F4D13220A9
:10FAB00017F048FF29889F480A234FF0000A5F3952
:10FAC0008DE8080437225E2309B215F0E3FB9D4B55
:10FAD00020461978F0F74CFE9B4B40F2A91019789C
:10FAE000F0F746FE82E001232A462146974809F0B6
:10FAF00011FD50B1964B1A78082A06D8954911F88D
:10FB0000123013B1013B03F0ECBA01232A4621461F
:10FB1000914809F0FFFC20B18D4B1A78082A43F276
:10FB2000D982BAF1190F08DDDFF80482B8F8003085
:10FB3000A3F17D029245C3F2D78201232A462146D2
:10FB4000824809F0E7FC002843F0EE8201232A46B0
:10FB50002146814809F0DEFC002843F0F682BAF124
:10FB6000190F08DDDFF8C881B8F80030A3F17D0275
:10FB70009245C3F22D8301232A462146734809F09A
:10FB8000C9FC002843F0458301232A4621467248D8
:10FB900009F0C0FC002843F04883BAF1190F06DDD4
:10FBA000634E3388A3F17D029245C3F24D83012356
:10FBB0002A462146654809F0ADFC002803F065831C
:10FBC000634B1B780B2B43F06083644A1378002B44
:10FBD00003F05B83012B43F25583023B1370012139
:10FBE0000920F6F729FD7A69012313707B691B78D8
:10FBF000002B01F03885594B504A19781278914200
:10FC0000984610D9564C207838B1524BD87BF3F730
:10FC100025FE0023237001F026BDF3F71FFE01230C
:10FC2000237001F020BD4FF4D470F0F70EFE494C64
:10FC3000012894F80F902AD14FF0000A0546A27BC4
:10FC400098F800309A421FFA8AF60CD80DB194F851
:10FC50000F904846F3F7B6FD31460246414816F08C
:10FC6000C6FE002507E00020F3F7ACFD3146024652
:10FC70003C4816F0BCFE0AF1010ABAF1080FA4F1E3
:10FC80000204DCD1374816F0E5FD01F0ECBC072595
:10FC900001264FF6FF7AA27B98F800309A420CD8E2
:10FCA0000EB194F80F904846F3F78CFD29460246B2
:10FCB0002C4816F09CFE002607E00020F3F782FD9A
:10FCC00029460246274816F092FE013DADB2554541
:10FCD000A4F10204DFD1D5E7052D40F0C880B7F8C4
:10FCE0001C90214D1FFA8AF801234A4641462846B6
:10FCF00009F010FC2C460646002855D0144E1B4D2A
:10FD000033782A78C2EB0308013BDBB2FF2B5FFAA2
:10FD100088F833702ED1164B1B785A1ED2B20C2A9B
:10FD200032702FD90D3B2B7028E000BF48B9FF1F60
:10FD30000488FF1F58C6FF1FF22103003988FF1FE8
:10FD4000FC87FF1FF08EFF1F2BC4FF1F5CB9FF1F36
:10FD5000A0C5FF1F2788FF1F70B9FF1F368EFF1F2A
:10FD6000C4C5FF1F18C5FF1F20B9FF1FE88EFF1F66
:10FD70002AC4FF1F9A4205D9013A2A7000210420A3
:10FD8000F6F75AFC33782A78618920899A1AE38930
:10FD90001944D2B2434689B2F2F714F80021052083
:10FDA000F6F74AFC01F05FBC414601234A4605F1E3
:10FDB000140009F0AFFB8046002838D0BE4ABF4887
:10FDC000137890F800E0CEEB03050133DBB2CEEB05
:10FDD00003010C29EDB21370B9499046814607DD45
:10FDE0000A789A4204D90EF101030370314607E004
:10FDF0000A789A4207D8002188F8001089F8001084
:10FE00000420F6F719FC98F8003099F80020618971
:10FE100020899A1AE3891944D2B22B4689B2F1F7A4
:10FE2000D1FF00210520F6F707FC01F01CBCA54B13
:10FE30001B88643B9A4581F21684FB69142B41F3BD
:10FE400012849D4B9D4A1B781278698928899B1AD8
:10FE5000EA891144DBB2FF2289B2F1F7B3FF062031
:10FE600041468BF80000F6F7E7FB01F0FCBB062DDE
:10FE700040F0AD82B7F81C80934C1FFA8AF601233C
:10FE800042463146204609F045FB814658B18F4C29
:10FE900000212078F1F7C0FF002120700720F6F73D
:10FEA000CBFB01F0E0BB01234246314604F11400D4
:10FEB00009F030FB824658B1844C01212078F1F7DB
:10FEC000ABFF494620700720F6F7B6FB01F0CBBB2D
:10FED00001234246314604F1280009F01BFB81460C
:10FEE00068B37A4D05238BF80030794B2878FF22D0
:10FEF00002211A70F1F790FF724B2870198875482B
:10FF00005F395346372209B214F014FBF4F7C8FFE7
:10FF1000714B2978012203201A70F6F78DFB664B8E
:10FF2000664A1B781278618920899B1AE289DBB2C4
:10FF3000114489B21A46F1F745FF01F094BB012341
:10FF40004246314604F1B40009F0E4FA8246002842
:10FF500000F028825D4C2378082B26464CD1DFF830
:10FF600058A15E4E9AF8003021784FF0A80808FB9F
:10FF70000363FF2283F891202846F6F75DFB0121F9
:10FF80000720F6F759FB4FF6FF71524812F0FFFFBA
:10FF900023785048CDF8049003EB430203EB820230
:10FFA0002D320923009312B25A23642115F072F9FD
:10FFB0002378484803EB430203EB82022D324B4681
:10FFC00012B2672114F0B6FA9AF8003008FB036603
:10FFD0003B4B96F891101B784A4607F170000AF0E7
:10FFE0005DF907F170013B4819F03CFA07F1700028
:10FFF00019F07DFB01F037BB23780B2B0FD12E4B73
:020000021000EC
:100000001A78364BA82101FB0233D3E920010122E3
:10001000F4F7BAFD09238BF8003001F024BB2378F4
:100020000C2B0FD1244B1A782C4BA82101FB023347
:10003000D3E922010122F4F7A7FD09238BF8003050
:1000400001F011BB2478E4B2092C0ED11A4B1A78B6
:10005000224BA82101FB0233D3E926010122F4F748
:1000600093FD8BF8004001F0FEBA3378012B0FD1DD
:10007000114B1A78194BA82101FB0233D3E9120165
:100080000122F4F781FD09238BF8003001F0EBBA6F
:1000900033780E4C032B23D1074B1A780F4BA82132
:1000A00001FB0233D3E916010122F4F76DFD0923A8
:1000B0008BF8003001F0D7BAA0C5FF1FE88EFF1FF4
:1000C0002AC4FF1F0488FF1F20B9FF1FE6C6FF1FB9
:1000D0000188FF1F58C6FF1FB8C7FF1F008FFF1FF3
:1000E0002378052B35D1C14D2C78002021460AF00C
:1000F000ADF880F00101C9B220460AF07FF8002176
:100100000720F6F799FA4FF6FF71B94812F03FFF52
:10011000002409238DE818006E223C236421B44892
:1001200015F0B8F823466E226721B14814F002FAA0
:10013000297820460AF08AF8F2F700FF297820464D
:100140000AF084F86D2102465120F2F7BBFD01F060
:100150008ABA2378062B51D1A44DA64E2C780120C3
:1001600021460AF073F880F00101C9B220460AF076
:100170004FF8337808B1013300E0013B002107203C
:10018000002433704FF00908F6F756FA4FF6FF7166
:10019000974812F0FCFE0194CDF800803C237B22AE
:1001A0006421934815F076F823467B226721904816
:1001B00014F0C0F9297801200AF048F8F2F7BEFEE1
:1001C0000194CDF8008008237B223D21884815F05A
:1001D00061F823467B223D21854814F0ABF9317844
:1001E0008348F0F784FB297801200AF02FF87A2160
:1001F00002465120F2F7A0FD01F035BA237803F052
:10020000FF057BBB794B1A787B4BA82101FB02339E
:1002100000200021C3E910014CF21861744812F06B
:10022000B6FE23787248019503EB430203EB82028A
:100230002D320923009312B23C23642115F02AF8D1
:1002400023786B4803EB430203EB82022D322B46EB
:1002500012B2672114F06EF968496548F0F743FB64
:1002600001F001BA2378022B30D1604B1A78624B2F
:10027000A82101FB023300200021C3E914014CF244
:1002800018615B4812F083FE2378594803EB430260
:1002900003EB8202002509232D328DE8280012B2DB
:1002A0003C23642114F0F6FF2378514803EB43020A
:1002B00003EB82022D322B4612B2672114F03AF979
:1002C0004E494B48F0F70FFB01F0CDB92578EDB260
:1002D000072D35D1454C26780320314609F0B6FF6D
:1002E00080F00101C9B2304609F0A6FF284600217E
:1002F000F6F7A2F94FF6FF713D4812F048FE0025CF
:1003000009238DE82800882246236421384814F008
:10031000C1FF2B4689226721354814F00BF921785B
:10032000032009F093FFF2F709FE2178032009F07A
:100330008DFF892102465120F2F7EAFD01F093B9C1
:1003400023780A2B41F08F812D4B2B4801221A7004
:10035000264B1978A82202FB010292F8683001337B
:10036000DBB2022B82F8683006D8546840F6FF7280
:10037000944207D0022B05D1A82303FB01010023DF
:1003800081F8683000210520F6F756F93078013001
:100390000021C0B2F1F740FD00210720F6F74CF92B
:1003A00001F061B901234246314604F1500009F0E1
:1003B000B1F8002803F0C380124B1B78082B03F020
:1003C000BE8051460820F6F737F901F04CB9092DE7
:1003D0001AD1BB8B7B84A7F820A007F1200393E8F8
:1003E0000300FBF71FFE01F03EB900BFA0C5FF1FD1
:1003F00058C6FF1FBBC7FF1F008FFF1FFD21030053
:10040000C8C5FF1FE6C6FF1F042D01F02C81022D79
:1004100040F08D80112300257B61BD61BA4B1B78B4
:10042000AB4201D0FF2B68D1BB69B84EB84AB7F8D0
:100430001C900133DBB27024BB6104FB0564002314
:100440001FFA8AF81370414601234A46204609F0F4
:1004500079FF48B1AF4B1B78032B05D1AE4B1B780E
:10046000012B2BD103F04BB93B69C3F1F00142469C
:10047000012389B2204609F065FF48B1A54B1B78DE
:10048000032B05D04FF4E170F0F7DFF90028E5D039
:10049000012342463969204609F054FF002803F041
:1004A0002E819C4B1B78032B03F029814FF4E170C4
:1004B000F0F7CBF90028D1D103F021B994F85830E6
:1004C000002B03F01C8194F825B0BBF1000F43F022
:1004D00016810320F4F75EFF8E4B1878F1F79CF835
:1004E0008D4B5A460121204683F800B00FF0ACFD39
:1004F000854B1D70894B01221A707B69013B0135C8
:1005000013F0FF03EDB27B6188D1BB6953B9824C14
:100510002378FF2B06D00120F4F73CFFF5F75EFEB1
:10052000FF2323700320F1F777F801F09CB80B2D1F
:100530007B4E30D1B7F81C807A481FFA8AF5012328
:100540004246294608F0E6FF002803F0C384DFF89E
:10055000FC9199F80040EF2C03F2BC840A34E4B219
:1005600040F2951089F80040F0F76FF9214617F036
:10057000F5F8348899F800003E3C009432231422A8
:10058000FA21F0F716F9A3B281B23222664809F0D7
:100590001FFA01F068B80C2D40F0858100216348F6
:1005A000634C644D12F0F3FCB7F81C802378BB61F8
:1005B0001FFA8AF60123424631465E4808F0AAFF38
:1005C000814658B32378013BDBB2FF2B23701AD14D
:1005D00059490A788AB9594B1B780B2B02D8013B31
:1005E000237010E00C2020700C2BA3F10D0008707C
:1005F00007D8013B23700A7003E0013A00230A7018
:100600002370F4F7FDFFEB89698922782889194462
:1006100089B2BB69F1F7D6FB01F025B80123424648
:10062000314605F1140008F075FF824620B32378A7
:10063000424A414910780A780133DBB29E18B04231
:10064000237006DC0B2881F8009084F8009008D90C
:1006500005E00C2B05D901320C230A702370F4F746
:10066000CFFFEB89698922782889194489B2BB694F
:10067000F1F7A8FB00F0F7BF01234246314605F130
:10068000280008F047FF8146002861D040F29F1003
:10069000F0F7DBF8022896BF411C5146C9B240F280
:1006A0009F10F0F765F8264907F1600019F05FF830
:1006B00040F29F10F0F7C9F81CF096F802460B467E
:1006C00000204FF0804119F00DFC1E4B00221CF061
:1006D00001F91CF0F7FB0222014607F1700019F046
:1006E000CCF8002307F1700207F16001164808F00A
:1006F000D5FF07F1700018F0FAFF07F1600018F05D
:10070000F6FF00F0B0BF00BF4288FF1FB8BCFF1F5C
:10071000C8C5FF1F2688FF1F0188FF1F3A88FF1FDB
:100720000488FF1F5CB9FF1F84B9FF1F58C6FF1F55
:10073000A0C5FF1F20B9FF1FE88EFF1F0BB9FF1FC9
:10074000881A030000405F4048B9FF1F70C5FF1FB3
:1007500001234246314605F13C0008F0DBFE00284B
:1007600000F08E80BC4CDFF83083BC48DFF804A377
:100770004FF6FF7112F00BFCB8F800302288B74832
:10078000CDF80490693B0B3A0B261BB212B24946D6
:10079000009614F07FFD2288B048CDF80490213AED
:1007A0000A25C82312B20F21009514F073FD228888
:1007B000AA480A3A4B4612B2052113F0BBFEA849DB
:1007C000A648F0F790F849464FF48C70EFF7D0FF49
:1007D00007F17000F5F72EF807F17000FDF7BEFA8B
:1007E0008AF8000007F1700018F081FF9AF80030D5
:1007F000002B00F03887B8F8003022889748693B12
:100800000B3A49468DE840021BB212B214F042FD89
:100810002288924800954FF4E3530B3A01934946DE
:10082000782312B214F036FD22888C480A3A4B46DF
:1008300012B2052113F07EFE8A498848F0F753F87A
:100840002A46082307F170008749EFF74BFE07F1AE
:100850007001824818F006FE07F1700018F047FF9B
:1008600022887E4800954FF478430B3A019312B2E8
:100870007823494612F058FEF4F7C2FE00F0F3BEAA
:1008800001234246314605F1640008F043FE00288A
:1008900003F0C2834FF4E570EFF7D7FF002803F0B1
:1008A000EB8303F0B9BB0D2D40F0C184B7F81C8079
:1008B0006E481FFA8AF601234246314608F02AFEA6
:1008C000B8B16B4C0023237020780130EFF7BDFFE7
:1008D000684A694B1278187082429CBFFF221A70D6
:1008E0001A78664B21781A700D20F5F7A5FE00F0F6
:1008F000BABE012342463146614808F00BFEB8B14A
:100900005B4C0223237020780130EFF79EFF594A99
:10091000594B1278187082429CBFFF221A701A78C5
:10092000564B21781A700D20F5F786FE00F09BBE1D
:10093000012342463146534808F0ECFDB8B14C4C17
:100940000323237020780130EFF77FFF494A4A4B99
:100950001278187082429CBFFF221A701A78474B97
:1009600021781A700D20F5F767FE00F07CBE012398
:1009700042463146444808F0CDFDB8B13C4C042312
:10098000237020780130EFF760FF3A4A3A4B127833
:10099000187082429CBFFF221A701A78374B217858
:1009A0001A700D20F5F748FE00F05DBE01234246A7
:1009B0003146364808F0AEFDB8B12D4C0523237002
:1009C00020780130EFF741FF2A4A2B4B127818703C
:1009D00082429CBFFF221A701A78284B21781A7025
:1009E0000D20F5F729FE00F03EBE012342463146B8
:1009F000274808F08FFDA0B11F4B1D4C19782078B7
:100A00001E4B0139C9B201301970EFF7B1FEFF2159
:100A10000D20F5F711FE21780D20F5F70DFE00F001
:100A200022BE0123424631461A4808F073FDA8B39E
:100A30000F4C114B20781978104B01301970EFF7DB
:100A400097FEFF210D20F5F7F7FD21780D20F5F732
:100A5000F3FD00F008BE00BF3C88FF1F58C6FF1F13
:100A600009220300751A030038C5FF1F20B9FF1FB4
:100A7000E6C6FF1F2AC4FF1FA0C5FF1FE88EFF1F89
:100A800048B9FF1F5CB9FF1F70B9FF1F4CBAFF1FA9
:100A900084B9FF1F98B9FF1F0488FF1F0123424636
:100AA0003146A94808F036FDA0B1A84BA84C1978EA
:100AB0002078A84B0131C9B201301970EFF758FE08
:100AC000FF210D20F5F7B8FD21780D20F5F7B4FDD5
:100AD00000F0C9BD0123424631469F4808F01AFD87
:100AE00080B19A4A1378013BDBB2FF2B137002BF2F
:100AF0009A4B1B781370964B0D201978F5F79CFDD7
:100B000000F0B1BD012342463146954808F002FD90
:100B100088B18E4A9149137809780133DBB2994242
:100B200013703CBF00231370894B0D201978F5F723
:100B300083FD00F098BD012342463146894808F004
:100B4000E9FC044628B1FF210D20F5F775FD00F002
:100B50008ABD012342463146834808F0DBFC002869
:100B60005ED0824A13780133DBB21370062B154630
:100B70007F4B88BF14701A782B78934203D113B13E
:100B80007A4A013313702B787A49012B07F1600000
:100B900003D118F0ECFD78491CE0022B03D118F0CA
:100BA000E6FD764916E0032B03D118F0E0FD744909
:100BB00010E0042B03D118F0DAFD72490AE0052B8E
:100BC00003D118F0D4FD704904E0062B09D118F0C8
:100BD000CEFD6E4907F1700018F0C9FD4FF4FC63BB
:100BE00008E018F0C4FD6A4907F1700018F0BFFD75
:100BF00046F22C3307F1600107F170025A4808F001
:100C00004DFD07F1700018F072FD07F1600018F05B
:100C10006EFD297840F21710EFF7AAFD00F023BD12
:100C20000123424631465B4808F074FC81460028A7
:100C300000F0B6804E494D480B7800785A1CD2B26D
:100C400090420A700C4602D108B102330B7023782F
:100C50005149062B82BF464B00221A702378012B84
:100C600007F1500008D118F082FD4C4907F16000EF
:100C700018F07DFD404935E0022B08D118F077FDD2
:100C8000464907F1600018F072FD3C492AE0032B49
:100C900008D118F06CFD414907F1600018F067FDBC
:100CA00037491FE0042B08D118F061FD3B4907F1DB
:100CB000600018F05CFD334914E0052B08D118F0F2
:100CC00056FD364907F1600018F051FD2E4909E044
:100CD000062B0ED118F04BFD304907F1600018F0DB
:100CE00046FD2A4907F1700018F041FD4FF4FC63FE
:100CF0000DE018F03CFD294907F1600018F037FDC0
:100D0000234907F1700018F032FD46F22C3307F149
:100D1000500107F1600200931E4807F1700308F0CC
:100D200005FD07F1700018F0E2FC07F1600018F013
:100D3000DEFC07F1500018F0DAFC217840F21510C3
:100D4000EFF716FD00F08FBCACB9FF1FA0C5FF1F69
:100D5000E6C6FF1FE88EFF1FC0B9FF1F2AC4FF1F92
:100D6000D4B9FF1FFCB9FF1F34B9FF1F348DFF1F1B
:100D7000ECC4FF1FE41A0300F01A0300F41A030086
:100D8000F81A0300FC1A03003B1603003716030091
:100D90000C1D0300E8B9FF1F001B0300E91A030044
:100DA000012342463146C34808F0B4FB002800F056
:100DB000AB80C14BDFF834831D78C04B98F80040FE
:100DC0001A784FF6E07395422CBF1D464FF4FC6530
:100DD000FF2C4FF4CD7046460AD1EFF736FDB849E7
:100DE00088F8000007F1600018F0C1FCB54961E027
:100DF000EFF72BFD844240F29B100AD1EFF725FD5F
:100E0000AF4988F8000007F1600018F0B0FCAE4967
:100E100050E0EFF71AFD84424FF4CE700AD1EFF79D
:100E200014FDA74988F8000007F1600018F09FFC46
:100E3000A6493FE0EFF709FD844240F29D100AD138
:100E4000EFF703FD9E4988F8000007F1600018F0F5
:100E50008EFC9F492EE0EFF7F8FC844208D19849B8
:100E600088F8009007F1600018F081FC994921E0B2
:100E70004CB90123924988F8003007F1600018F05E
:100E800076FC954916E0012C09D109238C4988F894
:100E9000003007F1600018F06AFC90490AE0092C64
:100EA0000ED10A23864988F8003007F1600018F057
:100EB0005EFC8B4907F1700018F059FC2B460EE0E0
:100EC000FF237F4988F8003007F1600018F04FFCDD
:100ED000844907F1700018F04AFC46F22C3307F100
:100EE000600107F17002734808F0D8FB07F1700049
:100EF00018F0FDFB07F1600018F0F9FB31784FF4B2
:100F00009070EFF735FCAEE3012342463146764858
:100F100008F000FB002800F0A280674B734D5E785C
:100F2000664B6C781A784FF6E07396422CBF1E46DB
:100F30004FF4FC66FF2C4FF4CD70A84609D1EFF7B3
:100F400084FC6B49687007F1600018F010FC5D4983
:100F50005BE0EFF77AFC844240F29B1009D1EFF797
:100F600074FC6349687007F1600018F000FC564992
:100F70004BE0EFF76AFC84424FF4CE7009D1EFF7F3
:100F800064FC5B49687007F1600018F0F0FB4F49A2
:100F90003BE0EFF75AFC844240F29D1009D1EFF795
:100FA00054FC5349687007F1600018F0E0FB4849B1
:100FB0002BE0EFF74AFC844208D100234C496B70C8
:100FC00007F1600018F0D3FB42491EE044B9012349
:100FD00047496B7007F1600018F0C9FB3E4914E007
:100FE000012C08D1092342496B7007F1600018F009
:100FF000BEFB3A4909E0092C0DD10A233C496B702C
:1010000007F1600018F0B3FB354907F1700018F0E4
:10101000AEFB33460DE0FF2335496B7007F16000EE
:1010200018F0A5FB2F4907F1700018F0A0FB46F25D
:101030002C3307F1600107F170022B4808F02EFBFA
:1010400007F1700018F053FB07F1600018F04FFB38
:1010500098F8011040F21F10EFF78AFB03E3012319
:1010600042463146234808F055FA002800F0FB823A
:10107000214C23786BB901232049237007F15000DC
:1010800018F075FB1E4907F1600018F070FB0D4960
:1010900097E0012B36D102231849237007F1500045
:1010A00018F065FB164907F1600018F060FB06496F
:1010B00087E000BF10BAFF1F3788FF1F2AC4FF1F39
:1010C0000B1B0300F01A0300F41A0300F81A0300C4
:1010D000FC1A03003B160300371603003F160300FB
:1010E000431603000C1D030024BAFF1FB9C7FF1FDE
:1010F000131B030038BAFF1FE4C6FF1F1B1B0300AE
:1011000079160300022B0DD10323C449237007F184
:10111000500018F02CFBC24907F1600018F027FBC3
:10112000C0494EE0032B0DD10423BC49237007F1C5
:10113000500018F01CFBBA4907F1600018F017FBCB
:10114000B9493EE0042B0DD10523B449237007F1C2
:10115000500018F00CFBB24907F1600018F007FBD3
:10116000B2492EE0052B0DD10623AC49237007F1BF
:10117000500018F0FCFAAA4907F1600018F0F7FADD
:10118000AB491EE0062B0DD10723A449237007F1BC
:10119000500018F0ECFAA24907F1600018F0E7FAE5
:1011A000A4490EE0072B13D108239C49237007F1B3
:1011B000500018F0DCFA9A4907F1600018F0D7FAED
:1011C0009D4907F1700018F0D2FA4FF4FC6312E069
:1011D00000239249237007F1500018F0C8FA904993
:1011E00007F1600018F0C3FA944907F1700018F095
:1011F000BEFA46F22C3307F1500107F1600200936A
:101200008F4807F1700308F091FA07F1700018F0A9
:101210006EFA07F1600018F06AFA07F1500018F052
:1012200066FA217840F2FB10EFF7A2FA1BE2102DCC
:1012300040F08181002323703388313B534519DC12
:10124000FB69132B16DC7F4BFF221A707E4B0124A7
:101250001C707E4B02201C70F4F79CF803238BF863
:101260000030F0F777FC7A4B002108461C70F5F748
:10127000E3F9F8E1B7F81C8076481FFA8AF60123F3
:101280004246314608F046F9054698B140F21B1037
:10129000EFF7DBFA20B1012814BF0021032100E0A1
:1012A000012140F21B10EFF763FAFE211020F5F741
:1012B000C3F9D8E1012342463146674808F02AF9CC
:1012C000044688B1654B33221A70654B20225A724E
:1012D0006420F3F789FFBB691B683B65614B3A6D7E
:1012E0001A60614B1D70BEE10123424631465F48E2
:1012F00008F010F9054660B3584B5D4934221A7066
:10130000574B18225A7207F1600018F030FA594909
:1013100007F1700018F02BFA4FF6E07307F1700236
:1013200007F16001514808F0B9F907F1700018F0B1
:10133000DEF907F1600018F0DAF96420F3F754FFE2
:10134000BB691B683B66474B3A6E1A60464B1C7084
:1013500089E1012342463146474808F0DBF804465C
:1013600060B33E4B454935221A703D4B14225A72E8
:1013700007F1600018F0FBF93E4907F1700018F022
:10138000F6F94FF6E07307F1700207F160013A4891
:1013900008F084F907F1700018F0A9F907F160006E
:1013A00018F0A5F96420F3F71FFFBB691B683B67C2
:1013B0002C4B3A6F1A602C4B1D7054E101234246AE
:1013C00031462F4808F0A6F8054600287FD04FF494
:1013D000D770EFF73AFA012858D121464FF4D77069
:1013E000EFF7C6F9274907F1600018F0C0F9264960
:1013F00007F1700018F0BBF946F22C3307F17002C8
:1014000007F160011E4808F049F907F1700018F073
:101410006EF907F1600018F06AF924E11B1B030064
:1014200079160300F81A0300FC1A03003B160300A8
:10143000371603003F160300431603000C1D03007C
:1014400038BAFF1F0188FF1FD0C5FF1FE5C6FF1F69
:101450003A88FF1F20B9FF1F34B9FF1FE6C6FF1FE0
:1014600054C4FF1FCC8EFF1FBBC7FF1F48B9FF1F0F
:101470002C1D0300311D03005CB9FF1F351D030047
:1014800070B9FF1F711903003B1D030001214FF4C8
:10149000D770EFF76DF9BD4907F1600018F067F9F3
:1014A000BB4907F1700018F062F94FF4FC6307F1D3
:1014B000700207F16001B74808F0F0F807F170001A
:1014C00018F015F907F1600018F011F9CBE00123CD
:1014D00042463146B04808F01DF8002800F0C380AD
:1014E0004FF48A70EFF7B1F9AC4CAD490230C0B29D
:1014F0001E28207007F1600088BF257018F037F9AA
:10150000217807F1700018F052F907F1600100230B
:1015100007F17002A04808F0C1F807F1700018F058
:10152000E6F807F1600018F0E2F821784FF48A70CD
:10153000EFF71CF997E00E2DDFF8A8923AD1328828
:10154000313A0023524523701BDCFA69132A18DC58
:10155000944A1370944BFF221A70944A012313701B
:10156000934A237013702370022003238BF80030FA
:10157000F3F710FFF0F7EEFA00210846F5F75CF8F4
:1015800071E0B7F81C8083481FFA8AF601234246AF
:10159000314607F0BFFF002802F0F786854D2B7813
:1015A000FF2B02F0F286844B1A78012A42F0ED8676
:1015B00002F0EFBD0F2D56D1804C267896B907F179
:1015C00070057F49284618F0D2F80F2300937D4814
:1015D00002960195DC2323222D2108F003F92846E9
:1015E00018F085F800217848744D11F0D0FC0121E5
:1015F000754811F0C6FC2178734801EB41014900A0
:1016000000232722323112F095FFB7F81C806F4873
:101610001FFA8AF601234246314607F07BFF002875
:1016200003F051822B781F2B03F24D8268496648E4
:10163000EFF759F92978674B31225A540131C9B271
:1016400029700A22C1F1200107F1700018F0C2F8D8
:1016500061484FF6E07207F1700107F0E9FF07F10A
:10166000700018F044F85D4B4FF4A0721A805C4B88
:10167000F0221A805B4B1B78012B06D15A4A5B493A
:101680005B48EFF757F905F026BCC820F2F72AF9B6
:101690004FF4CC70EFF7D9F803225649212888BFC0
:1016A000FF2016F00BF805F016BC0A2B1ED194F89B
:1016B0005830002B3DF4B9AB002D7DF4B6AB4E4B4A
:1016C0001878A38B83427DF4B0AB0125F3F7FAFBC6
:1016D000E5834A494A48EFF706F9E18B4848EFF7B6
:1016E00015F9FDF7A2BB0A2B3DF49FAB0B2B7DF444
:1016F0009CAB94F85830002B3DF497ABA38B092B8F
:1017000005D1404A337812789A4233D13BE00A2B14
:1017100004D13D4932780978914234D00A2B29D03E
:101720000B2B02D13278FF2A2DD00B2B22D00C2B81
:1017300002D13278FE2A26D00C2B1BD00D2B03D1E0
:1017400099F80020022A19D00D2B13D00E2B3DF44E
:101750006CAB0F2B3DF469AB98F8002042FA03F311
:10176000DB077DF562AB40F21910EFF76EF850B968
:10177000FDF75BBB0023E383FDF757BB0123E38346
:101780002384FDF752BB0123F5E700BF6619030070
:101790003B1D030070B9FF1F84B9FF1FA5C6FF1FC3
:1017A000411D0300C0C4FF1F0188FF1FD0C5FF1FDC
:1017B000E5C6FF1FF18EFF1FABC7FF1F0088FF1F8D
:1017C000AB1503005CB9FF1F58C6FF1FE8B9FF1F28
:1017D000F21A0300CCC4FF1F98B9FF1F0488FF1F33
:1017E0003C88FF1FFD87FF1FA086010051080000F5
:1017F000388EFF1F256F01003F88FF1F1422030052
:10180000848AFF1F00B9FF1FEAC9FF1F122B0CD1EA
:1018100000238BF80030BB8B7B84A7F820A0AC4B57
:10182000386ABA8C18609A8050E00A2B1DD1E38B7D
:1018300000228BF800208BB9A6491846CA187033CD
:1018400092F827500A2D08BFD083B3F5EE6FF5D17B
:10185000A14B207F18700125E58315E09E4BE283A4
:10186000FF201870F3F7C0FC5DE00B2B40F08C817B
:10187000A68BA6F10903032B2AD8984B1B7803F0FB
:10188000FD03012B5FD0FF20F3F7AEFCFDF73EBB5D
:10189000934DA28B2978914248D12B70297840F240
:1018A000AB10EEF765FF00228A4B8E48114693F885
:1018B0002760092E3DD01432B2F5AA7F03F17003E0
:1018C000F5D12B78E38300238BF80030FF20C9E7A4
:1018D0000D2E00F0BF800E2E00F0E2800F2E00F0E3
:1018E0001D8140F21910EEF7B0FF00283DF40EAB59
:1018F000E28B7D4D00238BF80030002A40F02B81D5
:1019000001232A78E383B3401343DBB2FF202B701B
:10191000F3F76AFC228C002A40F02481297840F2F7
:10192000C710EEF725FF0125FDF7F0BAD2B22A70F5
:10193000B4E793F85860002EBDD08618367C002E90
:10194000B9D0D983B7E7002362498BF80030184635
:1019500091F827200B2A07D1DAB2904504D08A8B60
:10196000093A92B2032A73D90133112B01F17001A4
:10197000EED15E4BA18B1B785D4DE68B002B14BF27
:101980004FF4807000200B2914D11EB90123E3838A
:10199000FF2157E0574B00212970E1831880564BF7
:1019A0001A78564BA82000FB023300250026C3E915
:1019B0000E5648E00C294FF0010E0CD11EB9A4F8C8
:1019C0001EE0FE213EE04B4B18804D4B0021E18391
:1019D00019802970E3E7474A474B26BB09290CBF0A
:1019E00048494949A4F81EE091F800801E781FFA82
:1019F00088F1FF2E118008D040461AF0F5FE3F4BCB
:101A0000A82202FB0636C6E90E01404B85F800808D
:101A10001A783A4BA82101FB023300210022C3E9C6
:101A20000E1229780FE01B7810800021FF2BE18334
:101A300007D0324AA82101FB032300210022C3E979
:101A40000E12002129704FF4F170EEF791FE3DE780
:101A5000C88389E72E4D2B780022022B8BF80020BB
:101A600004D10123E38303232B7014E0032BE283CF
:101A70004FF0010102D1228429700CE0012B4FF0BC
:101A8000020009BF287028702384194618BF2184DA
:101A900020460EF0C7FA002120460EF0C3FA15E7E3
:101AA00000238BF800301B4A1B4B1B78127803F085
:101AB0000F0302F00F02013201339342C8BF00232B
:101AC00099F80020638402F0F00213433BE000BF6A
:101AD000D0C7FF1FB8BCFF1F3F88FF1F6CC5FF1F8B
:101AE000F18EFF1F20B9FF1F01B9FF1F28C4FF1F80
:101AF0000FB9FF1FC6C5FF1F0988FF1F008FFF1FFB
:101B0000E8C9FF1F00B9FF1FEAC9FF1F0288FF1FB6
:101B1000B0C5FF1FDE8EFF1FDD8EFF1F00238BF879
:101B20000030AE4B1B781B09591CAD4B1A7899F845
:101B30000030120901329142C8BF002103F00F03A7
:101B4000618443EA0113DBB289F8003099F8001090
:101B50004FF4E47079E7E3832A780123B34022EA63
:101B60000303D3E694F822300133DBB2013293420F
:101B700008DDA08B297801228240002321EA02029D
:101B8000E3832A706384C9E6102B7DF4BFA9BAF100
:101B90004F0F21DCFB69632B0ADC924A182151723A
:101BA000BA691268FA6200238BF80030F96A0DE016
:101BB000FB698C2B7DF7AAA98A4A14215172BA6954
:101BC00012683A630023396B8BF80030864A116043
:101BD000864AFE20137045E6BAF1910F7DF796A96B
:101BE000FB69782B7DF792A97E4D002628468BF85D
:101BF0000060EEF7DEFE20236B72BB691B683B645E
:101C0000794B3A6C1A60794BFE201E70F3F7ECFAB0
